:020000040800F2
:10000000B06001200D020008651A0008D512000832
:10001000631A000801110008171B00080000000007
:10002000000000000000000000000000690100085E
:100030002102000800000000AD010008691A000854
:1000400027020008270200082702000827020008EC
:1000500027020008270200082702000827020008DC
:1000600027020008270200082702000827020008CC
:1000700027020008270200082702000827020008BC
:1000800027020008270200082702000827020008AC
:10009000270200082702000827020008270200089C
:1000A000270200082702000827020008270200088C
:1000B000270200082702000827020008270200087C
:1000C000270200082702000827020008270200086C
:1000D00027020008ED1A000827020008270200087E
:1000E000270200082702000827020008270200084C
:1000F000270200082702000827020008000000006D
:10010000270200080000000027020008270200085C
:100110002702000827020008C11A00082702000869
:10012000270200082702000827020008270200080B
:1001300027020008391100082702000827020008DA
:1001400027020008270200082702000827020008EB
:10015000DFF810D000F090FD00480047C5A9000866
:10016000AFF30080B0600120204B19680868B0E848
:10017000F00F80F30988BFF36F8F4FF0000080F31A
:1001800011884EF00D0E7047000000000648006810
:10019000006880F3088862B661B6BFF34F8FBFF383
:1001A0006F8F00DF00BF00BF08ED00E0EFF30980B4
:1001B000BFF36F8F0D4B1A6820E9F00F106008B580
:1001C0004FF0200080F3118817F0CCF84FF00000BA
:1001D00080F31188BDE8084019680868B0E8F00F9E
:1001E00080F30988BFF36F8F704700BF7C00002049
:1001F000EFF311804FF0200181F31188704780F3F5
:1002000011887047EFF3058070470000064880476B
:1002100006480047FEE7FEE7FEE7FEE7FEE7FEE7EB
:10022000FEE7FEE7FEE7FEE78D1A00085101000831
:100230002DE9F05F0546002092469B46884606461B
:10024000814640241BE0284641464746224600F0AE
:1002500039FA53465A46C01A914110D311461846EE
:10026000224600F020FA2D1A67EB01084F4622467D
:100270000120002100F017FA17EB00094E41201E63
:10028000A4F10104DFDC484631462A464346BDE876
:10029000F09F40EA01039B0703D009E008C9121F41
:1002A00008C0042AFAD203E011F8013B00F8013B30
:1002B000521EF9D27047D2B201E000F8012B491E5C
:1002C000FBD270470022F6E710B513460A460446F3
:1002D0001946FFF7F0FF204610BD421E12F8013FFD
:1002E000002BFBD111F8013B02F8013B002BF9D1A7
:1002F000704730B505462A460B4612F8010B13F835
:10030000014B08B1A042F8D01CB1002802D06D1CEE
:10031000F1E7284630BD421C10F8011B0029FBD133
:10032000801A704710B5002200E0521C835C8C5C80
:10033000A34201D1002BF8D1D8B2E1B2401A10BDCE
:1003400030B504460020034600E05B1C934203D214
:10035000E05CCD5C401BF8D030BD034611F8012BAA
:1003600000F8012B002AF9D11846704730B5054630
:100370000020034600E05B1C934205D2EC5CC85CA5
:10038000201A01D1002CF6D130BD00000FB400B509
:100390008DB010A909900B9000914FF0FF300A909A
:1003A00000200C9005480690054807906A4609A869
:1003B0000F9900F02BFA0DB05DF814FB2908000826
:1003C000470800082DE9FF5F1D464FF0FF3BD5E9C8
:1003D000014691465F464FF00008A9697F1C0198CD
:1003E0008847296A824688470028F6D1BAF1FF3F3C
:1003F0000CD024F4C064002E19DD600614D5BAF1C7
:100400002B0F09D0BAF12D0F0ED103E0584604B0DE
:10041000BDE8F09F44F48064A9697F1C0198884777
:10042000761E8246002E02DDBAF1300F03D0B9F1FC
:10043000000F26D032E0A969761E44F400747F1CB8
:10044000019888478246002E05DDBAF1780F06D064
:10045000BAF1580F03D0B9F1000F10D01EE0B9F176
:10046000000F02D0B9F1100F18D1A969761E24F43B
:1004700000747F1C019888478246102002E0082003
:1004800000E00A20814609E008FB0908A969761EF8
:1004900044F400747F1C019888478246002E05DDD5
:1004A0004946504600F09EF90028EDDAE9690198C6
:1004B0008847A00502D46FF00100A8E7E00725D126
:1004C000600613D5600502D5C8F1000000E0404683
:1004D00029680A1D2A600968220501D5087015E0FF
:1004E000220701D5088011E008600FE02868011D8F
:1004F00029600068210502D580F8008006E0210708
:1005000002D5A0F8008001E0C0F8008038467EE700
:100510002DE9FF5FD2E901A74FF0000891699946E4
:100520001446DDF838B0464601988847054659EA32
:100530000B0005D009E0A169761C019888470546A3
:10054000216A284688470028F5D1681C03D05FEA55
:10055000CA7005D015E04FF0FF3004B0BDE8F09F41
:100560002068011D2160D0F800800AE05FEACA70AF
:1005700001D108F8015BA169761C7F1E01988847AC
:100580000546002F1ADD681C18D0B9F1000F0DD0F8
:10059000E81705EBD060421120F01F0059F8221037
:1005A0002A1A012090400142E0D107E0BBF1000F80
:1005B000DCD1216A284688470028D7D0E169019814
:1005C0008847BBF1000F07D1002E05DD5FEACA7036
:1005D00002D1002188F80010A068B84203DDBBF109
:1005E000000F03D017B16FF00100B6E73046B4E753
:1005F0002DE9F04791460F4680460446002614F840
:10060000015B2DB100F06EF80068405DC007F6D1C7
:100610002B2D02D02D2D18D0641E4A463946204677
:1006200000F022F927B13968A14201D1C7F8008052
:1006300071054FF002040BD54042002803DD01F0A4
:10064000A9FA0460A007BDE8F08746F48066E4E7F5
:100650000028F8DA01F09EFA04606FF00040F2E73B
:1006600070B5064601F096FA046805460A22002194
:100670003046FFF7BDFF2C6070BD30B50B4601461C
:1006800000202022012409E021FA02F59D4205D331
:1006900003FA02F5491B04FA02F52844151EA2F1DB
:1006A0000102F1DC30BD202A04DB203A00FA02F11D
:1006B000002070479140C2F1200320FA03F3194350
:1006C00090407047202A04DB203A21FA02F00021F2
:1006D000704721FA02F3D040C2F120029140084352
:1006E0001946704700487047D086010810B5044687
:1006F000FFF7F8FF0068005D00F0010010BD00008A
:1007000007280FD2DFE800F00406080E0E0C0A00DE
:1007100005A070470AA0704713A070471DA070473E
:1007200022A070472BA070474E6F206572726F72C7
:1007300020286572726E6F203D2030290000000075
:1007400045444F4D202D2066756E6374696F6E2091
:10075000617267756D656E74206F7574206F6620A9
:1007600072616E67650000004552414E4745202D7D
:100770002066756E6374696F6E20726573756C7434
:10078000206E6F7420726570726573656E7461623D
:100790006C650000454E4F4D454D202D206F757402
:1007A000206F66206D656D6F7279000045494E5669
:1007B000414C202D20696E76616C696420617267FE
:1007C000756D656E7420746F2066756E6374696FE5
:1007D0006E000000556E6B6E6F776E206572726FE3
:1007E000720000003A2800D2303820F02002412A5E
:1007F00001D3A2F13700884201D34FF0FF30704798
:10080000026811441378016018467047D1600449AA
:1008100051610449116200211161114600F050BA82
:1008200001080008ED060008426842B1016811F8AD
:10083000013B23B1521EC0E9001218467047012146
:10084000C160881E704742685AB1C368016843B9E5
:1008500083688B4205D0491E521CC0E9001200205B
:1008600070474FF0FF3070472DE9F05F8246007807
:10087000002715468B460AF10104B946302801D0FD
:100880009DB113E014F8010B0127782803D05828F4
:1008900001D045B10AE00DB1102D07D10027102578
:1008A00014F8010B02E0082500E00A250026B046F6
:1008B0000EE005FB080005FB06F1012701EB1046E1
:1008C0001FFA80F8B6F5803F00D3B94614F8010B43
:1008D0002946FFF787FF0028EBDABBF1000F05D0B0
:1008E0000FB1641E00E05446CBF80040B9F1000F90
:1008F00006D001F04FF902210160C81EBDE8F09F4B
:1009000048EA0640FAE72DE9FE4F804681EA0300F7
:10091000C00F0C46009021F0004123F00045B8EBD9
:100920000200A94105D24046214690461C460B468E
:10093000024623F00040104347D0270DC7F30A00BA
:10094000C3F30A510290401A019040286BDAC3F3B6
:10095000130040F4801B0098924620B10023D2EB94
:10096000030A63EB0B0B01985946C0F14002504655
:10097000FFF799FE06460D4650465946019A00F08B
:100980008DF910EB08006141002487EA115284EAD6
:10099000E7731A4340D0009A62B3019A012A4FEAE2
:1009A000075215DC001B61EB02014FF0004202EA26
:1009B0000752CDE90042001C41F5801132462B461A
:1009C00000F025FB03B0BDE8F08F40462146F9E773
:1009D000001B61EB0201001C41F5801300185B4114
:1009E0002018A2F5001747EB030140EAD570B619AD
:1009F0006D4111E06D084FEA360645EAC0754FEAD1
:100A00000752001B61EB0201001C41F580114908EF
:100A10004FEA30000019514132462B4603B0BDE881
:100A2000F04F00F0E5BA0098012240000023D0EB1F
:100A3000020263EBE073009821464FEAE074B8EBE2
:100A4000000061EB0401E9E783F000435BE781F01C
:100A5000004158E72DE9FE4F81EA030404F0004409
:100A600021F0004100944FF0000B23F0004350EAC6
:100A700001045ED052EA03045BD0C3F30A54C1F30D
:100A80000A552C44A4F2F3340194A0FB0254C1F3A0
:100A9000130141F48011C3F3130343F4801301FBEA
:100AA000024400FB034E840A970A44EA815447EA51
:100AB0008357A4FB076802958D0A05FB07854FEA5B
:100AC000932C04FB0C542705029D4FEA065847EA75
:100AD0001637B5EB08056EEB070C870E920E47EA4A
:100AE000811742EA8312A7FB0201B6EB0B0164EB0C
:100AF00000042B0D43EA0C335E1844EB1C50DA461D
:100B00005146E7FB0201C5F313044FEA0B3343EAF6
:100B100014534FEA0432019C43EA0603A4F10C0487
:100B20000294009CCDE900B400F071FA03B0BDE876
:100B3000F08F00200146F9E72DE9F04D81EA03042A
:100B400004F0004B21F0004514464FF0000A23F05A
:100B5000004150EA050220D054EA01021DD0C5F33D
:100B60000A570246C5F31303C1F31300C1F30A5633
:100B700040F4801543F48013A7EB0608101BD646FB
:100B800008F2FD3873EB050002D308F1010801E01B
:100B900092185B41B8F1000F03DA00200146BDE86E
:100BA000F08D00204FF48011064684460EE0171B9E
:100BB00073EB050705D3121B63EB050306434CEAF1
:100BC000010C49084FEA300092185B4150EA0107D6
:100BD000EDD152EA030012D082EA040083EA050153
:100BE000084305D0101BAB4106D20122002306E0CA
:100BF00000224FF0004302E06FF0010253101AEBA5
:100C000006004CEB085110EB0A0041EB0B01BDE86C
:100C1000F04D00F0EDB9C1F30A52C1F3130140F2F7
:100C2000FF3341F480119A4202DA002001467047F6
:100C300040F233439A42A2F2334202DC5242FFF7BF
:100C400041BDFFF730BD000030B5041E71F1000456
:100C500004DB4FF00044404264EB0101141E73F1C9
:100C6000000405DB1C464FF00043524263EB0403D3
:100C7000994208BF904230BD064C074D06E0E0683F
:100C800040F0010394E8070098471034AC42F6D3D3
:100C9000FFF762FA588B0108788B0108202A06DBDF
:100CA000CB17203A41FA02F043EAE07306E041FA3A
:100CB00002F3D040C2F12002914008431946704728
:100CC0002DE9F34F8BB04FF0000801F10C000C46FA
:100CD0004FF0010B46460DF1080A019062690121AF
:100CE00001989047051E2DD0252D2CD0216A8847CC
:100CF000C0B16269012101989047216A88470028A4
:100D0000F7D1411E62690198904700E0761CA16905
:100D10000B988847216A88470028F7D1E1690B982A
:100D20008847DBE7A1690B9888470746A84201D1AD
:100D3000761CD3E7E1690B9888477F1C02D1B8F194
:100D4000000F6FD047E1002762693D4639460198A0
:100D500090472A2804D16269012101989047012512
:100D6000DFF888926269012101989047A0F1300173
:100D70000A290AD24F45E5DC07EB870100EB410762
:100D8000303FDFD445F01005ECE7E90601D46FF001
:100D900000476C280AD04C2814D0682815D06A283F
:100DA0000DD074281CD07A281AD01DE06269012168
:100DB000019890476C2802D045F0040514E045F0F6
:100DC00002050DE045F020050AE062690121019865
:100DD0009047682802D045F0080505E045F4006515
:100DE0006269012101989047C4E9015765283DD007
:100DF00019DC58287AD00CDC452837D004DC2528AB
:100E000026D0412831D131E046282FD047282CD197
:100E10002CE05B2877D0612828D063287CD0642818
:100E200023D15AE0D1E06F2848D008DC66281DD0D5
:100E300067281BD0692821D06E2816D127E070289A
:100E400045D0732868D0752847D078280DD14DE05B
:100E5000A1690B988847054625283FF469AFE169E9
:100E60000B9888476D1C3FF46AAFB4E023466A468E
:100E70006FF001000B99AFF300809FE045F0400058
:100E80006060A80723464FF0000236D43EE0E80732
:100E90007FF447AF2068011D21600068290501D556
:100EA00006701BE7290701D5068017E7A90703D5B8
:100EB000F117C0E9006111E706600FE745F0400057
:100EC0006060A80723464FF0080216D41EE040F6E3
:100ED0000E0125EA0100606016E045F04000606008
:100EE000A80723464FF00A0207D40FE045F0400060
:100EF0006060A80708D5234610226FF001000B9907
:100F0000AFF300805AE007E0234610226FF00100A3
:100F10000B99FFF757FA51E04FF000094F464B4647
:100F2000632802D05B2807D041E02079C00601D4B5
:100F30000120A06001273AE06269012101989047F1
:100F40005E2805D14FF00109626949460198904732
:100F5000216939B900210A46534643F82120491C2A
:100F60000829FADBB0B3216969B9C11700EBD16276
:100F700053110AEB830122F01F02821A01200B6831
:100F8000904003430B6062690121019890475D28FE
:100F9000E8D1B9F1000F09D00020514651F82020C6
:100FA000D24341F82020401C0828F7DB02AB224640
:100FB00000976FF001000B99FFF7AAFA00280CDAEE
:100FC000401C08D1BBF1000F05D04FF0FF300DB031
:100FD000BDE8F08FFFE74046F9E7E90701D108F1E6
:100FE000010806444FF0000B78E60000CCCCCC0C96
:100FF00010B5141E73F1000408DA401C41F1000121
:1010000092185B411A4301D120F0010010BD2DE977
:10101000F04D92469B4611B1B1FA81F202E0B0FA6E
:1010200080F220329046FFF73EFB04460F4640EA2E
:101030000A0041EA0B0153465A46084313D01146B1
:1010400053EA010019D0C8F140025046FFF73AFBBD
:1010500005460E46504659464246FFF724FB0843D4
:1010600005D0012004E020463946BDE8F08D00207F
:10107000054346EAE0762C4337430A986305E40AC1
:10108000A0EB08000022FD0A44EA47540A3002D5CA
:1010900000200146E9E7010510196941DDE908452D
:1010A00000196941BDE8F04DA2E770B58C1810F841
:1010B000015B15F0070301D110F8013B2A1106D19D
:1010C00010F8012B03E010F8016B01F8016B5B1EB7
:1010D000F9D12B0705D40023521E0DD401F8013B92
:1010E000FAE710F8013BCB1A921C03E013F8015BFE
:1010F00001F8015B521EF9D5A142D8D3002070BD82
:10110000FEE7000030B502464FF6FF70064D07E0DF
:1011100012F8013B4340DBB2040A35F8130060408B
:10112000491E89B2F4D230BDB67E010801490020C3
:10113000087070475C00002038B500200090094C12
:10114000204605F0C5FD012804D10748694600681E
:1011500016F049FC204605F0AFFD02480A3005F0C4
:10116000ABFD38BD06050400A001002038B5012202
:101170006B461146002005F059FE012803D1BDF849
:10118000000000F00404154D2868C00716D0286838
:10119000C00609D5002C06D111480DF09FFC286827
:1011A00020F01000286038BD002CFCD00C480DF059
:1011B000A2FC286840F01000286038BD002CFCD04C
:1011C000074808F01FFB06480DF095FC286840F022
:1011D00001002860024803F05BF938BD5800002088
:1011E0007C09002010B50120FFF7C0FF0022AFF2FC
:1011F0000B01BDE810404FF47A7010F097BC00006E
:101200001CB50021019190F83100C0061BD512A039
:1012100000F082FC144C01226B461146002005F0C0
:1012200005FEBDF8000000F0200000900199491C67
:10123000019110B90198A042EDD305F046FA0B4890
:101240000DF081FC1CBD0AA000F066FC05F036FA2A
:1012500006480DF0F5FB1CBD6E6574776F726B2050
:101260006973207570000000FFFF04007C090020F6
:101270006E6574776F726B20697320646F776E0090
:1012800070B505460E4607F013F80024ED0207E09E
:1012900005EBC42000F1006006F0B0FF641CA4B2AE
:1012A000B442F5D3BDE8704006F094BF70B5064671
:1012B0000C46154606F0FCFF06E03046216807F0B4
:1012C00013F82D1F361D241D002DF6D1BDE87040EA
:1012D00006F080BF002007F063F9FEE72DE9F0413A
:1012E000ADF5A26D0446884615461E462C4F0023D8
:1012F0004FF47A721946386816F027FA00284BD056
:1013000015F034FA0DF22C534FF480710DF20C40AD
:10131000DDF8282500F024FC0020CDF80C050DF2A6
:101320000C40012C06D0022C0ED0032C16D0042C1D
:1013300027D11DE0CDE900560290434619A21BA11A
:1013400003A800F0F9FB1CE0CDE9005602904346EB
:101350001CA216A103A800F0EFFB12E0CDE9005695
:101360000290434619A211A103A800F0E5FB08E092
:10137000CDE900560290434616A20CA103A800F046
:10138000DBFB03A815F09CFA15F0E4F900231A46DC
:101390001946386816F08AFA0DF5A26DBDE8F0819D
:1013A00010000020494E464F000000005B25735D91
:1013B0005B25735D5B25733A2534645D2025730DD1
:1013C0000A00000044454255470000005741524E74
:1013D000000000004552524F52000000FEB5054685
:1013E0000C46164600200290019301A80FF0E4FB82
:1013F0008DF808000298C0F3C00020700298C0F376
:10140000031028706946019800F0F8F8019901442A
:101410000191009A8B18591A022904DB01A80FF0D8
:10142000D1FB30800120FEBD7FB505460E46002071
:10143000039002920024009002A80FF0BDFB8DF8EB
:101440000C000398C0F3031002281AD101A90298D6
:1014500000F0D4F802990446421802920198104410
:10146000801A02280DDB02A80FF0A6FB8DF8000001
:10147000009800F00100287002A80FF09DFB30706A
:10148000012404B0204670BD2DE9FE4F0D46DDE974
:101490000C97DDE90E81044693461E46002002901B
:1014A00001918246009001A80FF086FB8DF808009C
:1014B0000298C0F3031103292DD1C0F3C00020709E
:1014C0000298C0F341002860029800F001008BF8F8
:1014D00000006946019800F091F80199824608449D
:1014E000019000994418224601A948460FF073FB69
:1014F00088B10198201A0ED42868002803DD01A8BD
:101500000FF060FB30800198201AC8F800000198A5
:1015100038604FF0010A5046BDE8FE8F2DE9FE4FBE
:1015200082460C980E4614461F464FF00009CDF82F
:1015300008900190C84601A80FF03EFB8DF8080006
:101540000298C0F30310092827D16946019800F0DA
:1015500055F8019980460844019000994518281AC9
:1015600002281ADB01A80FF02DFBAAF80000C4F82E
:1015700000900DE02068B04202DD4FF0FF380CE033
:1015800001A80FF019FB2268511C216047F82200C6
:101590000198A842EED34FF001084046BDE8FE8F07
:1015A0003EB500240294019400920B46024601A924
:1015B00002A8FFF713FF9DF808100B2900D10120A6
:1015C0003EBDF8B507460E460124002500203060D8
:1015D0006D1C042D0FDC01216846B84701280AD193
:1015E0009DF80020306802F07F0101FB04003060AC
:1015F000E4011006ECD42846F8BD0000024A106051
:101600000248FFF7DEBF0000AC010020252C0008D7
:1016100010B504460020CA1701EB526323F07F0285
:10162000891ACAB2D911002901DD42F080020346AD
:1016300000F10100E254EEDC10BD70B502460E462A
:101640001068002804D00546FEF765FE044601E058
:10165000956854683046FEF75EFE844205D1224606
:1016600031462846FEF782FE08B1002070BD0120F9
:1016700070BD0000401C802801DA401C7047B0F5A6
:10168000804F01DA801C70470349884201DAC01C90
:101690007047001D70470000FFFF1F007CB5054626
:1016A000069E002401940095042901DAA01E7CBD49
:1016B00062F3071463F3C3040194062A15D024F0DF
:1016C000060201929DF80410684615F0CFFE022133
:1016D0000098FFF79DFF0099084400903146684646
:1016E00015F0CAFE0098401B7CBD24F00602921C37
:1016F000E7E700002DE9FE4305460F461446029534
:10170000002601960096204600F092F88046FFF7EA
:10171000B1FFB84202DDB01EBDE8FE838DF8046063
:10172000019820F0F000103001909DF8041002A8FC
:1017300015F09CFE41460298FFF76AFF02990844A3
:101740000290207A042813D035A102A815F07AFE61
:10175000032102A815F08AFE8DF80060A17E009892
:1017600061F341000090E17E59B140F004000AE0CD
:101770002DA102A815F066FE042102A815F076FE40
:10178000EAE720F004000090410708D594F83D10E6
:1017900061F3C40094F83C1061F345100090206C94
:1017A00008B9A06C18B1009840F080000090E06C7F
:1017B00008B9606D18B1009840F0400000909DF8A5
:1017C000001002A815F052FE218B02A815F054FE5D
:1017D000D4E9042302A8E16815F05DFEE07E58B16B
:1017E000D4E90A2302A8616A15F055FED4E90D2355
:1017F00002A8216B15F04FFE009E300605D5D4E9F6
:10180000112302A8216C15F046FE700604D54C3455
:1018100002A80ECC15F03FFE0298401B7CE70000AA
:101820004D514973647000004D5154540000000044
:1018300070B504460025207A032802D0042802D07F
:1018400002E00C2500E00A25D4E90412E06800F06B
:10185000FDF80544AD1CE07E68B1D4E90A12606A67
:1018600000F0F4F8D4E90D120646206B00F0EEF813
:10187000304405442D1D206C08B9A16C29B1D4E970
:10188000111200F0E3F80544AD1CE06C08B9616D7D
:1018900029B1D4E9141200F0D9F80544AD1C28464A
:1018A00070BD0E2200F0B5B80C2200F0B2B82DE9E0
:1018B000FE4F0546DDE90C9A129E0F4690461C46E7
:1018C0000295002001900EA900960EC9204600F056
:1018D00032F88346FFF7CEFEB84203DD6FF0010019
:1018E000BDE8FE8F302068F3C30064F3420069F363
:1018F000000001909DF8041002A815F0B7FD5946AC
:101900000298FFF785FE0299084402900EA902A8EA
:101910000EC915F0C0FD002C03DD514602A815F0DC
:10192000ABFD324611990298FEF7B3FC02983044A1
:101930000290401BD4E77FB50546089C01A807C864
:1019400000F084F82044801C002D00DD801C04B0D1
:1019500070BD2DE9FF4F83B00646DDE91189109F68
:101960008A46934602960025019500244146384652
:1019700000F039F80090FFF77DFE504503DDA01E12
:1019800007B0BDE8F08F8DF80450019820F0F0000A
:1019900080306BF3C30020F00600801C01909DF89E
:1019A000041002A815F062FD00990298FFF730FEBE
:1019B00002990844029002A8069915F05DFD0DE019
:1019C00004EB440008EB800502A80ECD15F063FD82
:1019D00019F8241002A815F049FD641CBC42EFDB85
:1019E0000298801BCCE72DE9F04106460F46022500
:1019F000002409E004EB440007EB800307CB00F070
:101A000025F80544ED1C641CB442F3DB2846BDE810
:101A1000F0811CB50446002001900094022901DAEF
:101A2000801E1CBD8DF80400019862F30710019020
:101A30009DF80410684615F019FD00210098FFF785
:101A4000E7FD009901440091081B1CBD17B40098E4
:101A5000002803D000981EBCFEF75DBC01981EBC98
:101A60007047FEE77047000010B5FEF7C1FB16F0A7
:101A70008BF818B104494FF080500860BDE8104061
:101A80000020FEF7BCBB000004ED00E00A4801683E
:101A900041F00101016000214160C1620168074A13
:101AA000114001604FF47F018160016821F48021C1
:101AB000016010F0A7B9000000100240FFFFF6EA35
:101AC00010B5084C0121204614F031FB002807D046
:101AD0000121204614F028FB03480168491C0160DD
:101AE00010BD0000001000406400002010B506F09A
:101AF0001DFED0F8E800407D032807D0012801D062
:101B0000022807D1BDE8104003F0B0BABDE810408C
:101B100009F09EBB10BDFEE70FB4054B10B503A93D
:101B2000044A029800F022F910BC5DF814FB000092
:101B300081830008D40100200FB4084B10B504A91C
:101B400002AA039800F012F9044602A9002000F04E
:101B50009BFC204610BC5DF814FB000089240008A3
:101B60007CB50C001D461646014601D0601E00E003
:101B70000020CDE90010064B6A462946304600F0A9
:101B8000F5F8002C02D0009A002111707CBD0000F5
:101B90007324000800487047E401002002E008C8F0
:101BA000121F08C1002AFAD170477047002001E0D7
:101BB00001C1121F002AFBD17047002203E010F878
:101BC000013B1A44D2B2491E4B1CF8D11046704753
:101BD0002DE9FF5F82B00021DDE90430020DDDF860
:101BE00040B0034318D044F61050A2F2FF324243F3
:101BF0001514119801281FD0A5EB0B00401C5FEABB
:101C0000000A4FF000064E4FDFF83891B0465046BC
:101C100015D5CAF1000413E0119801244AA3012844
:101C200001D16FEA0B010298119AC0E90031C0E9B5
:101C3000024206B0BDE8F09FCBF10000DFE70446AA
:101C40000021404A491842EB0450CDE9001012E04F
:101C5000E00707D032463B4640464946FEF7FAFECB
:101C60008046894632463B4610461946FEF7F2FE4C
:101C700006460F466410002CEAD1DDE90401DDE9D7
:101C80000023BAF1000F06DAFEF7E4FE42464B46A7
:101C9000FEF7E0FE05E0FEF74FFF42464B46FEF73B
:101CA0004BFF04460E460022284BFEF7CDFF03D81B
:101CB0004FF0FF30014607E00022254B2046314619
:101CC000FEF721FEFEF7A7FF102409E0002C0ADB37
:101CD0000A220023FEF7ACFA039B30321A55641E29
:101CE00050EA0102F2D1641C039AC4F111031444B6
:101CF000119A012A03D0012208430DD10AE00843BA
:101D000004D000204FF0110B119072E7A3EB0B05EC
:101D10006D1E0DE05B4504DD4FF0000205F101058D
:101D200004E003DA4FF00002A5F10105002AECD02F
:101D300002981199C0E90231C0E9004579E7000035
:101D4000000014400000F03F300000000000F043AD
:101D50000000E03F506002604160086070474860EA
:101D600001607047D0E90010FFF7F9BF2DE9FF4F80
:101D700095B09A46884606460025EEE1252877D19B
:101D800000242746F94A0121039400E0044316F891
:101D9000013F203B01FA03F01042F7D130782A28A6
:101DA00011D06FF02F033078A0F13002092A16D835
:101DB000039A44F0020402EB820203EB4202104455
:101DC000761C0390EFE758F8042B0392002A03DAFD
:101DD000504244F40054039044F00204761C3078DE
:101DE0002E2816D116F8010F44F004042A280DD02D
:101DF0006FF02F023078A0F13003092B09D807EBE0
:101E0000870302EB4303C718761CF3E758F8047BFB
:101E1000761C30786C280FD006DC4C2817D0682848
:101E20000DD06A2814D104E0742810D07A280FD17C
:101E30000DE044F400140AE044F4801401E044F49A
:101E400040147278824202D104F58014761C761C0C
:101E5000307866280BD013DC582877D009DC0028AE
:101E600075D04528F6D04628F4D047281AD193E1FA
:101E700018E0632835D0642879D0652812D18BE129
:101E8000702873D008DC6728F1D069286FD06E28DD
:101E90000DD06F2806D1ACE073282CD0752874D0F3
:101EA000782853D05246179990476D1C54E1C4F3DB
:101EB0000250022809D003280DD0D8F800100428B9
:101EC0000DD00D6008F1040846E1D8F80010EA17BB
:101ED000C1E90052F6E7D8F800100D80F2E70D7066
:101EE000F0E718F8041B8DF8001000208DF80100B1
:101EF000EB46012003E058F804BB4FF0FF306107C8
:101F00004FF0000102D40DE009F101018946B94208
:101F10000FDA8145F8DB1BF809100029F4D108E03D
:101F200009F1010189468142FADB1BF809100029F9
:101F3000F6D103985346A0EB090721463846179A75
:101F400000F080FA284400EB090507E044E008E1CE
:101F50000DE01BF8010B524617999047B9F10109A2
:101F6000F7D2534621463846179AF2E039E00A2163
:101F7000C4F302524FF0000B0091022A06D058F829
:101F8000040BC117032A09D00AE023E008F1070077
:101F900020F00702F2E80201904605E000B2C11706
:101FA000042A01D140B2C117002906DA0A460021ED
:101FB000404261EB02012D2202E0220504D52B22D2
:101FC0008DF80420012203E0E20701D02022F7E788
:101FD000914657E00A2100E010214FF0000B0091DC
:101FE0000BE010214FF0000B44F00404082700918F
:101FF00003E008204FF0000B0090C4F30252022AC5
:1020000005D058F8040B0021032A08D008E008F195
:10201000070020F00702F2E80201904603E080B2D8
:10202000042A00D1C0B24FF0000922072AD5327825
:10203000702A07D0DDF800C08CF0100C5CEA0B0CA5
:1020400005D00EE040228DF80420012208E050EA7D
:10205000010306D030238DF804308DF805200222CC
:102060009146009B83F0080353EA0B030AD150EA20
:10207000010201D1620705D530228DF804204FF00E
:1020800001097F1E3278582A04D039A20C920CAA7A
:1020900002920BE03BA2F9E75B46009AFEF7C8F814
:1020A0000C9B9B5C029A521E0292137050EA010232
:1020B000F2D1029804A9081A00F1200B600702D59A
:1020C00024F4803400E001275F4502DDA7EB0B001C
:1020D00000E0002000EB0B01009003984944401AF7
:1020E0000390E00306D453462146179A039800F064
:1020F000A9F90544002706E001A85246C05D1799DA
:1021000090476D1C7F1C4F45F6DBE0030CD5534612
:102110002146179A039800F095F9054404E0302011
:102120005246179990476D1C0099481E009000294F
:10213000F5DC08E00298029952460078491C0291A9
:10214000179990476D1CBBF10001ABF1010BF1DC5D
:102150005BE100F065F90544761C307800287FF4D7
:102160000DAE19B02846BDE8F08F00000928010027
:1021700030313233343536373839616263646566FD
:1021800000000000303132333435363738394142BF
:102190004344454600000000600700D4062708F1CC
:1021A000070020F00700F0E80223804603F0004C0F
:1021B0005FEA0C0001D097A009E0200501D596A0A8
:1021C00005E0E00701D095A001E0AFF24C001390CC
:1021D000307823F0004365280CD006DC452809D070
:1021E00046281DD047287FD13BE0662818D06728B5
:1021F0007AD136E00021112F01DB112000E0781C9C
:10220000CDE9000104A90CA8FFF7E2FCDDE90D010E
:102210000C9A4FF0000B07F10109109200914EE06B
:102220004FF000400097CDE9011004A90CA8FFF77A
:10223000CFFCDDE90D020C9B0F994FF0000B91468E
:102240001093009211B9791C00EB0109B7EB09005A
:1022500003D4C0F1FF3B07F10109A9EB070001908E
:1022600042E0012F00DA01270021112F01DD1120AA
:1022700000E03846CDE9000104A90CA8FFF7A8FC4E
:10228000DDE90D010C9A00914FF0000BB946109258
:1022900021070FD4009A4A4503DA914601E0A9F1DB
:1022A0000109B9F1010F05DD109AA9F10101515C95
:1022B0003029F4D0B84202DA10F1040F03DA012118
:1022C000CDE9011010E0002803DC8344A9EB0001F4
:1022D00002E0411C494500DD8946A0EB0B00401C93
:1022E00001904FF000400290200705D40198484526
:1022F00002DB4FF0FF30019000208DF84B00029878
:102300000DF14B07B0F1004F25D002200C902B208F
:102310000D90029800280CDA404202902D200D907A
:1023200007E00A210298FEF7A8F93031029007F879
:10233000011D0C99481E0C900029F2DC029800281F
:10234000EFD1791E0D980870307800F0200040F031
:10235000450007F8020D11A8C01BC01D029013987C
:10236000007800B1012000EB0901019801EBE07158
:10237000029801440398401A401E0390E00306D4DB
:1023800053462146179A039800F05CF805441398C9
:10239000007818B15246179990476D1CE00323D579
:1023A00053462146179A039800F04CF805441BE069
:1023B000BBF1000F07DB0098584504DD1098179912
:1023C00010F80B0001E01799302052469047019811
:1023D0000BF1010B401E05F10105019004D12E20E7
:1023E0005246179990476D1CB9F10001A9F10109F6
:1023F000DEDC05E017F8010B5246179990476D1C7B
:102400000299481E02900029F4DC53462146179A8F
:1024100003989EE62D0000002B0000002000000025
:102420002DE9F041044600251E461746880404D4D1
:1024300005E039462020B0476D1C641EF9D52846BA
:10244000BDE8F0812DE9F041044600251E46904686
:10245000C80301D5302700E02027880404D505E013
:1024600041463846B0476D1C641EF9D52846BDE884
:10247000F0814A68002A06D00A68531C0B6010706D
:102480004868401E486070470A68531C0B60107013
:1024900070472DE9F04705460E46174605F1140032
:1024A00080460FF0E9FAB8B32878E96A0BF0CAFA67
:1024B00004464FF0FF3984B3666020460FF018FAE7
:1024C0002772214640460FF0C9FA38B365680021EB
:1024D00028460FF083FD0021284611F0B1FF0021AE
:1024E000284612F0DFF904220021284611F030F9C5
:1024F0000021284610F03EF90020606004F1100031
:1025000005460FF083FA28460FF0A5FA20460BF097
:1025100035FC4846BDE8F08701E003E004E06FF0D9
:102520000500F7E74846F5E7EB6A1BB100221146C4
:10253000284698470020EDE770B506460D46242052
:102540000EF038F8044624212046FDF7BBFE621D3C
:1025500011A130460CF0D6FB13A130460CF0B8FBAD
:10256000E07016A130460CF0B3FBA07017A1304606
:102570000CF0AEFB60831AA130460CF0A9FB208062
:10258000A969486810B94C6070BD0846016A002905
:10259000FBD1046270BD0000226964656E746966D7
:1025A000696572223A220000227746756E6374696B
:1025B0006F6E436F6465223A0000000022736C6105
:1025C000766541646472657373223A0022726567AE
:1025D000697374657241646472657373223A0000B2
:1025E000227265676973746572427974654E756DA0
:1025F000223A00002DE9F041074620200DF0DAFFD5
:1026000004460025E5612FA138460CF061FB60759A
:102610002FA138460CF05CFBE07530A138460CF079
:1026200057FBA075621C32A138460CF06BFB0C20E6
:102630000DF0C0FFA06105604560856030A138469F
:10264000FDF757FE054641262146284600F02AF9A7
:102650002FA12846FDF74DFE00F8016B05462878AE
:102660005D28F1D1607D03281DD11CA138460CF0F6
:102670002FFBA07516A138460CF02AFBE07525A1AA
:102680003846FDF736FE05466DB121462846FFF770
:1026900053FF1FA12846FDF72CFE00F8016B0546ED
:1026A00028785D28F1D11F49D1F8E80020B9C1F898
:1026B000E840BDE8F0810846C1690029FBD1C4614A
:1026C000F7E700002270726F746F636F6C223A003C
:1026D000226461746154797065223A0022626967EC
:1026E0004C6974746C65466F726D6174223A0000B7
:1026F000226465766963654964223A22000000001D
:102700002273656E736F7244617461223A5B0000DC
:102710007D00000022636F6D6D616E6444617461C1
:10272000223A5B008408002070B505462DA128469A
:102730000CF0CEFA2D4C24F8BE0C2DA128460CF03E
:10274000C7FAA0772DA128460CF0C2FA20772EA157
:1027500028460CF0BDFAA0612EA128460CF0B8FA6C
:1027600060772FA128460CF0B3FA44F8100CD43C43
:10277000621C2FA128460CF0C5FA04F1A4022FA177
:1027800028460CF0BFFA04F14A0230A128460CF0AA
:10279000B9FA04F1180232A128460CF0B3FA04F198
:1027A0007C0234A128460CF0ADFA04F1900235A168
:1027B00028460CF0A7FA37A12846FDF79AFD0446F3
:1027C0004125002C0CD02046FFF714FF34A12046F1
:1027D000FDF78FFD00F8015B044620785D28F0D1FD
:1027E00070BD000022706F7274223A0058090020F8
:1027F0002273746F70426974223A0000226461741B
:1028000061426974223A00002262617564726174E7
:1028100065223A0022636865636B426974223A005C
:1028200022696E626F756E6454696D65223A0000AC
:1028300022686F7374223A220000000022646576D9
:102840006963654964223A220000000022636F6DCB
:102850006D616E64546F706963223A22000000005B
:10286000226D657373616765546F706963223A22E4
:102870000000000022757365726E616D65223A2258
:10288000000000002270617373776F7264223A2235
:10289000000000006465766963654C69737400002C
:1028A0007D0000002DE9F84380460F46787D012821
:1028B0002FD002282DD0032856D128200DF07AFEE3
:1028C000044628212046FDF7FDFCA21C2EA140460F
:1028D0000CF018FA30A140460CF0FAF984F8220006
:1028E00030A140460CF0F4F9607033A140460CF082
:1028F000EFF9207034A140460CF0EAF9E08237A1EC
:1029000040460CF0E5F92084B9690868002833D006
:1029100035E030200DF04EFE054635A140460CF066
:10292000D7F9E861AA1D18A140460CF0EBF90D207B
:102930000DF040FE0646324632A140460CF0E2F968
:10294000002406EB44006A4632A1FDF71FFD9DF806
:1029500000002855641C062CF3DB304614F0BAFA4C
:10296000B969886818B98D60BDE8F8830846C16AFE
:102970000029FBD1C562F7E70C60F5E70846416A1C
:102980000029FBD14462EFE7226964656E746966D1
:10299000696572223A22000022707265636973656C
:1029A000223A0000227246756E6374696F6E436F3F
:1029B0006465223A0000000022736C617665416410
:1029C0006472657373223A00227265676973746575
:1029D0007241646472657373223A00002272656703
:1029E0006973746572427974654E756D223A0000A0
:1029F000226964656E746966696572363435223A97
:102A00000000000022646576696365494436343508
:102A1000223A2200253268687800000070B5054629
:102A20000C4605F083FED0F8E80000E0C0690028FD
:102A3000FCD12046FFF7DEFD20200DF0BBFD044653
:102A40002046FDF768FC01462046FDF73BFC07A445
:102A50002046FDF760FC024600232146284607F089
:102A60009FFC2046BDE8704014F034BA7B22777298
:102A70006974655F636F6E666967223A2265727278
:102A80006F72227D000000002DE9F04105460E46E0
:102A90000024164F0EF088FF04EB440157F8311064
:102AA00041B10EF0ABFF641C042CF3DB4FF0FF30A0
:102AB000BDE8F08104EB440847F838500EF09EFF63
:102AC00007EBC80000224260028142812978102968
:102AD00006D001218181C281026142612046E7E77F
:102AE0000EB10121F6E70021F4E700005C3E012071
:102AF0007CB50546089E0C4621A13046FDF7F9FB42
:102B000098B1FEF713FB20200DF054FD21A42046C0
:102B1000FDF701FC024600232146284607F040FC51
:102B20002046BDE87C4014F0D5B920A13046FDF721
:102B3000E0FB002823D030460EF0FCFD204A21A106
:102B400030460CF0DFF81E4A21A1143230460CF05A
:102B5000D9F81B4A22A1283230460CF0D3F86A4635
:102B600024A130460CF0CEF86846FDF779FD144AF2
:102B70009087204607F0C6F82249012008707CBDE6
:102B800022646863704D6F6465223A226F70656ECF
:102B9000220000007B2269705F636F6E66696722A6
:102BA0003A2273756363657373227D0022646863E0
:102BB000704D6F6465223A22636C6F73652200006A
:102BC000340800202269707634223A220000000086
:102BD000227375626E65744D61736B223A22000038
:102BE0002264656661756C744761746577617922EA
:102BF0003A220000227564704C6F67506F72742225
:102C00003A2200000C00002010B504F0F9FFBDE8E6
:102C100010400022024941F288300EF087BF0000C8
:102C2000092C000870B5054608460022054C05E051
:102C3000236813F8016B2E702360521C8242F7DB6D
:102C400070BD0000AC01002030B5002306E0C45C7C
:102C5000CD5CAC4201D0012030BD5B1C9342F6DB61
:102C6000002030BD2DE9F0470746089E894698466A
:102C7000002E02D0521CD5B200E0154600221146AB
:102C800025200BF0C1FF40F202600DF06BFF40F217
:102C90000E600DF067FFDFF8B0A04FF40073032261
:102CA0001821504605F06EFD4FF480642346032240
:102CB0000421504605F066FD4946384613F08EFF64
:102CC000092D38D00021384614F051F8B8F1020F20
:102CD00034D00021384614F038F8012E31D0022EBD
:102CE00000D000242146384614F01DF80021384653
:102CF00013F0D9FF0021384613F0CBFF04213846EA
:102D000014F019F80821384614F027F8384613F063
:102D1000A5FF0BF066FF40F20531384613F0D7FFF0
:102D20004FF44171384613F0D2FFBDE8F047062159
:102D3000064813F098BF4FF48051C4E74FF4005198
:102D4000C8E74FF4C064CDE70008014000380140F7
:102D50002DE9F04180460F4600240026002525E09D
:102D60000122012A02D0022A1CD10EE021460A20AB
:102D70000AF0F2FC18F80610C91E01F00F0101FB61
:102D80000055641CE4B202220CE021460A200AF03D
:102D9000E3FC18F806103339091101FB0055641CD7
:102DA000E4B20022002ADCD1761CF6B27F1EBFB24C
:102DB000D6D22846BDE8F0812DE9F047012002F087
:102DC000E5F8012008F09EFA304D314C02E0642015
:102DD00014F014F9287821780843F8D04FF42050E3
:102DE0000DF0E8FB04462046FDF795FA0146204623
:102DF000FDF768FA14F054F820460DF007FF20465E
:102E0000FFF792FC204614F065F814F057F805F02F
:102E10008DFC0746D7F8E8404FF4806528460DF052
:102E2000C9FB804628460DF0C5FB81464046FDF7AC
:102E300072FA01464046FDF745FA4846FDF76BFA3F
:102E400001464846FDF73EFA124D134E14E028782D
:102E500028B14A46414620460DF03AF804E0307861
:102E600010B1204613F098F9D7F8E840012005F09A
:102E700097FB642014F0C2F8002CE8D1404614F00F
:102E800029F84846BDE8F04714F024B8180000209F
:102E90000D0000200E0000200F0000200EB5086C71
:102EA000074BC2680078CDE9010200910F2205A10D
:102EB0000EA0FEF731FEBDE80E4018A0FEF72CBEB6
:102EC000948101082E2E5C6D717474636C69656E5B
:102ED000745C6D717474636C69656E745C6D71742F
:102EE00074636C69656E742E6300000025733A2567
:102EF0006420257328292E2E2E0A746F7069633A78
:102F00002025732C20716F733A2025642C200A6DC4
:102F10006573736167653A25730000000A0000005D
:102F2000034900220A600A688242FCD3704700000D
:102F30006400002000280BD0426A002A0FD0137BC7
:102F4000082B0CD10968526A914208D100F072BA7C
:102F500003A340F225320AA10DA0FEF7DDBD7047A4
:102F60002E2E5C6C7769702D312E342E315C73728D
:102F7000635C636F72655C646863702E630000005D
:102F80006E6574696620213D204E554C4C00000052
:102F9000417373657274696F6E20222573222066F7
:102FA00061696C6564206174206C696E65202564BC
:102FB00020696E2025730D0A000000002DE9FC41F8
:102FC0000546002D18D06C6A002C1ED0626B4FF0A5
:102FD0003C01501C4FF480374FF001064FF6FF7351
:102FE0001CD01E32B2FBF1F0B84200D3184682B2B8
:102FF000A283002A11D011E02BA34FF4697232A1F1
:1030000038A0FEF789FDBDE8FC8127A340F2A63277
:103010003FA134A0FEF780FDF5E7A683A26B501C0C
:1030200009D01E32B2FBF1F1B94200D319468AB27F
:10303000E28302B9E683A08BE28B904202D30AB10D
:103040000020A083A07B10B1A06A01900DE094F84D
:1030500024207F2A02D8FF20019006E0C02A03D353
:103060006FF07F40019000E00193E06A009028B982
:10307000606A0199084040F08070009004F12401DA
:1030800028460BF0F1FC01A928460BF055FD6946D6
:1030900028460BF0E2FC28460BF055FD0A2120469D
:1030A00001F0EEF9AFE700002E2E5C6C7769702D11
:1030B000312E342E315C7372635C636F72655C64B5
:1030C0006863702E63000000646863705F62696EFD
:1030D000643A206E6574696620213D204E554C4C43
:1030E00000000000417373657274696F6E202225C1
:1030F0007322206661696C6564206174206C696E5E
:103100006520256420696E2025730D0A00000000EB
:10311000646863705F62696E643A206468637020FB
:10312000213D204E554C4C0070B505466C6A082177
:10313000204601F0A5F9002204F12401284604F0FC
:103140005FFB607B401C60734FF4FA7040F2E73124
:10315000B1FBF0F0608370BD10B50E48046815E057
:10316000606A90B1C18B4A1EC283012906D0616A90
:10317000888B421E8A83012804D006E0204601F095
:10318000B2FA02E0204601F0A3FA2468002CE7D14D
:1031900010BD00001C0100202DE9F04105460C4641
:1031A0001646002D2CD0002C35D0206930B158A304
:1031B00040F27E625EA168A0FEF7AEFC606930B1AD
:1031C00053A340F27F626FA163A0FEF7A5FC00222B
:1031D0004FF49A77394610460BF0AAFD206100287B
:1031E00023D04089B84206D249A340F286626FA13B
:1031F00059A0FEF791FC617B7C48002918D01AE0A9
:1032000043A340F27C627AA153A0FEF785FC6FF0E5
:103210000D00BDE8F0813EA340F27D627CA14EA08E
:10322000FEF77AFC6FF00500F3E74FF0FF30F0E7B0
:103230000168491C01600068206020694068606185
:103240000121017060694170616995F82A008870F8
:1032500060690027C770206806F0F6FE6169486063
:1032600060690781606947816069C760082E08D07E
:10327000042E06D0032E07D1207B052801D0042878
:1032800002D161696868C860606907616069476107
:1032900060698761002095F82A10814203D92918B6
:1032A00091F82B1000E00021636900F11C02995491
:1032B000401C80B21028EED30020626900F12C017E
:1032C0005754401C80B24028F7D30020626900F1B7
:1032D0006C015754401C80B28028F7D36169544870
:1032E000C1F8EC0027830020626900F1F00150541E
:1032F000401C80B24428F7D301223521204600F03B
:1033000077FA3146204600F0B9FA002081E7000044
:103310002E2E5C6C7769702D312E342E315C7372D9
:10332000635C636F72655C646863702E63000000A9
:10333000646863705F6372656174655F6D73673A3B
:1033400020646863702D3E705F6F7574203D3D2072
:103350004E554C4C00000000417373657274696FE8
:103360006E2022257322206661696C656420617479
:10337000206C696E6520256420696E2025730D0A16
:1033800000000000646863705F6372656174655F6C
:103390006D73673A20646863702D3E6D73675F6F6D
:1033A0007574203D3D204E554C4C000064686370A0
:1033B0005F6372656174655F6D73673A206368650A
:1033C000636B207468617420666972737420706224
:1033D00075662063616E20686F6C6420737472750B
:1033E000637420646863705F6D736700E800002099
:1033F000646863705F6372656174655F6D73673A7B
:10340000206E6574696620213D204E554C4C0000AD
:10341000646863705F6372656174655F6D73673A5A
:10342000206468637020213D204E554C4C00000004
:1034300063825363F8B505466C6A0C21204601F09F
:103440001FF8042221462846FFF7A6FE0646300054
:103450001ED104223221204600F0CAF9606A06F02B
:1034600049FE0146204600F061FA204600F012FBBA
:10347000208BF03081B220690CF06CF90095432369
:10348000094A2169606813F049FA204600F00EF8F5
:10349000607B401C607342F603104FF4FA71B0FB7E
:1034A000F1F060833046F8BD4481010810B5044650
:1034B000002C02D0206948B10FE0BDE810400FA3F6
:1034C00040F2C96215A11DA0FEF726BB0BA340F276
:1034D000CA6225A119A0FEF71FFB606930B907A3D6
:1034E00040F2CB622AA115A0FEF716FB206908B1B5
:1034F0000CF008F800202061606110BD2E2E5C6C7D
:103500007769702D312E342E315C7372635C636F7A
:1035100072655C646863702E6300000064686370A9
:103520005F64656C6574655F6D73673A206468639A
:103530007020213D204E554C4C00000041737365B6
:103540007274696F6E2022257322206661696C6532
:1035500064206174206C696E6520256420696E208A
:1035600025730D0A00000000646863705F64656C79
:103570006574655F6D73673A20646863702D3E7093
:103580005F6F757420213D204E554C4C00000000AB
:10359000646863705F64656C6574655F6D73673ADA
:1035A00020646863702D3E6D73675F6F75742021B2
:1035B0003D204E554C4C0000F8B505466C6A002085
:1035C00060620621204600F05BFF0122214628466A
:1035D000FFF7E2FD0646300030D1022239212046B5
:1035E00000F006F9298D204600F010FA0422372158
:1035F000204600F0FDF80121204600F03FF90321AC
:10360000204600F03BF91C21204600F037F9062146
:10361000204600F033F9204600F03CFA208BF030D1
:1036200081B220690CF096F800954323114A216974
:10363000606813F073F92046FFF738FF607B401C89
:10364000C1B26173062902D20120884000E03C200B
:1036500000EB4001C1EBC0104FF6FF7101EAC00062
:1036600000F2F3104FF4FA71B0FBF1F060833046D2
:10367000F8BD00004481010870B50B4804680025BE
:103680000EE0606A58B1418B012903D9A1F1010113
:10369000418304E003D14583204601F097F8246874
:1036A000002CEED170BD00001C010020F8B5446A6A
:1036B0000020A062E062204EA6F12805F1780029E2
:1036C00001D0E9682163317911B12969616302E0B0
:1036D000216B49086163717911B16969A16301E0E6
:1036E000216BA163A16809696162B17931B1A869EF
:1036F00006F0AAFCA0620120A07300E0A073F0799C
:1037000018B1E86906F0A0FCE06200240CE004F1C6
:10371000080055F8200006F097FC00906946204606
:1037200002F016F8641CE4B23019007A002801D0C7
:10373000022CECD3F8BD000084E7002070B50446ED
:10374000656A20460BF07CF90A4920460BF08CF99B
:10375000084920460BF081F9064920460BF0ECF9A8
:103760000C21284600F08CFE2046BDE87040FFF793
:1037700023BF00004081010870B505466C6A094806
:10378000807800280DD007482838806806F05CFC57
:103790002062A068006960622846BDE8704000F0C1
:1037A000F9BD70BD84E7002070B505466C6A002C39
:1037B0001CD0217B002604290FD004DC002915D061
:1037C000032904D109E0052907D00A2905D0667329
:1037D0002846BDE87040FFF7EFBE28460BF030F9F1
:1037E00066732846BDE8704000F04CBC70BD000018
:1037F00070B504460E461546228BA81C104444287A
:1038000006D90AA340F2F642104911A0FEF784F946
:10381000208B411C21836169F0300E54208B411CA8
:1038200021836169F0300D5470BD00002E2E5C6C58
:103830007769702D312E342E315C7372635C636F47
:1038400072655C646863702E630000005089010833
:10385000417373657274696F6E202225732220662E
:1038600061696C6564206174206C696E65202564F3
:1038700020696E2025730D0A0000000070B5044613
:103880000D46208B442806D306A340F201520DA119
:103890001BA0FEF741F9208B411C21836169F030A8
:1038A0000D5470BD2E2E5C6C7769702D312E342E28
:1038B000315C7372635C636F72655C646863702E05
:1038C00063000000646863705F6F7074696F6E5F9F
:1038D000627974653A20646863702D3E6F70746914
:1038E0006F6E735F6F75745F6C656E203C2044482B
:1038F00043505F4F5054494F4E535F4C454E00006C
:10390000417373657274696F6E202225732220667D
:1039100061696C6564206174206C696E6520256442
:1039200020696E2025730D0A0000000070B5044662
:103930000D46208B001D442806D911A34FF4A26226
:1039400017A127A0FEF7E8F8208B2A0E411C21833F
:103950006169F0300A54208B2A0C411C2183616973
:10396000F0300A54208B2A0A411C21836169F0300F
:103970000A54208B411C21836169F0300D5470BDC5
:103980002E2E5C6C7769702D312E342E315C737263
:10399000635C636F72655C646863702E6300000033
:1039A000646863705F6F7074696F6E5F6C6F6E6771
:1039B0003A20646863702D3E6F7074696F6E735F38
:1039C0006F75745F6C656E202B2034203C3D204465
:1039D0004843505F4F5054494F4E535F4C454E0043
:1039E000417373657274696F6E202225732220669D
:1039F00061696C6564206174206C696E6520256462
:103A000020696E2025730D0A0000000070B5044681
:103A10000D46208B801C442806D90AA34FF4A162CE
:103A2000104911A0FEF778F8208B2A0A411C218347
:103A30006169F0300A54208B411C21836169F030A8
:103A40000D5470BD2E2E5C6C7769702D312E342E86
:103A5000315C7372635C636F72655C646863702E63
:103A6000630000000C890108417373657274696F0B
:103A70006E2022257322206661696C656420617462
:103A8000206C696E6520256420696E2025730D0AFF
:103A90000000000010B50446002C02D0606948B157
:103AA0000FE0BDE8104017A340F2DE621DA126A082
:103AB000FEF732B813A340F2DF622EA122A0FEF778
:103AC0002BF8208B442806D30EA34FF4DC6234A1DC
:103AD0001DA0FEF721F8208BFF22411C2183616984
:103AE000F0300A54002204E0411C21836169F03067
:103AF0000A54208B442801D3810701D04428F3D3F2
:103B000010BD00002E2E5C6C7769702D312E342E86
:103B1000315C7372635C636F72655C646863702EA2
:103B200063000000646863705F6F7074696F6E5F3C
:103B3000747261696C65723A206468637020213D1B
:103B4000204E554C4C000000417373657274696FD0
:103B50006E2022257322206661696C656420617481
:103B6000206C696E6520256420696E2025730D0A1E
:103B700000000000646863705F6F7074696F6E5F4F
:103B8000747261696C65723A20646863702D3E6D71
:103B900073675F6F757420213D204E554C4C0A00B1
:103BA000646863705F6F7074696F6E5F747261696F
:103BB0006C65723A20646863702D3E6F7074696F33
:103BC0006E735F6F75745F6C656E203C2044484374
:103BD000505F4F5054494F4E535F4C454E0A0000C2
:103BE0002DE9F34F83B004464FF0000B0021029102
:103BF0000A21CB48FCF766FB049949892C2904D299
:103C00006FF0010005B0BDE8F08F04994968A1602C
:103C1000F0270498B0F80880049E06E0391A8FB2A5
:103C2000A8EB00001FFA80F8366816B17089B84218
:103C3000F4D916B1D6F804A03FE16FF00100E1E736
:103C40004FF0FF34B81C1FFA80F97289781C824249
:103C500003D90AEB0700407805E0306810B14068EE
:103C6000007800E00020054634297DD00BDC0329D4
:103C70003AD003DC29B301290DD127E0062942D02F
:103C8000332908D15EE035297DD0362968D03A291C
:103C900067D03B2974D000253844801C87B2002DA2
:103CA0000ED0002001900A2C06D39EA340F2AD5204
:103CB000A4A1A9A0FDF730FF9948005D00286ED0AF
:103CC000E2E0002005467F1EBFB2E5E7042809D0E8
:103CD00094A340F27B52ABA19FA0FDF71DFF6FF0B4
:103CE00005008FE70624D7E70425042809D28DA311
:103CF0004FF4B062A6A198A0FDF70EFF6FF005008B
:103D000080E70724C8E7810709D086A340F28552DF
:103D1000A4A191A0FDF700FF6FF0050072E708284D
:103D200001D2054600E00825A84209D27DA34FF440
:103D3000B16297A188A0FDF7EFFE6FF0050061E783
:103D40000824A9E704280DD076A340F28C528DA157
:103D500081A0FDF7E1FE6FF0050053E704E012E0FB
:103D600020E02DE0032497E701280AD06DA34FF44B
:103D7000B26290A178A0FDF7CFFE6FF0050041E799
:103D80002CE0002488E701280AD066A340F2945270
:103D900088A171A0FDF7C0FE6FF0050032E72BE0AF
:103DA000012479E7042809D05EA34FF4B36275A11A
:103DB00069A0FDF7B1FE6FF0050023E702246BE771
:103DC000042809D057A340F29C526EA162A0FDF7CF
:103DD000A3FE6FF0050015E704245DE7042809D071
:103DE00050A34FF4B46267A15BA0FDF795FE6FF09E
:103DF000050007E705244FE7042D01D22A4600E01D
:103E000004224B4601A930460BF0F0FA042D1DD9CF
:103E1000A80709D043A340F2B35269A14EA0FDF711
:103E20007BFE6FF00500EDE63D4901200855019845
:103E300006F00AF93A49283941F824002D1FEDB25D
:103E400009F104091FFA89F9641C2CE7042D0BD031
:103E5000012D0ED033A340F2BD525EA13EA0FDF76E
:103E60005BFE6FF00500CDE6019806F043F9019086
:103E700002E09DF8040001902949012008552848D6
:103E80000199283840F824107089B84215D8391A99
:103E90008FB2A8EB00001FFA80F8474515D2B8F1A1
:103EA000000F12D0366836B91EA340F2C9524EA197
:103EB00029A0FDF731FED6F804A036B11AF8071094
:103EC000FF2902D04745FFF4BBAE154A1078A0B1D8
:103ED000A2F12800006800211170012804D00228F6
:103EE00005D0032806D008E04FF0010B05E00120C3
:103EF000029002E0012002908346BBF1000F05D042
:103F00004FF0000B6C274FF0EC0885E6029828B1C3
:103F1000002002902C274FF06C087DE6002071E60F
:103F200084E700202E2E5C6C7769702D312E342EA4
:103F3000315C7372635C636F72655C646863702E7E
:103F400063000000636865636B206465636F64658C
:103F50005F69647800000000417373657274696F73
:103F60006E2022257322206661696C65642061746D
:103F7000206C696E6520256420696E2025730D0A0A
:103F8000000000006C656E203D3D20340000000004
:103F90006C656E203E3D206465636F64655F6C6593
:103FA0006E0000006C656E20252034203D3D2030E1
:103FB000000000006C656E203D3D203100000000D7
:103FC0006465636F64655F6C656E20252034203DF9
:103FD0003D203000696E76616C6964206465636FB2
:103FE00064655F6C656E00006E6578742070627544
:103FF0006620776173206E756C6C0000F8B505461D
:104000006C6A0421204600F03BFA03222146284630
:10401000FFF7C2F8064630001BD1022239212046A4
:10402000FFF7E6FB298D2046FFF7F0FC2046FFF75F
:1040300031FD208BF03081B220690BF08BFB0095B5
:1040400043230F4A2169606812F068FC2046FFF79D
:104050002DFA607B401CC0B260730A2803D24FF473
:104060007A71484301E042F2107080B200F2F3101E
:104070004FF4FA71B0FBF1F060833046F8BD0000F8
:1040800044810108F8B50646746A0321204600F011
:10409000F7F9032221463046FFF77EF8054628004F
:1040A00028D1022239212046FFF7A2FB4FF41071DC
:1040B0002046FFF7ABFC042232212046FFF798FB95
:1040C000606A06F017F801462046FFF72FFC2046ED
:1040D000FFF7E0FC208BF03081B220690BF03AFB57
:1040E000009643230E4A2169606812F017FC2046AF
:1040F000FFF7DCF9607B401CC0B260730A2803D272
:104100004FF47A71484301E042F2107080B200F23D
:10411000F3104FF4FA71B0FBF1F060832846F8BD5C
:10412000448101082DE9F041054617466C6A7E6816
:10413000A068002806D034A340F211623AA13FA043
:10414000FDF7EAFC78894FF000082C2854D330782A
:10415000022851D1002095F82A1008E02A183318B7
:1041600092F82B201B7F9A4246D1401CC0B281425C
:10417000F4D8706805F0BEFF216888423CD139460A
:104180002046FFF72DFD50BB3748407838B33648FE
:1041900028380079052802D0062815D01DE0207B9C
:1041A000012806D003280BD0042809D0052807D001
:1041B00022E02846FFF77AFA2846FEF7B5FF1BE013
:1041C0002846FEF7FBFE17E0237B032B08D0012BCC
:1041D00006D0042B04D0052B02D0022804D00BE01B
:1041E0002846FFF7ABFA07E0207B062804D1A4F8A5
:1041F0001A802846FFF7C0FAC4F808803846BDE8A0
:10420000F0410BF07FB900002E2E5C6C7769702DA9
:10421000312E342E315C7372635C636F72655C6443
:104220006863702E630000007265706C792077619E
:10423000736E277420667265656400004173736550
:104240007274696F6E2022257322206661696C6525
:1042500064206174206C696E6520256420696E207D
:1042600025730D0A0000000084E70020F8B505461C
:104270006C6A0021204600F003F900202062606291
:10428000A062E062A06360632063072221462846A3
:10429000FEF782FF0646300013D12046FFF7FAFBF7
:1042A000208BF03081B220690BF054FA0095432343
:1042B00004F120022169606812F030FB2046FFF70C
:1042C000F5F8607B401CC0B260730A2803D24FF43B
:1042D0007A71484301E042F2107080B200F2F310AC
:1042E0004FF4FA71B0FBF1F0608328460AF0A8FBA6
:1042F000064928460AF0B8FB044928460AF0ADFBF7
:10430000024928460AF018FC3046F8BD40810108F1
:10431000F8B505466C6A0521204600F0B1F8032285
:1043200021462846FEF738FF064630001CD10222FF
:1043300039212046FFF75CFA298D2046FFF766FBFE
:104340002046FFF7A7FB208BF03081B220690BF0ED
:1043500001FA0095432304F120022169606812F0FC
:10436000DDFA2046FFF7A2F8607B401CC0B2607304
:104370000A2803D24FF4FA61484301E044F6206072
:1043800080B200F2F3104FF4FA71B0FBF1F06083E9
:104390003046F8BDF8B505466C6A0121204600F0AC
:1043A0006FF8032221462846FEF7F6FE0646300047
:1043B00048D1022239212046FFF71AFA298D2046DA
:1043C000FFF724FB042232212046FFF711FA606A2E
:1043D00005F090FE01462046FFF7A8FA0422362198
:1043E0002046FFF705FA206A05F084FE01462046C4
:1043F000FFF79CFA042237212046FFF7F9F9012143
:104400002046FFF73BFA03212046FFF737FA1C212D
:104410002046FFF733FA06212046FFF72FFA204601
:10442000FFF738FB208BF03081B220690BF092F956
:1044300000954323114A2169606812F06FFA204603
:10444000FFF734F8607B401CC1B26173062902D2C9
:104450000120884000E03C2000EB4001C1EBC0108F
:104460004FF6FF7101EAC00000F2F3104FF4FA7149
:10447000B0FBF1F060833046F8BD000044810108D4
:10448000027B8A4203D0017300214173418370474C
:1044900070B505466FF00D06002D0AD06C6A95F8D0
:1044A000310020F0080085F8310080060AD430463B
:1044B00070BD2FA340F27A2235A139A0FDF72CFB65
:1044C000304670BD288D4FF0FF36B0F5107F01D219
:1044D000304670BD002C39D0606808B112F0D6F9B2
:1044E000206930B122A340F29E2238A12CA0FDF712
:1044F00013FBA06830B11EA340F29F2239A128A06F
:10450000FDF70AFB3C212046FBF7DCFE12F088F9A0
:10451000606028B3017A41F02001017244223649DB
:10452000606811F061FF43223349606811F0D2FFE7
:104530002A463249606812F0A5F92846FFF73CF890
:1045400080B1284600F05CF8304670BD3C2006F093
:10455000AFFB0446200001D06C62D3E7304670BD4B
:10456000304670BD15F8311F41F00801297070BD4B
:104570002E2E5C6C7769702D312E342E315C737267
:10458000635C636F72655C646863702E6300000037
:104590006E6574696620213D204E554C4C0000002C
:1045A000417373657274696F6E20222573222066D1
:1045B00061696C6564206174206C696E6520256496
:1045C00020696E2025730D0A000000007062756678
:1045D00020705F6F7574207761736E277420667228
:1045E000656564007265706C79207761736E2774FD
:1045F000206672656564000040810108254100085D
:1046000010B500281CD050F8244F417B21F0080140
:104610004173002C1DD0606818B112F037F90020EA
:104620006060A06830B10BA340F2DA4211A116A07D
:10463000FDF772FA2046BDE810400021FFF720BFC9
:10464000BDE8104003A340F2C7421AA10EA0FDF737
:1046500063BA10BD2E2E5C6C7769702D312E342E0E
:10466000315C7372635C636F72655C646863702E47
:10467000630000007265706C79207761736E277437
:104680002066726565640000417373657274696FBA
:104690006E2022257322206661696C656420617436
:1046A000206C696E6520256420696E2025730D0AD3
:1046B00000000000646863705F73746F703A206E6E
:1046C0006574696620213D204E554C4C0000000069
:1046D000416A097B012903D00A2901D0052901D1AA
:1046E000FFF716BE7047416A097B012903D00A29EA
:1046F00001D0052901D1FFF781BC7047A0B000208F
:104700001C90224D224C01264FF47A77217811B16A
:10471000012936D106E01D48FFF7BAFE00201C90A3
:1047200026702EE068681C901C98A0B1666002207C
:1047300020701648FFF764FF9DF873009DF8721013
:10474000CDE900109DF871309DF8702011A103A8EB
:10475000FDF7F2F915E0686A407B042811D90320BF
:1047600020700A48FFF74CFF16481F906FF07F40FB
:104770001E9015481D901DAB1EAA1FA903480AF0E4
:1047800048F9384612F03AFCC0E700007C090020E6
:104790005C0000200D0A44484350202D2D206576F2
:1047A000616C20626F617264206970206164647260
:1047B0006573733A2025642E25642E25642E2564A6
:1047C000200D0A00C0A80064C0A8000110B504466E
:1047D000626A117B0C2913D0062911D0012914D04B
:1047E000082922D005292DD0042930D0032943D10E
:1047F000507B02283BD22046BDE81040FFF742BC68
:104800002046BDE81040FEF7D7BE507B052804D8EF
:104810002046BDE81040FFF7BDBD2046FFF726FD4E
:104820002046BDE81040FEF7C7BE507B012804D8E3
:104830002046BDE81040FEF777BC2046BDE810409A
:10484000FEF7BCBB2046BDE81040FFF761BD507BC2
:10485000082804D82046BDE81040FFF7CFBB20460B
:10486000FFF704FD2046BDE81040FEF7A5BE204638
:10487000BDE81040FEF7A0BE10BD000010B5FEF769
:104880006BFCBDE81040002202494EF660200DF09E
:104890004DB900007D48000810B5FEF7EDFEBDE8FB
:1048A0001040002202494FF4FA700DF03FB90000A9
:1048B0009948000870B50D46164604464BF2306123
:1048C000401A8C4231D014DC4BF22161A4EB010080
:1048D0008C4224D008DCA4F53644113C19D0012CBC
:1048E00017D0022C13D114E0012818D002280ED1C1
:1048F00015E061280DD006DC012816D0022814D05E
:10490000032804D111E0622803D0632801D00020DD
:104910001DE011A20221284600F0AAFA19E00FA218
:104920000221284600F0A4FA13E00EA20321284633
:1049300000F09EFA0DE02C5C333C04F00F012411D2
:1049400004EB840201EB42011954401C80B2B042D6
:10495000F1D3304670BD00005858580058582E58B2
:104960005800000058582E58585858002DE9F0416A
:1049700096B004460D4616463C2103A8FBF7A2FC60
:10498000002012901390149015902168CDF84910D2
:10499000A188ADF84D1001218DF8501002278DF837
:1049A0005170029005F133008DF80800280A333069
:1049B0008DF80900BDF80800ADF852000E2212A9CA
:1049C000204600F028FB4FF0FF38002803DA40466D
:1049D00016B0BDE8F0812B463C2203A92046009783
:1049E00000F0F8FA002801DA4046F1E79DF81500DA
:1049F0003346801E82B206A92846FFF75BFFE7E731
:104A00001FB50446204600F0FCF901004FF0FF30CE
:104A100010D4217A84290FD003AA0021535C3333A8
:104A20005354491CC9B20229F8D36189039A9142AF
:104A300000D1002004B010BD0020FBE72DE9F05F9D
:104A40000D4617461E469C494FF400784A14441AF6
:104A500013024FF47D4C4FF47E4A4FF400398842E4
:104A600064D064DC954CA0EB0401A04210D030DC93
:104A7000934CA0EB0401A0420AD013DCB0F5407FB8
:104A800006D006DC002803D0904201D0404578D102
:104A9000ABE0B0F5806F04D0984202D0B0F1011FB6
:104AA0006FD1A2E040F2FE32A1F2FE30914209D075
:104AB00009DCFE2906D0B1F5FF7F03D0A1F5007116
:104AC000FE395ED191E0B0F57C4F01D0604558D100
:104AD0008BE07C4C081BA1420AD012DCB1F5FF3FF1
:104AE00006D006DC914203D041457ED051457AD1B3
:104AF0007BE07548081878D0984276D0484572D146
:104B000073E0B0F57A0F77D009DC98426DD0B0F53C
:104B1000790F71D06FF47901C84264D16CE06FF401
:104B20007A01401868D0B0F1FF1F5CD174E067498A
:104B3000DFF89CB1601A4FF47F4E8C427AD027DCAC
:104B40004C4577D011DC9C426DD006DC944263D09A
:104B5000644561D0744546D165E014EB0B0062D02A
:104B6000604567D050453ED164E0B4F5403F61D028
:104B700008DC584820185DD060455BD0504532D1E4
:104B800058E030E05448201854D060452BD151E013
:104B9000524C011BA0423FD012DC984251D006DC9F
:104BA000904247D0404545D070451CD149E010EBBC
:104BB0000B0046D0904244D04949C84213D12BE063
:104BC00048480B1A81424AD008DC914224D046481A
:104BD00008183DD04549C84205D151E0444818184D
:104BE0004ED001284CD0002060E0334641A2042181
:104BF000284600F03DF95BE0334641A203212846F8
:104C000000F036F900202918C978333932181171AB
:104C1000401C0528F7DB4BE033463BA20221284627
:104C200000F026F944E0334639A20321284600F07B
:104C30001FF93DE0334632A20321284600F018F95F
:104C400036E0334634A20221284600F011F92FE065
:104C5000334629A20221284600F00AF928E0002064
:104C60000BE0295C333901F00F02091101EB8101DE
:104C700002EB41013154401C80B2B842F1D317E03D
:104C8000002004E0295C33393154401C80B2B84222
:104C9000F8D30DE0295C333901F00F02091101EB63
:104CA000810102EB41013154401C80B2B842F1D382
:104CB0003846BDE8F09F0000000201020002020039
:104CC0000200010000FE05000002FDFF00FF0300DE
:104CD00000FFFEFF00FFFDFF00FFFCFF00010700DB
:104CE0000001FAFF01FFF902FE018CFFFFFB7FFECE
:104CF000000106FE5858585858582E5858000000C1
:104D000058582E58585858005858582E58000000D7
:104D10005858582E58585800582E585858000000C7
:104D2000F0B595B005460C4616463C2102A8FBF7A7
:104D3000C9FA002211921292139214922868CDF8A7
:104D40004500A888ADF8490011208DF84C000420DA
:104D50008DF84D00019204F133008DF80400200A13
:104D600033308DF80500200C33308DF806003320E9
:104D700000EB14608DF807000198CDF84E0010226A
:104D800011A9284600F047F94FF0FF37002802DA52
:104D9000384615B0F0BD0120009023463C2202A900
:104DA000284600F017F9002801DA3846F1E79DF8A7
:104DB00011003346001F82B20DF116012046FFF7A5
:104DC0003DFEE6E71FB50446204600F01AF8010054
:104DD0004FF0FF3011D4217A942910D003AA00217A
:104DE000535C33335354491CC9B20429F8D3D4F863
:104DF0000A10039A914200D1002004B010BD002097
:104E0000FBE72DE9F041044617464FF0FF3607292E
:104E100002DA3046BDE8F0812078682807D1E079D1
:104E2000682804D1651815F8010C162801D0304601
:104E3000F0E7891E2046FCF7C0FEC0B215F8021C40
:104E4000814201D03046E5E7207A010601D43046A0
:104E5000E0E7400602D515F8030CDBE706223946E9
:104E6000601CFBF76DFA08B13046D3E70020D1E7AC
:104E70002DE9F843154698460026FDF769FF0746D9
:104E8000002403E0285D2E2817D0641C2846FBF779
:104E900042FAA042F6D831460A2008F05DFCB7FB82
:104EA000F0F000EE100AB8EE400A8DED000A00980E
:104EB000C8F800000020BDE8F8832846FBF72BFA6D
:104EC000061B761E002EE6DA4FF0FF30F3E70000F7
:104ED0002DE9F0410F46164612F050FE05460E4CE5
:104EE00012F04CFE431B606800EB4001C1EBC010A8
:104EF000B3EBC00F02D90020BDE8F08194F8D000D8
:104F00000128EDD10449321F0C313846FBF7C1F9B5
:104F100094F8D100001FEFE7D83F01202DE9F047BA
:104F20000E461546C8211648FBF7CCF90A20FDF7B6
:104F3000F7FFDFF850904FF4807801224146484651
:104F400003F00EFC0024104F0BE0315D384611F0E9
:104F500081FE0721384611F08FFE0028F9D0641C2D
:104F6000A4B2AC42F1D900224146484603F0F8FB16
:104F700003490020C831487008702846BDE8F08712
:104F8000E03F0120000801400038014010B5044610
:104F900001221102044803F0E3FB04494C600020A5
:104FA000087081F8D10010BD00080140D83F0120F1
:104FB00030B404464FF0FF30012B05D0022B07D14F
:104FC000204630BCFFF7D2BC204630BCFFF7A8BE5D
:104FD00030BC70472DE9F0410646069C0F469846C6
:104FE000F56839463046A8470146022C05D0012C09
:104FF0000AD04FF0FF30BDE8F081434632463846D4
:10500000BDE8F041FFF7FCBC434632463846BDE8F8
:10501000F041FFF7D7BE2DE9F04107460C46154693
:1050200068202070E07116206619B61E7070A91EE7
:105030002046FCF7C2FD3070AAB221463846BB6854
:10504000BDE8F04118473CB50022009201926B4642
:10505000C2F105058C5C5C55521C062AF8DB0099F0
:105060000160BDF8041081803CBD000070B5174D93
:105070000521284611F000FE154C98B194F8D10096
:10508000C7280CD2284611F0E1FD114914F8D12FA0
:10509000083150542078401C04F8D10902E0284619
:1050A00011F0D4FD94F8D10000280DD00421284639
:1050B00011F0E2FD002807D04FF44171284611F0AD
:1050C000FCFD012084F8D00070BD000000380140D4
:1050D000D83F012010B50024204600F005F8641CDC
:1050E000E4B2042CF8D310BD70B50546C5EBC5007D
:1050F000364900EB800001EBC004042D06D334A335
:1051000040F281223AA141A0FCF706FD2078002858
:1051100046D0C5EBC5012D4B01EB810103EBC1036B
:10512000002601220C3301280CD0022816D00328B7
:1051300043D0BDE8704026A340F2C5223EA133A073
:10514000FCF7EABC0220207030466670A270E07066
:105150002A46BDE87040194600F02CBAA078401EDF
:1051600010F0FF00A0701BD1E078401CC0B2E070CE
:10517000042807D0A07060782A46BDE87040194620
:1051800000F018BA6078401C02280AD2324911EBAC
:10519000800506D051F8201019B16070A270E67039
:1051A00070BDD4F8105125B100211846D4F814214F
:1051B000A8472670C4F8106170BDA068401EA060AA
:1051C000FAD12670C4F8106170BD000090E700208D
:1051D0002E2E5C6C7769702D312E342E315C7372FB
:1051E000635C636F72655C646E732E630000000025
:1051F000617272617920696E646578206F757420C0
:105200006F6620626F756E64730000004173736592
:105210007274696F6E2022257322206661696C6545
:1052200064206174206C696E6520256420696E209D
:1052300025730D0A00000000756E6B6E6F776E208F
:10524000646E735F7461626C6520656E7472792040
:1052500073746174653A0000F800002030B50323D0
:1052600011F8012BB3EB921F10D009E004780D78F0
:10527000AC4201D0012030BD491C401C521ED2B2AC
:10528000002AF3D1401C0A78002AE9D1002030BD61
:105290002DE9F04706468946002007460024DFF83E
:1052A000A080DFF8A0C098F80010C4EBC40303EBA3
:1052B00083030CEBC3052B785BB1032B05D12B7952
:1052C000CB1ABB4201DDDFB22046641CE4B2042CE1
:1052D000EBD3042C10D1042807D2C0EBC00303EB9E
:1052E00083031CF83340032C03D04FF0FF30BDE89C
:1052F000F08704460CEBC305012028702971491C76
:1053000088F80010C5F81091C5F814213046FBF755
:1053100002F8FF2803D23046FAF7FDFF00E0FF2035
:1053200007463A46314605F10C00FAF7B2FF002075
:10533000E91908732046FFF7D7FE6FF00400D6E79F
:10534000EC00002090E700202DE9F04104460D46D6
:1053500016461F4612484068002808D03DB134B1B7
:10536000207820B12046FAF7D6FFFF2803D96FF046
:105370000D00BDE8F081204604F022F9411C02D165
:10538000204600F03FF8411C02D028600020F0E7E2
:105390003A4631462046BDE8F041FFF779BF0000AC
:1053A000EC00002038B50F480F4C20F00300A0603F
:1053B0000EA004F005F900906068002811D111F0EA
:1053C0002FFA606000280CD000220C4911F00CF874
:1053D00000220B49606811F055FA6946002000F080
:1053E000B7F938BDF3EB0020EC0000203230382E46
:1053F00036372E3232322E323232000040810108EE
:105400007554000870B506460024104DC4EBC40165
:1054100001EB810115F83100032806D105EBC1012C
:105420000C313046FAF77EFF30B1641CE4B2042C34
:10543000ECD34FF0FF3070BDC4EBC40000EB800034
:1054400005EBC000D0F80C0170BD000090E7002013
:10545000032210F8011BB2EB911F08D002E0401CA0
:10546000491EC9B20029FAD101780029F1D1401CA6
:10547000704700002DE9FE4F17463A89B2F5007FCC
:105480006ED81A2A6CD3DFF8208100233846D8F86A
:10549000081009F0ABFF3989884261D1D8F808605B
:1054A000308804F0DDFD042879D2C0EBC0003F490C
:1054B00000EB800001EBC004207802286FD10320AC
:1054C0002070F07800F00F006071B08804F0C8FD23
:1054D0008146F08804F0C4FD0546B078000651D539
:1054E0006079E0BBB9F1010F4CD1D8F8081004F194
:1054F0000C000C318246FFF7B1FE80BBD8F80800E3
:105500000C30FFF7A5FF001D4FF480784FF4806941
:1055100036E0FFF79DFF0646316800917168019102
:105520003089ADF80800BDF80000404520D1BDF835
:10553000020040451CD1BDF80800484518D101982B
:1055400004F0D8FDA0601A49884200D9A160D6F8BD
:105550000A00C4F80C01D4F810310BB101E011E0DD
:105560001DE004F586715046D4F81421984716E0E2
:10557000BDF8080004F074FD30440A306D1EADB271
:10558000002DC6D1D4F810312BB1002104F10C004C
:10559000D4F81421984700202070C4F81001384630
:1055A000BDE8FE4F09F0AEBFEC00002090E7002000
:1055B000803A09002DE9F84304460D469146022C35
:1055C00006D339A34FF40F723FA145A0FCF7A4FA0C
:1055D0004E4810EB840702D050F8240030B932A3B3
:1055E00040F23D224AA13EA0FCF796FA00224FF479
:1055F0008871104609F09CFB064630004FD0306899
:1056000030B129A340F243224AA135A0FCF784FA25
:1056100074684FF00008C4F80080C4F80480C4F82F
:105620000880484604F01CFD20800120A070020282
:10563000A2800C346D1E6D1C2346641C002004E007
:1056400004F8011B401CC0B26D1C29782E2901D022
:105650000029F5D1187028780028ECD104F8018BC6
:10566000ADF80020ADF8022000982060B088201A24
:10567000001D81B230460AF06DF8244C39460C3CCE
:105680003522606810F026FF3A46352331466068BF
:1056900011F030F90446304609F034FF01E04FF0D4
:1056A000FF342046BDE8F8832E2E5C6C7769702DA0
:1056B000312E342E315C7372635C636F72655C648F
:1056C0006E732E6300000000646E73207365727643
:1056D0006572206F7574206F662061727261790047
:1056E000417373657274696F6E2022257322206680
:1056F00061696C6564206174206C696E6520256445
:1057000020696E2025730D0A00000000F8000020BB
:10571000646E732073657276657220686173206EA3
:105720006F204950206164647265737320736574DF
:105730000000000070627566206D757374206265EC
:1057400020696E206F6E65207069656365000000DA
:1057500002280CD2064A5268002A08D0002906D036
:105760000968002903D0024A0C3242F82010704721
:10577000EC00002010B500F00BF8BDE8104000224E
:1057800002494FF47A700CF0D1B900007557000847
:1057900003484068002801D0FFF79CBC7047000018
:1057A000EC00002010B50446216891F9080010F1C2
:1057B000090F01DA20711CE0FA2020714868C0B19D
:1057C000097801F0F00110290ED0202906D04029D7
:1057D0000FD1A1680AF056FF20710AE0A289A168E2
:1057E00010F002FE207104E0A289A1680CF0F8FB21
:1057F00020712068BDE810400C300CF067B9000043
:105800002DE9F0410446002C06D153A34FF43C721D
:1058100059A15DA0FCF780F92078102806D04EA38E
:1058200040F2F12263A158A0FCF776F960780428D1
:1058300006D049A340F2F22266A153A0FCF76CF90E
:10584000606830B944A340F2F3226BA14EA0FCF78C
:1058500063F9A06A30B940A34FF43D726BA14AA02E
:10586000FCF75AF9A06A007A00F0010600F002077E
:10587000032825D000251DB1002160680CF0AEFB87
:105880006068017E01291DD036B100210EF0D8FDDF
:10589000002160680CF04BFB1FB1002160680FF025
:1058A00001F845B10422002160680DF051FF00218C
:1058B00060680CF05FFF4DB160680CF019FC0AE005
:1058C0000125D8E700210CF032FBF4E73A463146D7
:1058D00060680FF01DFA20B16068007E012821D0B9
:1058E00027E0A16A00200871A062607035B1606095
:1058F000E36A1BB100220421204698472EB1E36AD7
:105900001BB100221146204698472FB1E36A1BB114
:10591000002202212046984704F10C00BDE8F04126
:105920000CF0D4B80CA340F22D323FA116A0FCF726
:10593000F3F8464960680EF0B5FF042244496068F8
:105940000DF006FF434960680CF014FF21466068C3
:10595000BDE8F0410CF042BB2E2E5C6C7769702DD7
:10596000312E342E315C7372635C6170695C6170DE
:10597000695F6D73672E6300696E76616C69642080
:10598000636F6E6E00000000417373657274696F1F
:105990006E2022257322206661696C656420617423
:1059A000206C696E6520256420696E2025730D0AC0
:1059B000000000007468697320697320666F7220AC
:1059C000746370206E6574636F6E6E73206F6E6C9F
:1059D00079000000636F6E6E206D757374206265D0
:1059E00020696E207374617465204E4554434F4E98
:1059F0004E5F434C4F53450070636220616C72658B
:105A000061647920636C6F7365640000636F6E6E10
:105A10002D3E63757272656E745F6D736720213DF4
:105A2000204E554C4C000000436C6F73696E67202C
:105A300061206C697374656E20706362206D61799A
:105A4000206E6F74206661696C2100007116010878
:105A50000DFE0008C16F000810B5044620684368B9
:105A6000002B17D0017801F0F001102922D0202955
:105A700019D0402911D027A340F203422DA133A011
:105A8000FCF74AF8FA2020712068BDE810400C307D
:105A90000CF01CB8F4202071F6E71846A1680AF053
:105AA000F9FD2071F0E7A2891846A16810F012FDF7
:105AB0002071E9E7417811B1F7202071E4E70BF09C
:105AC00017FF2068A289A16840682B4B0CF008FCE6
:105AD00020710028D8D1206890F82010C1F340012F
:105AE00003224270002906D0206810F8201F41F0E0
:105AF0000401017005E0206810F8201F21F0040166
:105B0000017003D04FF0FB002071BDE72068846274
:105B100010BD00002E2E5C6C7769702D312E342E56
:105B2000315C7372635C6170695C6170695F6D7335
:105B3000672E6300496E76616C6964206E657463DC
:105B40006F6E6E207479706500000000417373659C
:105B50007274696F6E2022257322206661696C65FC
:105B600064206174206C696E6520256420696E2054
:105B700025730D0A000000007D5B000870B5044627
:105B80001546002C0CD06078032806D022A340F2E2
:105B9000B63229A130A0FBF7BFFFA06A18B10DE013
:105BA0006FF0050070BD94F82000400706D41AA3DA
:105BB00040F2B73233A128A0FBF7AEFFA06A00B1D4
:105BC00005712078102803D115B920460BF090FEFE
:105BD00094F8200040F380056D1C20F0040084F848
:105BE00020000026A66266704DB90BF0DDFE94F928
:105BF000081011F1090F00DB26720BF0FFFEE36ABB
:105C00001BB100220221204698471DB104F10C006F
:105C10000BF05CFF002070BD2E2E5C6C7769702D40
:105C2000312E342E315C7372635C6170695C61701B
:105C3000695F6D73672E6300636F6E6E2D3E7374C4
:105C4000617465203D3D204E4554434F4E4E5F43A9
:105C50004F4E4E4543540000417373657274696F33
:105C60006E2022257322206661696C656420617450
:105C7000206C696E6520256420696E2025730D0AED
:105C80000000000028636F6E6E2D3E6375727265B2
:105C90006E745F6D736720213D204E554C4C29205A
:105CA0007C7C20636F6E6E2D3E696E5F6E6F6E5FE3
:105CB000626C6F636B696E675F636F6E6E65637452
:105CC0000000000070B5044621684878002810D014
:105CD00002280ED003280CD00878102806D031A353
:105CE00040F2473237A13FA0FBF716FFFB2020719F
:105CF00033E003280AD191F82000400706D429A3F5
:105D000040F24A3242A137A0FBF706FF206807F0B5
:105D1000A1FF20684268A2B1017801F0F0011029CA
:105D200027D00025202905D0402908D110460AF0A7
:105D30000DFD04E0D5612068406810F0A7FD2068E3
:105D400045602068C36A13B1002211469847206855
:105D5000C36A13B100220221984720680C300BF06F
:105D6000BBFE00281CD02068BDE870400C300BF052
:105D7000ADBE816A09B9406A30B10AA340F25F3210
:105D80002BA118A0FBF7C8FE21680420487003204F
:105D90002072206884622068BDE87040FFF730BD43
:105DA00070BD00002E2E5C6C7769702D312E342E64
:105DB000315C7372635C6170695C6170695F6D73A3
:105DC000672E63006D73672D3E636F6E6E2D3E749C
:105DD000797065203D3D204E4554434F4E4E5F54F3
:105DE00043500000417373657274696F6E20222501
:105DF0007322206661696C6564206174206C696E31
:105E00006520256420696E2025730D0A00000000BE
:105E1000626C6F636B696E6720636F6E6E6563742F
:105E200020696E2070726F677265737300000000E6
:105E3000616C72656164792077726974696E67203C
:105E40006F7220636C6F73696E67000070B50346F4
:105E50000D46144619462068FAF764FA30B10BA3D0
:105E600040F2FA5211A11AA0FBF756FE55B1E168B3
:105E700000200870606829680160A068BDE8704073
:105E80000BF024BEE168FA200870F6E72E2E5C6C59
:105E90007769702D312E342E315C7372635C6170C2
:105EA000695C6170695F6D73672E6300444E5320B7
:105EB000726573706F6E736520666F722077726F94
:105EC0006E6720686F7374206E616D65000000005E
:105ED000417373657274696F6E2022257322206688
:105EE00061696C6564206174206C696E652025644D
:105EF00020696E2025730D0A0000000010B50446CD
:105F00006FF00C0220684068002840D0217C19B155
:105F1000A1680068086002E0A1684068086000208D
:105F200020712068017801F0F001102925D0202986
:105F300012D0402907D019A340F29B521FA125A0DF
:105F4000FBF7EAFD24E0217C21B14068E168007C98
:105F500008801DE022711BE0217C21B14068E168CE
:105F6000408A088014E04068017C490701D422710E
:105F70000EE0E168808A08800AE0217C11B1406867
:105F8000408B01E04068808BE168088000E022716E
:105F90002068BDE810400C300BF098BD2E2E5C6CD4
:105FA0007769702D312E342E315C7372635C6170B1
:105FB000695C6170695F6D73672E6300696E7661FD
:105FC0006C6964206E6574636F6E6E5F7479706562
:105FD00000000000417373657274696F6E202225A2
:105FE0007322206661696C6564206174206C696E3F
:105FF0006520256420696E2025730D0A00000000CD
:1060000010B504462346D4E90001064AFFF79CF97F
:10601000E1680870401D04D0A068BDE810400BF096
:1060200055BD10BD4D5E000870B50446206890F95E
:10603000081011F1090F01DA217108E0F321217133
:10604000426822B10178102907D0F220207120681F
:10605000BDE870400C300BF039BD40780028F6D117
:10606000FF2110460CF06AFF0546A5B120681030EC
:106070000BF002FD38B1206810300BF0C7FC20682F
:1060800010300BF0E8FC00262671206814300BF06D
:10609000F3FC18B108E0FF202071D8E72068002148
:1060A00014300BF0BDFC2071207928B128460CF08B
:1060B0001FF820684660CAE72168022048702068FF
:1060C0004560284621680BF089FF20680249406836
:1060D0000BF02DFFBBE700009324000810B5044629
:1060E0000020207120684068002802D1204609F075
:1060F00001FC2068BDE810400C300BF0E7BC2DE936
:10610000F04105460020287128684168002914D014
:106110000078102811D1AC684FF480384FF6FF7723
:10612000444501D33E4600E0A6B2286831464068A7
:106130000EF0E4F9A41B002CF2D12868BDE8F04170
:106140000C300BF0C3BC70B50446206890F9081001
:1061500011F1090F01DA21712CE0F3212171456859
:1061600045B3007800F0F000202815D0402821D158
:10617000A06810F1080F09D0816839B100F1080258
:10618000016828460AF0FCFA207113E001682846ED
:106190000AF0F2FA20710DE0A06810F1080F0FD09C
:1061A000816869B1838900F108020168284610F00E
:1061B000A1FB20712068BDE870400C300BF086BC5C
:1061C0000168284610F078FB2071F3E710B504460B
:1061D000206890F9081011F1090F01DA217104E02B
:1061E0000178102906D0FA212171BDE810400C3049
:1061F0000BF06CBC417811B1FB212171F5E74168CE
:10620000002920D0012141702068816A09B9406AC3
:1062100030B10EA340F24C5214A11BA0FBF77CFC42
:10622000E06830B909A340F24E5222A116A0FBF754
:1062300073FC206884622168002048622068BDE801
:10624000104000F041B8F3212171CEE72E2E5C6C96
:106250007769702D312E342E315C7372635C6170FE
:10626000695C6170695F6D73672E6300616C726554
:106270006164792077726974696E67206F72206338
:106280006C6F73696E670000417373657274696F38
:106290006E2022257322206661696C65642061741A
:1062A000206C696E6520256420696E2025730D0AB7
:1062B000000000006D73672D3E6D73672E772E6CA6
:1062C000656E20213D2030002DE9F04704464FF057
:1062D0000008A16A94F820000E7C800701D47007A2
:1062E00001D5012700E0002734B95AA340F2C34288
:1062F00060A164A0FBF710FC6078012806D055A3CC
:1063000040F2C4426AA15FA0FBF706FCA06A30B964
:1063100050A340F2C5426EA15AA0FBF7FDFB606896
:1063200030B94CA340F2C64270A156A0FBF7F4FB73
:10633000D4E90901C968884206D346A340F2C7429E
:1063400070A150A0FBF7E8FBA16A606A8A6802EBC3
:106350000009CB68191AB1F5803F04D34FF6FF75D9
:1063600046F0020600E08DB26168B1F86620AA42EC
:1063700007D215461FB125B96FF0060616E046F0A4
:1063800002062844984206D932A340F2F5426AA197
:106390003CA0FBF7C1FB33462A46494660680FF034
:1063A00005F80646300001D0701C22D187B1A06AE2
:1063B000C068A8420CD9E36A1BB12A4603212046D3
:1063C000984794F8200040F0100084F8200010E076
:1063D000606840F66732B0F86610914203D9B0F8B1
:1063E0006800052805D3E36A1BB12A46032120462D
:1063F00098474FF0000916B1701C11D011E0606A87
:1064000028446062A16ACA68904200D027B1C8607F
:106410004FF00108C4F8249060680CF053FE05E0CA
:10642000A7B14FF00108A06AC0F80C90B8F1000FB6
:1064300009D0A06A0671C4F8289084F8019004F18C
:106440000C000BF043FB0020BDE8F08760680CF007
:1064500039FEEBE72E2E5C6C7769702D312E342ED1
:10646000315C7372635C6170695C6170695F6D73EC
:10647000672E6300636F6E6E20213D204E554C4C9D
:1064800000000000417373657274696F6E202225ED
:106490007322206661696C6564206174206C696E8A
:1064A0006520256420696E2025730D0A0000000018
:1064B000636F6E6E2D3E7374617465203D3D204E9A
:1064C0004554434F4E4E5F5752495445000000001B
:1064D000636F6E6E2D3E63757272656E745F6D7361
:1064E0006720213D204E554C4C000000636F6E6EBE
:1064F0002D3E7063622E74637020213D204E554CFA
:106500004C000000636F6E6E2D3E77726974655F9C
:106510006F6666736574203C20636F6E6E2D3E63FC
:10652000757272656E745F6D73672D3E6D73672E45
:10653000772E6C656E000000646F5F77726974651A
:106540006D6F72653A20696E76616C6964206C6566
:106550006E677468210000000D4801680D4A114003
:106560000160002141608160C16082694FF6417322
:106570001A4042F080028261C16107488169074A7E
:10658000114041F00871816101680549016070475F
:10659000008002400F8130FD00900240233FDEF872
:1065A0000060C10210B540F60E2420460AF0F6FA4B
:1065B00020460AF0E5FABDE8104000F051BB08B5EE
:1065C000009002E00098401E009000980028F9D149
:1065D00008BD000002464FF0FF30062907D2DFE871
:1065E00001F01F1D0B03071B9088C0F30C007047C0
:1065F0005068C0F30C4070471168C1F30D40042887
:1066000008D9001F084A12689201F4D58906F2D50C
:10661000001D704700207047906870479068704771
:106620001078C0F3C3007047008002402DE9F041AC
:1066300000210025DFF87480DFF874C040F2F454C4
:10664000B0F5E00F12D01B4A02F1A0070523DE07C8
:1066500044F2F455C8F80C20CCF810200020CCF8F7
:106660000400CCF80000A3F1010C1BE0114A5032E9
:10667000114F05234FF48016C8F81020CCF80C20D9
:10668000ECE702EB01100660456001FB0478C0F8FE
:106690000880614504D200F11008C0F80C8000E0C9
:1066A000C260491C9942ECD3BDE8F08100900240E1
:1066B00068000020F00900205428002000B500F0F8
:1066C00043FC5DF804EB00F0E7BB00B500F04EFCC6
:1066D0005DF804EB00F0F0BB70B50022214D2B6992
:1066E0001C68002C01DA002070BDD0B123042AD42C
:1066F000E30528D5A30526D5C4F30D431B1F1A4E69
:106700003668B60102D5A40600D51B1D8B4206D9FA
:10671000002070BD29698968895C8154521C9A42A5
:10672000F8D328694FF000410160104A5169090609
:1067300003D5802151610021916041684B0404D54B
:10674000C06828610CE0002070BD090402D5D06843
:10675000286105E01168C1F3840108441030286104
:10676000012070BD680000200080024000900240BF
:1067700030B500221E4BDC682468002C01DA0020B2
:1067800030BD40F2F454A14201D9002030BD28B9F7
:1067900006E0DD68845CAD68AC54521C8A42F8D3D4
:1067A000D8684160016841F0405141F0004101600A
:1067B000104A516901F00401546904F02004214396
:1067C00002D05161002151600168CC0202D5C0683D
:1067D000D8600AE0890202D51069D86005E0116826
:1067E000C1F3840108441030D860012030BD00009E
:1067F000680000200090024010B540F202600AF0EC
:10680000B1F940F203600AF0ADF940F204600AF019
:10681000A9F94FF4C0600AF0A5F94FF0C0600AF082
:106820003BF8002001F0A2FF354C04220123114661
:10683000204601F0A7FF042202231146204601F062
:10684000A1FF04231A461821204601F09BFF0422D1
:1068500008231146204601F095FF042280231146AB
:10686000204601F08FFF274C0422012311462046C9
:1068700001F088FF042202231146204601F082FF26
:10688000A31504221821204601F07CFF04222315C1
:106890001146204601F076FFE31404221821204619
:1068A00001F070FFA31404221821204601F06AFFB2
:1068B000631404221821204601F064FF124C0223C5
:1068C00004221821204601F05DFF04231A461821F6
:1068D000204601F057FF042208231146204601F00C
:1068E00051FF042210231146204601F04BFF2023C4
:1068F00020460422BDE81040114601F043BF0000CD
:1069000000080140000C0140001001402DE9F8434F
:1069100004460E461746002500200090804600F0F1
:1069200025FA30B98A48FFF74AFE00F01FFA00281E
:106930007ED0FFF711FE012C7BD004F40060C0086C
:1069400004F4804140EA510000906B46002201218E
:10695000022000F06BFA00286CD06FF07F40FFF748
:106960002EFE7C4B186820F4B040204318607A4912
:1069700070050AD5186840F480601860886920F0B6
:10698000806206F080601043886158683843586020
:10699000724C2068C2070FD062681E68704D2E408E
:1069A000ED4315402E431E608E6926F0C00602F4AA
:1069B000407246EA92028A61820705D5A5680A6894
:1069C000684E32402A430A60420705D5E5680A68E6
:1069D000654E32402A430A60020706D525690A68D7
:1069E0004CF20206B2432A430A60C20605D5656925
:1069F0008A695E4E32402A438A6182060ED5A269B8
:106A00008E695B4D2E40ED4315402E438E610E681E
:106A100026F0800602F0800216430E60420605D57D
:106A2000E269DD696FF310051543DD61020602E0DE
:106A300040E041E089E011D5226A9E694FF6417538
:106A40002E4022EA05052E439E6151F8806F26F004
:106A5000770602F4EE4246EA12220A60C10501D529
:106A6000616A9960810501D5A16AD960410506D5A1
:106A7000E26A596840F2DE75A94311435960010585
:106A800005D5226B19683B4D294011431960C1049B
:106A900005D5626B196821F4400111431960800427
:106AA00005D5A16B186820F4602008431860012008
:106AB000BDE8F8834046FBE7DFF8BC9001226B4657
:106AC0001146002000F0B2F9BDF8000000F004000B
:106AD00000906D1C08B94D45F0D34D4501D140469D
:106AE000E6E700244FF4805000906B46002201211D
:106AF000022000F09BF908B94046D9E701226B4615
:106B00001146002000F092F9BDF8000000F02000CE
:106B10000090641C08B94C45F0D34C4501D1404667
:106B2000C6E76B4610220121002000F07FF9BDF876
:106B30000000410702D54FF4006400E00024800704
:106B40003FF50FAF44F480440BE74046B0E7000048
:106B5000FFFF8F000080024000900240B409002037
:106B60007FFFFFFDFFFFFEF8FFC001FFE73FDEFDF7
:106B7000FBFFFFFE8FDDFEFFFFFF0400374B802889
:106B80001A6851D018DC08283DD00ADC012830D022
:106B9000022833D0042803D142F004001860D960E1
:106BA0007047102834D0202837D04028F8D142F040
:106BB00040001860D9617047B0F5006F43D00DDC1C
:106BC000B0F5807F35D0B0F5007F37D0B0F5806F5D
:106BD000F1D142F480601860D9627047B0F5805FEF
:106BE00036D0B0F5005FF8D142F4005018609963D8
:106BF000704742F0010018605960704742F002008F
:106C000018609960704742F0080018601961704779
:106C100042F0100018605961704742F0200018607F
:106C200021F080009861704742F08000186019627E
:106C3000704742F4807018605962704742F40070E7
:106C400018609962704742F40060186019637047D9
:106C500042F480501860596370470000B409002066
:106C600008480021016041608160C16001614161AB
:106C70008161C161016241628162C16201634163FC
:106C800081637047B409002010B500F01F01012294
:106C9000084B8A4041F21C0403EB9011B4EB901FA7
:106CA00003D108681043086010BD0868904308606D
:106CB00010BD00000080024000F01F020121914041
:106CC000024A02EB90100160704700000080024011
:106CD000064A02EB9011096800F01F020120904063
:106CE000014201D00120704700207047008002401F
:106CF0000A794B7942EA0323074A104403640A786D
:106D0000CB7842EA03628B7849781B0443EA01217D
:106D10000A434264704700000080024010B540F210
:106D20000E5009F01FFF40F20F5009F01BFF4FF407
:106D3000A26009F017FFFFF735FC00F0CDF870B145
:106D400004212020FFF71AFF00224FF48061012068
:106D5000FFF7DCFD044918B10120086010BDFEE713
:106D60000020086010BD000058000020F8B5002584
:106D7000234E306920F01C04012009F097FD2149C1
:106D8000214A0144914202D244F0080416E01F490E
:106D90001F4A0144914202D244F00C040EE01D4906
:106DA0001D4A0144914209D31C491D4A01449142A4
:106DB00002D31C4988421DD144F0040434614FF4CD
:106DC000004000906B4600220121022000F02EF8C6
:106DD00090B11548FFF7F3FB00226B4601211046E6
:106DE00000F024F850B1BDF80000000400D40125E3
:106DF0002846F8BD2846F8BD2846F8BD2846F8BD07
:106E00000080024000D3CEFEC0E1E40040F1E9FD85
:106E100040787D0100796CFC005A6202001F0AFA7A
:106E200000990D04007A030AFFFF0400F0B5002466
:106E30000026144D2F694FF6C37C27EA0C074FF448
:106E4000F86C0CEA82124FF6FF7C02430CEAC12177
:106E50000A433A4342F00101022801D11A886A61CB
:106E60002961094A296901F00101641C09B19442B0
:106E7000F8D12969C90700D1012608B968691880C5
:106E80003046F0BD00800240FFFF0400416821F061
:106E900000414160704700000548816921F002010E
:106EA00081610448016821F004010160704700001D
:106EB00000900240008002400548016841F0040152
:106EC00001600448816941F002018161704700005E
:106ED000008002400090024010B500210020094BC4
:106EE0001A6842F001021A60074C1A6802F00102A7
:106EF000491C0AB1A142F8D11968C90700D1012083
:106F000010BD000000900240FFFF040010B507F024
:106F10006DFEFFF771FCFFF701FF0448FFF7B4FEB9
:106F20000248BDE810400A38FFF7AEBE1007040063
:106F3000002806D0026822F440020A4302600120C1
:106F4000704700207047000000B50648816921F4B1
:106F50000051816100F01CF80348016821F008012C
:106F6000016000BD009002400080024000B506486C
:106F7000016841F00801016000F00AF803488169E6
:106F800041F40051816100BD008002400090024048
:106F900010B500210020084B9A6942F480129A61D2
:106FA000064C9A6902F48012491C0AB1A142F8D336
:106FB000002A00D1012010BD00900240FFFF040014
:106FC0002DE9F04104460E46002C06D132A34FF4C1
:106FD000B17239A13CA0FAF79FFD002767600AF063
:106FE000E3FC26720AF00AFD65786770E36A1BB15C
:106FF0000022042120469847E36A1BB10022114673
:1070000020469847E36A1BB1002202212046984798
:1070100004F1100080460AF02FFD18B1002140460F
:107020000AF01CFD04F1140080460AF025FD18B199
:10703000002140460AF012FD012D0FD0042D0DD085
:10704000032D0BD0A06A002824D0BDE8F04112A384
:107050004FF4C97227A11CA0FAF75EBD94F8200076
:10706000C0F3800120F0040084F82000002911D131
:10707000A06A30B908A340F28B1225A112A0FAF73A
:107080004BFDA06A0671A76204F10C00BDE8F04157
:107090000AF01CBDBDE8F0812E2E5C6C7769702D66
:1070A000312E342E315C7372635C6170695C617087
:1070B000695F6D73672E6300636F6E6E20213D20E4
:1070C0004E554C4C00000000417373657274696F3B
:1070D0006E2022257322206661696C6564206174CC
:1070E000206C696E6520256420696E2025730D0A69
:1070F00000000000636F6E6E2D3E63757272656EE8
:10710000745F6D7367203D3D204E554C4C00000070
:10711000636F6E6E2D3E63757272656E745F6D7314
:107120006720213D204E554C4C0000002DE9FC47C6
:10713000054689461746002D07D078892A280CD2A3
:10714000384608F0DFF9BDE8FC873FA340F2BB22D8
:1071500046A14AA0FAF7E0FCF5E77E6806F10E04C6
:107160004FF4807A2088504508D12079062805D12F
:107170006079042802D16088082803D0384608F0D6
:10718000C1F9E0E7D4F80E000190A0690090291D34
:1071900006D0696821B1884205D14FF0010804E0AA
:1071A0004FF0000801E04FF00008B8F1000F01D0E7
:1071B000012300E0022304F1080201A9284600F09F
:1071C00041FDE088504503D0B0F5007F37D132E073
:1071D000B8F1000F33D0022002F042FFE080D4F873
:1071E0000E00A0616868C4F80E0095F82A00062811
:1071F00006D015A340F211322B4920A0FAF78CFCDF
:10720000A068C4F81200A089E082A0683060A0895C
:10721000B080D9F80000A060B9F80400A081D9F8C6
:107220000000C6F80600B9F804007081AA69394662
:107230002846904703E001A92846FBF77BFE384625
:1072400008F060F97FE700002E2E5C6C7769702DE6
:10725000312E342E315C7372635C6E657469665CCA
:107260006574686172702E63000000006E65746959
:107270006620213D204E554C4C0000004173736543
:107280007274696F6E2022257322206661696C65B5
:1072900064206174206C696E6520256420696E200D
:1072A00025730D0A00000000688A010870B50546C4
:1072B0000024094E04EB840006EB8000817C29B198
:1072C0008068A84202D1204600F034F9641CE4B280
:1072D0000A2CEFD370BD0000BC3E01202DE9F34F16
:1072E00085B080460A20039002900A2700244FF0C0
:1072F00000094FF0000A01904FF0000B524904EBD7
:10730000840001EB80060490B57C0A2F01D1002D8A
:1073100018D0002D22D0012D08D0022D06D24BA36B
:1073200040F22B1252A162A0FAF7F6FBB8F1000F5F
:107330000AD0D8F800007168884205D160B207B061
:10734000BDE8F08F67B209E0012D13D0022D05D3FF
:10735000F07C504502D361B202918246641CE4B2D3
:107360000A2CCBD306984FF0FF3180071CD40A2F8C
:1073700013D015E03448049950F8210030B1F07C66
:107380005845EBD361B201918346E7E7F07C48456D
:10739000E4D361B203918146E0E70698C00703D0C9
:1073A0000A2F03DAFCB22BE00846C8E702980A2845
:1073B0000FDA0298C4B2244804EB840150F821008B
:1073C00090B122A340F2711244A139A0FAF7A4FBB4
:1073D0000AE003980A2802DA0398C4B204E001988C
:1073E0000A282EDA0198C4B20A2C06D317A340F259
:1073F000831240A12EA0FAF78FFB204600F09AF8E6
:107400000A2C06D311A340F287123AA128A0FAF75A
:1074100083FB0D4804EB840100EB8105A87C30B1AF
:107420000AA34FF4C47238A121A0FAF775FBB8F192
:10743000000F02D0D8F8000068600020E87460B245
:107440007DE708467BE70000BC3E01202E2E5C6CE9
:107450007769702D312E342E315C7372635C6E65EA
:107460007469665C6574686172702E630000000068
:107470007374617465203D3D204554484152505F0E
:1074800053544154455F50454E44494E47207C7CFF
:10749000207374617465203E3D204554484152502C
:1074A0005F53544154455F535441424C45000000E2
:1074B000417373657274696F6E2022257322206692
:1074C00061696C6564206174206C696E6520256457
:1074D00020696E2025730D0A000000006172705F44
:1074E0007461626C655B695D2E71203D3D204E5577
:1074F0004C4C000069203C204152505F5441424CAA
:10750000455F53495A4500006172705F7461626C57
:10751000655B695D2E7374617465203D3D20455443
:10752000484152505F53544154455F454D50545962
:107530000000000070B50C4E00EB8004002556F8EA
:107540002400002803D007F0DDFF46F8245006EBA6
:1075500084008574C574856045600449D1F80620AF
:10756000C2604989018270BDBC3E0120888101084A
:107570002DE9FC4104460E461546002C06D148A3D1
:1075800040F275324FA153A0FAF7C6FA36B944A3B8
:1075900040F276325AA14FA0FAF7BEFA280006D17F
:1075A0003FA340F2773259A14AA0FAF7B5FA0E216B
:1075B000304608F03DF818B16FF00100BDE8FC81DD
:1075C0002146286801F0FCFD08B1544B40E02868D2
:1075D000C0F303110E2926D0A168636800EA0102F6
:1075E0000B409A420BD080B2A0F57E41A93906D05B
:1075F00014F10C0F34D0E06888B304F10C05484B4B
:10760000484A187800EB800102EB81018F7C022F41
:1076100029D32F6849688F4225D10246314620463A
:1076200000F082F8CAE701208DF8000000208DF8F4
:1076300001005E208DF80200687800F07F008DF870
:107640000300A8788DF80400E8788DF805006B46F3
:1076500004F12B023146204600F084FAAEE7FFE742
:107660006FF00300AAE7002000EB800102EB81012C
:107670008F7C022F0AD32F6849688F4206D1C2B28D
:107680001A703146204600F04FF897E7401C40B290
:107690000A28E9DB32462946204600F0B1F88DE79A
:1076A0002E2E5C6C7769702D312E342E315C737206
:1076B000635C6E657469665C6574686172702E6384
:1076C000000000006E6574696620213D204E554C17
:1076D0004C000000417373657274696F6E2022253F
:1076E0007322206661696C6564206174206C696E28
:1076F0006520256420696E2025730D0A00000000B6
:107700007120213D204E554C4C0000006970616491
:10771000647220213D204E554C4C000088810108A8
:1077200098010020BC3E012070B505460E46134866
:1077300002EB820100EB8104A07C022806D210A398
:107740004FF4537217A123A0FAF7E6F9A07C0228A0
:1077500009D1E07CE42806D3211D284600F0F0F989
:1077600008B90320A07404F10C0305F12B02314683
:107770002846BDE8704000F0F5B90000BC3E01208D
:107780002E2E5C6C7769702D312E342E315C737225
:10779000635C6E657469665C6574686172702E63A3
:1077A000000000006172705F7461626C655B617201
:1077B000705F6964785D2E7374617465203E3D204E
:1077C0004554484152505F53544154455F535441CE
:1077D000424C4500417373657274696F6E202225B7
:1077E0007322206661696C6564206174206C696E27
:1077F0006520256420696E2025730D0A00000000B5
:107800002DE9F74F82B08B46174602982B30019036
:107810004FF0FF394C46DBF80000029901F0D0FC34
:1078200098B9DBF80000C0F303110E290DD0BBF1AD
:10783000000F0AD048B101215846FFF74FFD064618
:10784000300005D505B0BDE8F08F6FF00D00F9E709
:10785000DFF8D8A006EB86080AEB8805A87C08B9F3
:107860000120A874A87C012808D0022806D230A3E1
:1078700040F2194237A141A0FAF74EF9A87C01283D
:1078800000D02FB95946029800F05AF904466FB15A
:10789000A87C02280CD344480670DDE9012005F1DC
:1078A0000C03394600F05EF904463DE02046C9E786
:1078B000012839D100253C4640F23E4611E060895E
:1078C0002189884207D1206828B119A3324637A1FF
:1078D0002AA0FAF721F9207B012801D0012502E036
:1078E0002468002CEBD185B121890022032007F008
:1078F0001FFA05466DB13946284607F081FC40B1B4
:10790000284607F0FFFD002503E03D46284607F026
:10791000E3FF45B15AF8280008B107F0F3FD4AF833
:107920002850002400E04C4620468BE7BC3E012056
:107930002E2E5C6C7769702D312E342E315C737273
:10794000635C6E657469665C6574686172702E63F1
:10795000000000006172705F7461626C655B695D5C
:107960002E7374617465203D3D2050454E44494E50
:1079700047206F7220535441424C45004173736558
:107980007274696F6E2022257322206661696C65AE
:1079900064206174206C696E6520256420696E2006
:1079A00025730D0A00000000980100206E6F207002
:1079B00061636B65742071756575657320616C6CAE
:1079C0006F776564210000002DE9F05FDDF82CB0D1
:1079D0000746884691469A46002F06D132A340F2C8
:1079E000A5423AA13DA0FAF797F800222A210320E8
:1079F00007F09EF90646300053D070892A2806D237
:107A000029A34FF4966240A134A0FAF785F875686F
:107A100005F10E040D9802F023FBE08097F82A0090
:107A2000062806D020A34FF4976244492BA0FAF70A
:107A300073F8DAF80000A060BAF80400A081DBF85F
:107A40000000C4F81200BBF80400E082D9F800007E
:107A50002860B9F80400A880D8F80000C5F806002E
:107A6000B8F8040068810A980068C4F80E000C9801
:107A70000068A0614FF4807020800820608006209C
:107A80002071042060714FF4C160A881BA69314649
:107A9000384690470446304607F034FD2046BDE89E
:107AA000F09F4FF0FF30FAE72E2E5C6C7769702D57
:107AB000312E342E315C7372635C6E657469665C62
:107AC0006574686172702E63000000006E657469F1
:107AD0006620213D204E554C4C00000041737365DB
:107AE0007274696F6E2022257322206661696C654D
:107AF00064206174206C696E6520256420696E20A5
:107B000025730D0A00000000636865636B207468CC
:107B10006174206669727374207062756620636197
:107B20006E20686F6C642073747275637420657462
:107B3000686172705F68647200000000688A010802
:107B40001FB50123064C021DCDE90213CDE9002427
:107B500000F12B031946A21FFFF736FF04B010BD3A
:107B60008E8101082DE9F0410746884616461D46DC
:107B7000D8F8044097F82A00062806D00BA340F254
:107B8000A312134913A0F9F7C7FF28682060A8883B
:107B9000A0803068C4F80600B08860810820A08109
:107BA00041463846BA69BDE8F04110472E2E5C6C5C
:107BB0007769702D312E342E315C7372635C6E6583
:107BC0007469665C6574686172702E630000000001
:107BD000688A0108417373657274696F6E2022258B
:107BE0007322206661696C6564206174206C696E23
:107BF0006520256420696E2025730D0A00000000B1
:107C000070B500240E4D04EB840005EB8000827CEF
:107C10008AB1C17C491CC9B2C174F02903D2012ABE
:107C200005D1022903D32046FFF784FC03E0032A91
:107C300001D102218174641CE4B20A2CE3D370BD2B
:107C4000BC3E01202DE9F04104460D4616461F4674
:107C500094F82A00062806D01EA340F2C31226A1DB
:107C60002FA0F9F759FF85B3286870B3214601F0BA
:107C7000A7FA50BB2878C0F303100E2826D0394647
:107C80002846FFF72BFB00281DDB304A00EB800164
:107C900002EB81000223837484603368C360B3887D
:107CA00003820023C37452F821505DB142F82130A1
:107CB000334604F12B0229462046FFF753FF28469E
:107CC00007F020FC0020BDE8F081FFE76FF00D0019
:107CD000F9E700002E2E5C6C7769702D312E342E62
:107CE000315C7372635C6E657469665C657468614F
:107CF00072702E63000000006E657469662D3E6828
:107D000077616464725F6C656E203D3D2045544828
:107D10004152505F4857414444525F4C454E000029
:107D2000417373657274696F6E2022257322206619
:107D300061696C6564206174206C696E65202564DE
:107D400020696E2025730D0A00000000BC3E012052
:107D500070B504460D4660890E2843D9606886894F
:107D60000178CA0715D0012905D006222049F8F765
:107D7000E7FA50B10DE0417859B980785E2808D112
:107D8000607B40F01000607303E0607B40F008000F
:107D90006073082E03D0B6F5C16F23D116E095F8B5
:107DA000310080061ED56FF00D01204607F040FC23
:107DB00038B110A340F24F5217A120A0F9F7ACFE42
:107DC00010E02946204601F01BFA09E095F8310041
:107DD000800607D5224605F12B012846FFF7A6F9B4
:107DE000002070BD204607F08DFB002070BD000014
:107DF000888101082E2E5C6C7769702D312E342E0F
:107E0000315C7372635C6E657469665C657468612D
:107E100072702E630000000043616E2774206D6F46
:107E20007665206F76657220686561646572206989
:107E30006E207061636B65740000000041737365B0
:107E40007274696F6E2022257322206661696C65E9
:107E500064206174206C696E6520256420696E2041
:107E600025730D0A0000000010B50446002C06D151
:107E70000AA34FF49D7216A119A0F9F74DFE4720F1
:107E800084F83200442084F83300204860612048A0
:107E9000A061204601F0B6FC002010BD2E2E5C6CC7
:107EA0007769702D312E342E315C706F72745C479F
:107EB000443332463330785C4672656552544F53D2
:107EC0005C65746865726E657469662E6300000097
:107ED0006E6574696620213D204E554C4C000000B3
:107EE000417373657274696F6E2022257322206658
:107EF00061696C6564206174206C696E652025641D
:107F000020696E2025730D0A0000000071750008BD
:107F1000519900080F4C00236422194660680FF045
:107F200014FC0128F7D109F03FFD0646206801F056
:107F3000E3FC0546304609F061FD002DEBD02168D9
:107F400028460A6990470028EDD0284607F0DAFA5B
:107F5000E1E700009C0100202DE9F0470446884637
:107F6000002C7DD0A569002D0FDA09F01DFDA56953
:107F7000002D08DAB8F1000F01D16D1EA561BDE832
:107F8000F04709F03BBD09F039FD284600F0D6FB6B
:107F90000646300064D009F007FD81460127B8F19C
:107FA000050F13D2DFE808F003070B0D10007089EE
:107FB000401C708111E07089401E70810DE0B78116
:107FC0000BE00020B08108E0F78106E034A340F226
:107FD00019523BA13EA0F9F79FFD706920B1DFF86F
:107FE0001C81D8F8004051E04846BDE8F04709F050
:107FF00005BD6069A8BB0020B6F90A1000290DDD97
:10800000A16859B1EA1705EB5272D210895C05F0EC
:10801000070207FA02F2114200D00120B18971B1C2
:1080200068B9E16859B1EA1705EB5272D210895C60
:1080300005F0070207FA02F2114200D00120F1898F
:1080400089B180B9216971B1EA1705EB5272D2107A
:10805000895C05F0070207FA02F2114203D001E041
:108060001BE006E0012020B1676104F1180009F06F
:108070002DFDD8F804A0484609F0C0FC09F094FC96
:108080008146D8F804008245ABD12468002CB0D1D9
:108090004846BDE8F04709F0B1BCBDE8F0870000F4
:1080A0002E2E5C6C7769702D312E342E315C7372FC
:1080B000635C6170695C736F636B6574732E6300DE
:1080C000756E6B6E6F776E206576656E740000005E
:1080D000417373657274696F6E2022257322206666
:1080E00061696C6564206174206C696E652025642B
:1080F00020696E2025730D0A000000008401002015
:1081000010B58EB0044600F011FB00F1A40209A1E5
:1081100001A8F9F711FD01A8F8F7FDF802460023C0
:1081200001A9204602F03CF9342101A8F8F7CAF869
:108130000EB010BD7B2266696E645F64657669630C
:1081400065223A222573227D0000000000B5034617
:1081500000F00AF85B1E012801D1002BF8D101289C
:1081600000D1042000BD000000200849CA68D207E1
:1081700001D001207047CA68D20601D5032070479C
:10818000C9684907FBD50220704700000020024063
:1081900000B5034600F00AF85B1E012801D1002B50
:1081A000F8D1012800D1042000BD000000200849BA
:1081B000CA6CD20701D001207047CA6CD20601D523
:1081C00003207047C96C4907FBD5022070470000A7
:1081D000002002400748016941F080010161064921
:1081E0000988B1F5007F03D9016D41F08001016577
:1081F0007047000000200240E0F7FF1F70B5044602
:108200002748284D284E0088B0F5007F32D92748EE
:10821000844215D23046FFF799FF00280FD1286914
:1082200040F0020028616C61286940F0400028613C
:108230003046FFF78BFF296921F00201296170BDEB
:108240003046FFF7A5FF0028F9D1286D40F0020065
:1082500028656C65E869800700D56C61286D40F081
:10826000400028653046FFF793FF296D21F0020199
:10827000296570BD3046FFF769FF0028F9D12869EC
:1082800040F0020028616C61286940F040002861DC
:108290003046FFF75BFF296921F00201296170BDBB
:1082A000E0F7FF1F002002400000FF0FFFFF07085C
:1082B00009480169094A0B06094901D54260416034
:1082C000084B1B88B3F5007F04D9036D1B0601D54D
:1082D000426441647047000000200240230167456A
:1082E000AB89EFCDE0F7FF1FF0B504460D462048FF
:1082F000204E214F0088B0F5007F26D91F488442C8
:1083000011D23846FFF722FF00280BD1306940F028
:108310000100306125603846FFF718FF316921F010
:1083200001013161F0BD3846FFF732FF0028F9D175
:10833000306D40F00100306525603846FFF728FFBA
:10834000316D21F001013165F0BD3846FFF7FEFEC9
:108350000028F9D1306940F00100306125603846CD
:10836000FFF7F4FE316921F001013161F0BD000039
:10837000E0F7FF1F002002400000FF0FFFFF07088B
:1083800003B583B0094890F9001000290BDB1021D8
:10839000074ACDE900210023012203A990F900003A
:1083A00002F03EF8039805B000BD00001400002064
:1083B0007408002070B50D46044602E02946FFF718
:1083C000DFFF14F8010B0028F8D170BD10B50028AC
:1083D00021D0114B0022001F196803E0814203D80D
:1083E0000A4649680029F9D152B11368841A9C429F
:1083F00004D1006818441060104602E0506000E0AC
:10840000186039B102680B1A934203D10B681A4401
:1084100002604968416010BDDC0100202DE9F04197
:1084200004460F466668002565602581256109F0D0
:10843000BBFA256009F0E2FA002E0AD027B13046D7
:10844000BDE8F04107F05EB83046BDE8F04105F008
:108450008CB9BDE8F081000030B5114B1A46114DC2
:1084600045F255542C60EC6804F00104521E01D012
:10847000002CF8D10CB1002030BD6960E96801F032
:1084800002015B1E01D00029F8D109B1002030BDE6
:10849000C0F30B00A8604AF6AA202860012030BD76
:1084A000FFFF0F000030004002494CF6CC4008604E
:1084B000704700000030004001490020086070470C
:1084C00000300040024945F25550086070470000F6
:1084D0000030004010B540F2026008F043FB4FF45A
:1084E0008074234603221021034800F04BF9024810
:1084F0001430046010BD00000008014002494FF430
:1085000080700860704700001408014002494FF471
:108510008070086070470000100801402DE9F041AC
:1085200005460E460024FFF7F1FF0A4F0BE0295DD8
:1085300038460EF08FFB062138460EF09DFB0028D2
:10854000F9D0641CA4B2B442F1D3BDE8F041FFF706
:10855000D5BF00000038014070B504460E4830F821
:10856000140008F0FFFA0C4D03221435A5F10C0697
:1085700055F8243056F82400102100F003F956F87D
:10858000241055F824004861BDE870404FF40061A4
:10859000024800F0E3B8000038000020000C014061
:1085A0000449044A0C3A51F8201052F82000416165
:1085B000704700004C0000200449044A0C3A51F86E
:1085C000201052F820000161704700004C0000208C
:1085D0002DE9FF41074600F0A9F8D0F8E8803846B9
:1085E000F7F799FE384435A1F9F7A6FA59E038466D
:1085F000F7F791FE08F101010091384498F8163020
:1086000098F815203149F9F797FAD8F818008668D4
:10861000046845680AE03846F7F77DFE009638445E
:10862000B31D2BA1F269F9F787FAF66A002EF2D191
:1086300012E03846F7F76FFE94F82210238C267864
:10864000A21CCDE90221CDE900633844E38A6278B7
:108650002E49F9F771FA646A002CEAD13846F7F727
:108660005AFE3844401E2AA1F9F766FA0DE0384652
:10867000F7F751FE2988EA78CDE900213844AB7834
:108680006A8B2849F9F758FA2D6A002DEFD1384640
:10869000F7F741FE3844401E23A1F9F74DFAD8F808
:1086A0001C80B8F1000FA2D13846F7F734FE04B0B1
:1086B0003844BDE8F0411CA1F9F73EBA2264657662
:1086C0006963654C697374223A5B0000488801084D
:1086D0007B226964656E7469666965723634352219
:1086E0003A25642C226964656E7469666965722234
:1086F0003A222573222C22646576696365494436E3
:108700003435223A222573227D2C0000848701080B
:108710005D2C2022636F6D6D616E64446174612213
:108720003A5B0000F48701085D7D00000048704757
:10873000840800200048704734080020042801D332
:1087400000207047044900EB400001EBC0000168C5
:108750000029F6D1002070475C3E0120016170477E
:10876000002A01D0016170474161704704494A689D
:1087700022F400024A604A6802434A6070470000DF
:10878000000001402DE9F04301F00F04CD0602D5B1
:10879000042A18D0144300224FF00F0C012707FAC7
:1087A00002F51D401AD0D0F8009096000CFA06F899
:1087B00029EA080904FA06F848EA0908282908D02D
:1087C000482908D008E044F00304C26B1A43C2638E
:1087D000E1E7456100E00561C0F80080521C92B2FB
:1087E000082ADCD3082207FA02F51D4016D0D0F87B
:1087F0000490A2F10806B6000CFA06F829EA080966
:1088000004FA06F848EA0908282902D0482902D0C3
:1088100002E0456100E00561C0F80480521C92B29C
:10882000102AE0D3BDE8F083F0B5154C002801DA3A
:10883000E36900E06368C0F30346420D120185B2AC
:10884000C0F301579540032F07D0C2020CD5032275
:10885000B240934343F0E06209E023F0E0626368D2
:1088600023F0E063636002E0AB4343F0E06201B1F8
:108870002A43002801DAE261F0BD6260F0BD000029
:108880000000014001F03EBA2DE9F04387B00446F4
:108890008846914600220121022001F0C9FF0546C9
:1088A0006FF00107002D03DA384607B0BDE8F0830A
:1088B0000026B9F1000F1DD0204600F081FE039084
:1088C00010208DF8080002208DF809001FFA88F0AA
:1088D00001F0C6FBADF80A0004960596102202A925
:1088E000284601F065FA48B31DA0F9F715F94FF0D5
:1088F000FF30DAE7019601AB1F4A01A92046FCF7D9
:1089000023FD06964FF4FA6404E00A3206926420CE
:108910000EF074FB019810B9069AA242F5DB069896
:10892000A04204DB15A0F9F7F7F83846BDE701A827
:1089300000F014FF00F044FE0390C1E740F6B830A9
:108940000690042041F20602009006ABD11F284693
:1089500001F01EFE0EA0F9F7DFF82846A5E700009B
:10896000636F6E6E656374207365727665722065E1
:1089700072726F72200D0A00A98B0008646E73205A
:10898000676574206661696C757265200A00000075
:10899000636F6E6E656374207365727665722073A3
:1089A000756363657373200D0A0000002DE9F041C3
:1089B0000E46DDE90678114605461A462846FFF7B9
:1089C00063FF0446002C0ADB32462946204600F0AD
:1089D0000FF842463946204600F0A2F80546002C22
:1089E00002DB2046FFF74EFF2846BDE8F08100007D
:1089F00070B505460E4614464FF480612448F7F7DB
:108A000061FC24A12248F9F797F8002C39D02146BF
:108A10001F48F7F762FC21A11D48F7F75EFC22A171
:108A20001B48F7F75AFC31461948F7F756FC20A1C6
:108A30001748F7F752FC1FA11548F7F74EFC22A183
:108A40001348F7F74AFC27A11148F7F746FC2BA17A
:108A50000F48F7F742FC16A10D48F7F73EFC0C480B
:108A6000F7F759FC04460A492BA0F9F755F82246B6
:108A70000749284601F0A3FF002807DC4FF0FF302C
:108A800070BD26A10248F7F728FCC4E7012070BD9D
:108A9000F3010020474554200000000020485454B2
:108AA000502F312E310D0A00486F73743A200000A8
:108AB0000D0A0000436F6E6E656374696F6E3A2035
:108AC000636C6F73650D0A004163636570743A20CF
:108AD0006170706C69636174696F6E2F6A736F6E19
:108AE0000D0A0000557365722D4167656E743A205A
:108AF00073746D3332663230370D0A004361636838
:108B0000652D436F6E74726F6C3A206E6F2D6361CA
:108B10006368650D0A000000257300002F00000047
:108B20002DE9F04781460E4617464FF4007A52462B
:108B30001B49484600F0B4F84FF0FF35002802DC2E
:108B40002846BDE8F087164916A0F8F7E5FF144857
:108B500000F0CAF8804652461149484600F0A0F895
:108B600004460F490FA0F8F7D7FF022CF3DC01D021
:108B70002846E6E70025002352460949484601F009
:108B8000BDFA0446002C05DD701922460449F7F7AA
:108B900080FB2544002CEEDC3D604046D1E7000020
:108BA000F30500202573000010B50446084601684F
:108BB000116000F0D3FD21460246BDE8104001A03F
:108BC000F8F7AABF25733A25730D0A00FEB5214CAC
:108BD00002E064200EF012FA20680128F9D10A2080
:108BE00007F0E8FC044600202060606020812046F9
:108BF00008F00CF818A12046F7F77BFB28BB4FF4D0
:108C0000904007F0D7FC0546322007F0D3FC06461B
:108C1000144A15A13046F8F78FFF02A8CDE900509D
:108C2000002341F69272314618A0FFF7BFFEC82814
:108C300005D1284608F02CFC184901200870284668
:108C40000EF048F930460EF045F920460EF042F994
:108C5000FEBD0000600000207463705F636F6E668D
:108C600069670000E80100202F696F742F7472613A
:108C70006E736D69742F6765745472616E736D697C
:108C800074436F6E6669672F257300006770752ED9
:108C900072696E677A6C652E636F6D001800002034
:108CA0002DE9F84381460E460024002700974FF037
:108CB0000A08551E0EE0002301226946484601F0CD
:108CC0001DFA002801DCCDF8008020469DF8001038
:108CD000641C3154AC4203DA9DF800000A28EAD142
:108CE00037552046BDE8F88310B5044609220EA189
:108CF0002046F7F73BFB40B109220EA12046F7F7CB
:108D000035FB10B14FF0FF3010BD627A303AA17AD6
:108D10003039E07A3038642312FB03F201EB810131
:108D200002EB4101084410BD485454502F312E31FC
:108D300020000000687474702F312E312000000074
:108D40000A46032100F060B92DE9FE4F044688462B
:108D5000656828780007870E79428A46204606F023
:108D600067FC00287ED1208904287BD360680078C6
:108D7000002878D0082876D10126DFF84891D9F864
:108D80000000C0F303110E2900D10026414600F077
:108D900017FA00B100265EB120890828E5D32046E5
:108DA00000F0B4F948B12046BDE8FE4F06F0AABB7A
:108DB0002046BDE8FE4F06F0A5BB2221204606F066
:108DC00037FC00283CD03946204606F031FC30B153
:108DD0003DA3982245A152A0F8F79EFE3CE02189D0
:108DE0000022022005F0A4FF0646002E34D071892F
:108DF00007F10800814205D233A3A12253A148A064
:108E0000F8F78AFE2146304606F0FAF930B12EA373
:108E1000A5225CA142A0F8F77FFE1DE075685146CF
:108E2000304606F005FC30B127A3AB225FA13CA081
:108E3000F8F772FE10E0204606F064FB344610E0BE
:108E40006FF02101204606F0F3FB50B11EA3B522BE
:108E500056A133A0F8F760FE2046BDE8FE4F06F0AD
:108E600051BB01E028E022E06068D9F80010E96019
:108E70005B4909682961002606704680FF20287238
:108E80006E813946204606F0D3FB30B10EA3DA22BC
:108E900054A123A0F8F740FE09E00120CDE9010824
:108EA000FF23002207490096204600F0C5FA20461D
:108EB000BDE8FE4F06F026BB2046BDE8FE4F06F09B
:108EC00021BB0000800100202E2E5C6C7769702D84
:108ED000312E342E315C7372635C636F72655C6932
:108EE0007076345C69636D702E63000069636D7029
:108EF0005F696E7075743A206D6F76696E67207069
:108F00002D3E7061796C6F616420746F20697020F0
:108F1000686561646572206661696C65640A000059
:108F2000417373657274696F6E2022257322206607
:108F300061696C6564206174206C696E65202564CC
:108F400020696E2025730D0A0000000063686563C8
:108F50006B20746861742066697273742070627526
:108F6000662063616E20686F6C6420737472756331
:108F700074207468652049434D50206865616465BC
:108F80007200000069636D705F696E7075743A20DD
:108F9000636F7079696E6720746F206E65772070DB
:108FA000627566206661696C65640A0069636D704C
:108FB0005F696E7075743A20726573746F72696E52
:108FC00067206F726967696E616C20702D3E7061F9
:108FD000796C6F6164206661696C65640A000000E9
:108FE0007C01002043616E2774206D6F7665206FD1
:108FF0007665722068656164657220696E207061B3
:10900000636B6574000000002DE9FE4307460E46C1
:10901000914600222421012005F08AFE0546280001
:109020002DD06889242806D216A34FF499721EA168
:1090300028A0F8F771FDD7F804806C68267084F8D2
:1090400001900026A680E6806868796808301C22B6
:10905000F7F71FF966806989204600F051F86080B3
:10906000D8F80C0002900120CDE90060FF2302AA8D
:109070000021284600F08EF9284606F043FABDE8A4
:10908000FE8300002E2E5C6C7769702D312E342EFD
:10909000315C7372635C636F72655C697076345CBB
:1090A00069636D702E630000636865636B2074688C
:1090B00061742066697273742070627566206361E2
:1090C0006E20686F6C642069636D70206D657373CA
:1090D00061676500417373657274696F6E20222544
:1090E0007322206661696C6564206174206C696E0E
:1090F0006520256420696E2025730D0A000000009C
:1091000010B501F031FCC04380B210BD70B505460A
:109110000024002613E06989686801F025FC2044DA
:1091200081B201EB1044A87AC00707D0C6F1010054
:10913000C6B2E0B2C4F3072141EA00242D68002D35
:10914000E9D126B1E0B2C4F3072141EA0024E043AB
:1091500080B270BD1FB5FDF7D9FE01F0A7FB00F08E
:1091600047FB0BF0E9FB00240420CDE90004C50116
:10917000029423462A460CA10D4803940EF086FC67
:10918000FFF724FD0320CDE90004029400232A46C2
:1091900008A10A4803940EF079FC03F0FFFF0020B9
:1091A0000DF052FFFBE70000444843500000000070
:1091B000FD4600084441544100000000B92D00085C
:1091C00008B50090421C07D0020005D091F831206C
:1091D000920703D4002008BD012008BD4A688242DE
:1091E00001D1002008BD896800EA01030A409342CA
:1091F00002D10143491C01D0002008BD012008BD57
:109200002DE9F05F07460E464FF0010A7D68042104
:109210002878B1EB101F05D0384606F073F900200E
:10922000BDE8F09F00F00F004FF6FF7101EA800BE0
:10923000688800F061FF01467889584502D3388973
:10924000884204D2384606F05DF90020E8E7384647
:1092500006F080FADFF834912869C9F80000A9F116
:109260000400E96801604FF00108344694F83100C9
:10927000C0070BD0201D09D0616839B1D9F80000B2
:10928000884211D02146FFF79BFF68B9B8F1000F63
:1092900004D04FF000083E48046800E02468B4425F
:1092A00000D12468002CE1D15CB9687A112808D17A
:1092B00005EB0B004088B0F5884F02D134464FF0E3
:1092C000000ABAF1000F10D0DFF8C080A8F104083E
:1092D000D8F8000048B13146FFF772FF78B998F826
:1092E0000000C0F303100E2809D06CB1E88830F0FC
:1092F000C0000ED0384606F005F9002090E7384649
:1093000006F000F900208BE7384606F0FBF8002055
:1093100086E71E4C103C6660A5603146384607F073
:10932000C1F950BB687A012814D006280DD0112845
:1093300006D03146D9F80000FFF742FF78B119E0B6
:10934000314638460DF0F0F817E03146384609F05E
:1093500089FA12E031463846FFF7F6FC0DE099F83D
:109360000000C0F303100E2804D07D6002213846AF
:10937000FFF7E6FC384606F0C5F800206060A06004
:109380000249091F0860C9F8000049E78001002070
:109390001C0100202DE9FE43DDE90A5604468846FB
:1093A00017469946E089012806D00CA340F23932CD
:1093B00013A116A0F8F7B0FB384600F0E1F850B161
:1093C000CDE9005602904B463A464146204600F011
:1093D00033F8BDE8FE836FF00300FAE72E2E5C6CD5
:1093E0007769702D312E342E315C7372635C636F3C
:1093F00072655C697076345C69702E6300000000F1
:10940000702D3E726566203D3D20310041737365CD
:109410007274696F6E2022257322206661696C6503
:1094200064206174206C696E6520256420696E205B
:1094300025730D0A000000002DE9F84FDDE90AABA5
:10944000DDF830800546894616461F46E889012822
:1094500006D027A34FF427722EA131A0F8F75CFBAA
:10946000002E3AD01421284606F0E2F818B16FF029
:109470000100BDE8F88F6C686889142806D21CA327
:1094800040F2C92231A126A0F8F746FB277284F8E2
:1094900009B0306820614520207084F801A0288937
:1094A00000F0DEFD60804FF0000AA4F806A0334F04
:1094B000388800F0D5FDA0803888401C3880B9F18C
:1094C000000F06D0D9F8000018B1E060A4F80AA097
:1094D00007E0D8F80400E060F8E7686800690090E9
:1094E0006E46D8F814303246294640469847C0E7C1
:1094F0002E2E5C6C7769702D312E342E315C737298
:10950000635C636F72655C697076345C69702E634E
:1095100000000000702D3E726566203D3D20310048
:10952000417373657274696F6E2022257322206601
:1095300061696C6564206174206C696E65202564C6
:1095400020696E2025730D0A0000000063686563C2
:109550006B20746861742066697273742070627520
:10956000662063616E20686F6C642073747275632B
:10957000742069705F686472000000007001002050
:1095800010B502460C4800680BE090F83110C9078E
:1095900006D08168146843680C400B409C420AD096
:1095A00000680028F1D10548006818B190F8311022
:1095B000C90700D1002010BD1C010020200100209F
:1095C00008B5694600F006F808B1009808BD4FF0EC
:1095D000FF3008BD2DE9FF410F466D460278A2F12C
:1095E00030010A2903D3002004B0BDE8F081002433
:1095F0000A23302A06D110F8012F782A0BD0582AD6
:1096000009D00823A2F13006092E08D804FB036410
:1096100010F8012FF6E7102310F8012FF2E7102BB6
:1096200013D1A2F16106052E03D9A2F1410105294A
:109630000BD8192E01D8612100E04121511A0A31BD
:1096400041EA041410F8012FDCE72E2A0ED0B2B143
:10965000202A14D00C2A12D00A2A10D00D2A0ED09B
:10966000092A0CD00B2A0AD00020BDE703A98D429D
:1096700001D30020B8E710C510F8012FAFE7684606
:10968000281A012101EBA000052829D2DFE800F00B
:10969000032E050E1A000020A6E7B4F1807F01D347
:1096A0000020A1E7009844EA00641FE0B4F5803F81
:1096B00001D3002098E700980199000640EA014094
:1096C000044313E0FF2C01D900208DE70098019995
:1096D000000640EA0140029940EA0120044305E007
:1096E00006A3F3220FA112A0F8F716FA1FB1204625
:1096F00000F0AAFC3860012076E700002E2E5C6C9A
:109700007769702D312E342E315C7372635C636F18
:1097100072655C697076345C69705F616464722E36
:1097200063000000756E68616E646C656400000023
:10973000417373657274696F6E20222573222066EF
:1097400061696C6564206174206C696E65202564B4
:1097500020696E2025730D0A0000000010220149C7
:1097600000F002B84C3E01202DE9FC4703460846B4
:10977000002519680191044601AFAC464FF00A0973
:10978000EA4600233E78B6FBF9F809FB1868B6FBF9
:10979000F9F139701E4608F130085B1CDBB20AF89B
:1097A00006800029EED10AE029466D1C914202DBB9
:1097B0000020BDE8FC871AF8031004F8011B5B1EAB
:1097C000DBB2F1D229466D1C914201DB0020F0E7AB
:1097D0002E2104F8011B7F1C0CF1010C0CF0FF0C76
:1097E000BCF1040FCDD3002104F8011CE1E7000017
:1097F00010B501200DF060FF0149086010BD0000A8
:10980000100000202DE9FF41044606202834A070F6
:109810000220E0702E48017821710188090A6171E7
:109820000168090CA1710068000EE0710025257225
:1098300040F2DC50208022206072283C254E3460AB
:109840007068002811D10322002101200DF059FF7A
:10985000706020B100231A4619460EF027F8002345
:109860001A46194670680DF070FF04F12B010020B4
:10987000FDF73EFA4FF4E000FCF7D8FE4FF460200D
:10988000FCF7D4FE0024144E06EB0410FDF7FEFA9C
:10989000641C052CF8D30024104E4FF4400706EB4F
:1098A00004103946FDF744FB641C052CF7D3052052
:1098B000CDE90005029500234FF4AF7208A10D48D1
:1098C00003950EF0E3F8BDE8FF41FCF7FEBE000093
:1098D000E8F7FF1F9C010020F0090020400A00204B
:1098E00045544845524E455449465F494E5055549B
:1098F00000000000157F00082DE9F0410027002539
:10990000124E02213068FCF765FE84B205213068F2
:10991000FCF760FE06462CB103222146104605F0F6
:1099200007FA07465FB13C4607E062897119606833
:10993000F6F7AFFC608905442468002CF5D10021BE
:109940000846FCF7C9FE3846BDE8F08178000020E3
:109950002DE9F0410C460025A846234EB0680028AA
:109960000BD10322002101200DF0CBFEB06020B10D
:1099700000231A4619460DF099FF0023FA221946D2
:10998000B0680DF0E2FE38B308F00EF8074617484D
:10999000026810680028FDDB01211046FCF71AFE62
:1099A000804609E0628908EB05006168F6F771FC02
:1099B0006089284485B22468002CF3D12946002010
:1099C000FCF7D6FE8046384608F018F800231A4601
:1099D0001946B0680DF06AFFB8F1010F00D0FEE73C
:1099E0000020BDE8F08100009C01002074000020F0
:1099F0002DE9F04387B088461546FEF79FFE0446E2
:109A00004FF0FF3774B1206890F8201089070BD50C
:109A1000B4F90A10002907DC0B202061384607B092
:109A2000BDE8F0833846FAE706A903F053FFDFF8F4
:109A3000389188B121680978102902D05F2020610F
:109A4000EDE74142102903D2A9EB8000006800E055
:109A5000052020613846E2E7069830B943A34FF469
:109A6000AD724AA14DA0F8F757F8069890F820106B
:109A700041F0080180F82010002304AA05A904F091
:109A80002BFA06466EB1069804F0CEF87042102804
:109A900003D2A9EB8600006800E00520206138466B
:109AA000BDE70026B8F1000F24D035B92FA340F24E
:109AB0006B1245A139A0F8F72FF80096019602968F
:109AC00003964FF010098DF8009002208DF80100E8
:109AD000BDF8100000F0C4FAADF80200059801903E
:109AE0002868102801D9C5F80090694640462A68C0
:109AF000F6F7CFFB01210698F8F7C6FF0546681C6C
:109B00002BD0042D06D319A34FF4BF7235A123A087
:109B1000F8F702F806983949C06A884206D013A3BC
:109B200040F27F1236A11DA0F7F7F6FF3D4905EB85
:109B3000450001EBC00707F037FF01460698B7F96B
:109B40000A208369DB4302FA83F27A818561084641
:109B500007F054FF2661284661E7069804F064F890
:109B60001720206138465AE7488101082E2E5C6C88
:109B70007769702D312E342E315C7372635C6170A5
:109B8000695C736F636B6574732E63006E657763D6
:109B90006F6E6E20213D204E554C4C004173736515
:109BA0007274696F6E2022257322206661696C656C
:109BB00064206174206C696E6520256420696E20C4
:109BC00025730D0A00000000616464722076616CE8
:109BD00069642062757420616464726C656E204EE5
:109BE000554C4C00696E76616C696420736F636BD1
:109BF000657420696E64657800000000597F000874
:109C00006E6577636F6E6E2D3E63616C6C6261632F
:109C10006B203D3D206576656E745F63616C6C62A0
:109C200061636B005C3E0120F8B50D461746FEF7F8
:109C300085FD04464FF0FF3614B1102F07D101E027
:109C40003046F8BD6878022801D1A8070AD012A3CF
:109C500040F2A31218A11FA0F7F75EFF05202061B4
:109C60003046F8BD68680090688800F045FA024602
:109C70006946206803F01EFF58B14142102904D202
:109C80001F49A1EB8000006800E0052020613046FC
:109C9000F8BD00202061F8BD2E2E5C6C7769702D18
:109CA000312E342E315C7372635C6170695C736F4A
:109CB000636B6574732E63006C7769705F62696EA5
:109CC000643A20696E76616C6964206164647265CF
:109CD00073730000417373657274696F6E2022257F
:109CE0007322206661696C6564206174206C696E02
:109CF0006520256420696E2025730D0A0000000090
:109D00004881010870B50025FEF718FD04462CB106
:109D1000206840B10078102803D00DE04FF0FF30EC
:109D200070BD012508E0606830B108A34FF4E67209
:109D30000EA114A0F7F7F0FE206803F075FF294686
:109D40002046FEF76BFB002070BD00002E2E5C6CE1
:109D50007769702D312E342E315C7372635C6170C3
:109D6000695C736F636B6574732E6300736F636BF1
:109D70002D3E6C61737464617461203D3D204E55CD
:109D80004C4C0000417373657274696F6E2022251C
:109D90007322206661696C6564206174206C696E51
:109DA0006520256420696E2025730D0A00000000DF
:109DB000F8B50D461746FEF7C1FC04464FF0FF36D6
:109DC00014B1102F07D101E03046F8BD68780228A1
:109DD00001D1A8070AD012A340F2E31218A120A0D3
:109DE000F7F79AFE052020613046F8BD68680090BC
:109DF000688800F081F902466946206803F0B6FEE3
:109E000058B14142102904D22049A1EB80000068DA
:109E100000E0052020613046F8BD00202061F8BD3B
:109E20002E2E5C6C7769702D312E342E315C73725E
:109E3000635C6170695C736F636B6574732E630040
:109E40006C7769705F636F6E6E6563743A20696EDC
:109E500076616C69642061646472657373000000EC
:109E6000417373657274696F6E20222573222066B8
:109E700061696C6564206174206C696E652025647D
:109E800020696E2025730D0A00000000488101083A
:109E900010B505E0C46901460A2001F0E9F8204642
:109EA0000028F7D110BD00002DE9F84F8046084684
:109EB00091469A4600260027BAF1000F12D00021E1
:109EC000CAF8001058EA00010ED04FF4803468B18F
:109ED000F6F7C6FB0646002E01DDA64206DBC920CA
:109EE000BDE8F88FCA20FBE7C820F9E7B8F1000FFA
:109EF00006D06946404604F083F818B1CA20EFE75F
:109F00002B4800903025B8F1000F0FD04046F6F7EF
:109F100002FA0746781CA04206D326A340F2351267
:109F20002CA131A0F7F7F8FD07F13105B5F5997FC0
:109F300006D320A340F2391236A12BA0F7F7ECFD8F
:109F40000A2001F015F9044620002FD02946F6F723
:109F5000B9F904F12005009868604FF0020B85F80C
:109F600001B010202870B0B200F07AF86880C4F810
:109F700004B0B9F1000F05D0D9F80800A060D9F8F5
:109F80000C00E060B8F1000F09D004F13000A061CE
:109F90003A464146F6F77DF9A1690020C8551020E0
:109FA00020616561CAF80040002099E7CB2097E75F
:109FB0007F0000012E2E5C6C7769702D312E342EBF
:109FC000315C7372635C6170695C6E657464622E8F
:109FD000630000006E616D656C656E2069732074AE
:109FE0006F6F206C6F6E6700417373657274696F79
:109FF0006E2022257322206661696C65642061747D
:10A00000206C696E6520256420696E2025730D0A19
:10A0100000000000746F74616C5F73697A65203CA6
:10A020003D204E455444425F454C454D5F53495A8F
:10A03000453A20706C65617365207265706F72744B
:10A040002074686973210000010600F47F4241EA30
:10A05000022100F47F0241EA122141EA10607047B8
:10A060000106090C41EA1020704710B507F0C8FC42
:10A0700000F0C0FD01F050F804F0CAFC00F014FC40
:10A080000CF050FA08F0ECFBFBF78CF9BDE810403F
:10A0900007F0D2BD70B50D46FEF750FB04464FF0F9
:10A0A000FF363CB1002D01DDFF2D05DA002D04DC6B
:10A0B000002502E0304670BDFF25E9B2206804F0BB
:10A0C00025F890B121680978102902D05F2020611D
:10A0D00070BD4142102904D20549A1EB80000068FF
:10A0E00000E005202061304670BD0020206170BD79
:10A0F00048810108FFF7A8BFFFF7B2BF1CB50024D5
:10A100000094019400F002F81CBD00002DE9FF4FFF
:10A1100087B00446DDF854A01646002006900027BC
:10A1200080462046FEF70AFB0446200003D1401E6D
:10A130000BB0BDE8F08F606808B106904CE00A985B
:10A14000000704D4206890F82000800712D5B4F9E5
:10A150000A0000280EDC002F07DD3946206804F0D5
:10A16000DBFA002020613846E2E70B2020614FF047
:10A17000FF30DDE72068017810290DD006A904F032
:10A18000D3F8F0B1002F0BDD3946206804F0C4FA93
:10A19000002020613846CBE706A904F075FAF0E705
:10A1A0004142102904D25D49A1EB8001096800E019
:10A1B000052121610C3002D04FF0FF30B8E70020BC
:10A1C000B6E7069830B956A340F271225CA15FA0B1
:10A1D000F7F7A2FC069860602068007810280CD081
:10A1E0000698D0F800B0BBF808002389C01A1FFAFF
:10A1F00080F94E4504D94D4603E0DDF818B0F2E78A
:10A20000B5B208982A46C119584605F0EFF82F4410
:10A2100020680078102837D04FF00108B8F1000FFF
:10A220002ED0149860B3BAF1000F29D020680178BD
:10A23000102942D0069800F1080B80890590002073
:10A24000009001900290039010208DF800000220F1
:10A250008DF80100BDF81400FFF702FFADF8020011
:10A26000DBF800000190DAF80000102802D9102075
:10A27000CAF800006946DAF800201498F6F709F8E1
:10A280000A98C00721D037E0AE4206D224A340F29C
:10A290008D2239A12DA0F7F73FFC761B56B19BF814
:10A2A0000D00C00706D1B4F90A00002802DD0A98A3
:10A2B000C007B3D04FF00108B0E70DF1100B002339
:10A2C00005AA594603F008FEB9E72068017810296D
:10A2D00009D1A9EB0501002905DD069860602089F8
:10A2E0002844208108E00021616021810078102845
:10A2F00010D0069803F039FAB8F1000F3FF41BAF05
:10A30000002F03DD3946206804F006FA00202061A2
:10A3100038460DE7069805F0F5F8EDE748810108A5
:10A320002E2E5C6C7769702D312E342E315C737259
:10A33000635C6170695C736F636B6574732E63003B
:10A3400062756620213D204E554C4C00417373656B
:10A350007274696F6E2022257322206661696C65B4
:10A3600064206174206C696E6520256420696E200C
:10A3700025730D0A00000000696E76616C69642027
:10A38000636F70796C656E2C206C656E20776F75CD
:10A390006C6420756E646572666C6F7700000000F7
:10A3A0002DE9FE4381460F4690461D464846FEF77E
:10A3B000C5F904464FF0FF3674B1206801780020DB
:10A3C00010290BD0009001902B4642463946484652
:10A3D00000F026F8BDE8FE833046FBE7022101EAE3
:10A3E000D50304215B1C01EA55010B43029002A82E
:10A3F000009042463946206804F0FEF94142102997
:10A4000004D20649A1EB8001096800E00521216121
:10A4100008B13046DEE70298DCE700004881010819
:10A420002DE9FF5FDDE90E598246884616469B46B8
:10A430005046FEF783F904464FF0FF37002C15D045
:10A4400020680078102815D0B6F5803F06D32BA3DE
:10A4500040F2323231A13AA0F7F75EFBB6B255EACC
:10A4600009001ED0B9F1100F10D10AE0384604B02F
:10A47000BDE8F09F5B46324641465046FFF790FFED
:10A48000F5E76878022801D1A8070AD01BA34FF48A
:10A490004D7236A12AA0F7F73FFB05202061384610
:10A4A000E5E70020019000903DB16868029068885F
:10A4B000FFF722FEADF80C0002E00290ADF80C00B0
:10A4C00032464146684603F0ABF9054625B9694670
:10A4D000206804F037F90546684603F059F96842E8
:10A4E000102804D22948A0EB8500006800E0052070
:10A4F00020610DB13846BAE73046B8E72E2E5C6CC5
:10A500007769702D312E342E315C7372635C61700B
:10A51000695C736F636B6574732E63006C7769702D
:10A520005F73656E64746F3A2073697A65206D7528
:10A5300073742066697420696E207531365F74000B
:10A54000417373657274696F6E20222573222066D1
:10A5500061696C6564206174206C696E6520256496
:10A5600020696E2025730D0A000000006C77697069
:10A570005F73656E64746F3A20696E76616C6964AE
:10A5800020616464726573730000000048810108F3
:10A590002DE9F04788B082460F4616469946504648
:10A5A000FEF7CCF8054600244FF0FF387DB1B9F135
:10A5B000000F0ED087B3062F3BD0B7EB18500CD04E
:10A5C0005C2454B32C61404608B0BDE8F087404697
:10A5D000FAE70E2028614046F6E7082E09D0202E23
:10A5E00007D0A6F58050063803D0042806D05C2496
:10A5F000E7E710980428E4D21624E2E7109804282C
:10A6000000D2162428680178202903D14068007CF4
:10A610008007D6D56124D4E700E01BE0012E03D0EB
:10A62000022E01D05C24CCE710980428C9D216244D
:10A63000C7E71098042801D21624C2E728680078DA
:10A64000102801D00020BFE7012EBAD0022EB8D0CA
:10A650005C24B6E70195CDF808A003970496CDF8E1
:10A66000149010A806908DF81C40012201A90848FA
:10A670000BF0B2FA286800210C3007F09AF99DF926
:10A680001C00286108B140469EE700209CE70000BE
:10A6900095A6000870B50546002D06D145A340F6E5
:10A6A00022024CA14EA0F7F737FA2C68AA68E96895
:10A6B0002869002A46D0062A5AD0A2F57062FF3ACD
:10A6C0000CD03CA340F6E20250A145A0F7F724FAD3
:10A6D0002068BDE870400C3007F0F8B908290FD0A9
:10A6E00020290DD0A1F58051063917D0042919D0A1
:10A6F00030A340F65F0249A139A0F7F70DFAE7E76A
:10A70000006828B120684068027A0A430272DFE7D5
:10A7100020684068027A8A430272D9E7216800689B
:10A72000C861D5E7006830B120684068017C41F01D
:10A7300001010174CCE720684068017C21F001012F
:10A740000174C5E701290ED0022907D019A340F6EC
:10A75000940232A122A0F7F7DFF9B9E72168007867
:10A7600049688872B4E72168007849684872AFE7A1
:10A77000012909D0022917D00EA340F6BE0227A155
:10A7800017A0F7F7C9F9A3E7006830B1206840685F
:10A79000817F41F0400181779AE720684068817F9E
:10A7A00021F04001817793E7216800684968C1F88A
:10A7B0008C008DE72E2E5C6C7769702D312E342E37
:10A7C000315C7372635C6170695C736F636B657439
:10A7D000732E630061726720213D204E554C4C0062
:10A7E000417373657274696F6E202225732220662F
:10A7F00061696C6564206174206C696E65202564F4
:10A8000020696E2025730D0A00000000756E6861D6
:10A810006E646C6564206C6576656C00756E68614D
:10A820006E646C6564206F70746E616D650000000D
:10A8300070B54FF0FF35012917D002290AD003293E
:10A8400001D0284670BDD1B2164A402003F0B8FCB2
:10A85000044617E0882A06D02020124A002103F07F
:10A86000AFFC04460EE02120F7E70E4A002110203D
:10A8700003F0A6FC04462CB194F8200040F0080038
:10A8800084F820003CB100212046F8F7FDF8411C77
:10A8900003D0A06170BD284670BD204603F0C4F906
:10A8A000284670BD597F00087047000030B587B05A
:10A8B000002108460BF0C0F9002406940594049486
:10A8C00023492248CDE90041029004AB05AA06A91C
:10A8D000204804F031F81F4804F0ACF81D4804F09B
:10A8E00032F9012203AB11460020FCF79FFABDF8B4
:10A8F0000C004107184803D5016841F010010160C0
:10A900000068164D112813D0124804F099F802205F
:10A91000FDF746FE0320287011490E4804F0DAF8CE
:10A92000002210494FF4FA6007F000F907B030BD7B
:10A9300008483130017841F010010170313804F0DD
:10A9400002F90220FDF738FE2C70E5E7F55C0108FE
:10A95000697E00087C090020580000205C0000206F
:10A9600001120008E511000818B50022009200F05D
:10A970000103002B0BD0002909DD10F8014B8DF8E5
:10A980000140491E03E030F8024B2244891E012990
:10A99000F9DC002902DD00788DF80000BDF8000028
:10A9A000104481B201EB104081B201EB104023B1A1
:10A9B000C1B2C0F3072040EA012080B218BD0023D5
:10A9C000FFF7EEBC1FB51CA11E48F7F7B5F84FF412
:10A9D000C06006F0C7F801211B48FDF725FF0020E5
:10A9E000FDF7BAFD0120FDF7B7FD0220FDF7B4FD2C
:10A9F0004FF4407004F056F9FDF76CFD002401237C
:10AA000008224FF4E13111480094F8F72BF90BF0CC
:10AA100045FA0CF0D7FC0020FDF7CEFD0120CDE972
:10AA2000000402020294002309A10B4803940DF0D4
:10AA30002DF80CF01DFCFEE744547465737430303F
:10AA400030310000E80100200002300000380140F1
:10AA5000494E49540000000055910008F0B50B30F4
:10AA6000154D20F007010024144A0FE003688B42C3
:10AA70000BD38B4205D95E1A43184768C3E90067B8
:10AA800000E04368136002C004E0021D1068002863
:10AA9000ECD12046002802D1286808B10020F0BD82
:10AAA000064A07481060074A121A22F00702C0E956
:10AAB000002401202860D7E7E0010020DC0100200D
:10AAC000B4400120B050012070B50446002C40D0A5
:10AAD000A00706D01FA34FF4A07226A12EA0F7F75F
:10AAE0001BF8384D2868844202D36868844206D334
:10AAF00018A34FF4A17234A127A0F7F70DF8286826
:10AB0000844202D36868844205D306F04DFFBDE855
:10AB1000704006F073BF2B4800210C3006F049FF4F
:10AB2000083C207930B90BA340F253122CA11AA093
:10AB3000F6F7F2FF00202071A868844200D2AC60D2
:10AB4000204605F0AFF8BDE870401E480C3006F016
:10AB5000BDBF70BD2E2E5C6C7769702D312E342EEA
:10AB6000315C7372635C636F72655C6D656D2E63DF
:10AB7000000000006D656D5F667265653A20736167
:10AB80006E69747920636865636B20616C69676EB8
:10AB90006D656E7400000000417373657274696FB7
:10ABA0006E2022257322206661696C6564206174C1
:10ABB000206C696E6520256420696E2025730D0A5E
:10ABC00000000000080100206D656D5F667265651C
:10ABD0003A206C6567616C206D656D6F727900005D
:10ABE0006D656D5F667265653A206D656D2D3E75AC
:10ABF0007365640010B51248124A20F0030010601B
:10AC00004FF4A053038000214180017100F5A05151
:10AC1000516001240C710B804B809060012102F186
:10AC20000C0006F033FF002808D0BDE8104006A352
:10AC30004FF496720CA113A0F6F76EBF10BD000082
:10AC4000F6ED0020080100202E2E5C6C7769702D37
:10AC5000312E342E315C7372635C636F72655C6D90
:10AC6000656D2E63000000006661696C6564207488
:10AC70006F20637265617465206D656D5F6D7574BD
:10AC800065780000417373657274696F6E202225C8
:10AC90007322206661696C6564206174206C696E42
:10ACA0006520256420696E2025730D0A00000000D0
:10ACB0002DE9F04700280ED0C01C4FF6FC7100EAC9
:10ACC00001050C2D00D20C254FF4A057BD4204D92C
:10ACD0000020BDE8F0870020FBE700213E4806F099
:10ACE00068FE3D4E0C3E3268B168881A80B2C5F5E8
:10ACF000A05C69E014182379002B64D123881B1A07
:10AD0000083BAB425FD3238805F1140C1B1A083BA8
:10AD10004FF00108634519D3431908331FFA83FC28
:10AD200002EB0C034FF0000983F80490B4F8009094
:10AD3000A3F800905880A4F800C084F80480188814
:10AD4000B84205D0931C20F803C001E084F80480C9
:10AD50008C4213D1706801E0098811440B790BB162
:10AD60008142F9D1B160814208D0087930B11BA38A
:10AD700040F2622221A128A0F6F7CEFE164806F086
:10AD8000A5FE601971680830884206D913A340F205
:10AD900066222CA120A0F6F7BFFE04F10805A90742
:10ADA00006D00EA34FF41A7232A11BA0F6F7B4FE20
:10ADB000A10706D009A340F26A223AA116A0F6F72D
:10ADC000ABFE284685E7105A844593DC024806F01E
:10ADD0007DFE00207DE70000140100202E2E5C6C1B
:10ADE0007769702D312E342E315C7372635C636F22
:10ADF00072655C6D656D2E63000000006D656D5FB2
:10AE00006D616C6C6F633A20216C667265652D3ED6
:10AE10007573656400000000417373657274696F37
:10AE20006E2022257322206661696C65642061743E
:10AE3000206C696E6520256420696E2025730D0ADB
:10AE4000000000006D656D5F6D616C6C6F633A2092
:10AE5000616C6C6F6361746564206D656D6F727990
:10AE6000206E6F742061626F76652072616D5F6520
:10AE70006E642E006D656D5F6D616C6C6F633A2062
:10AE8000616C6C6F6361746564206D656D6F727960
:10AE90002070726F7065726C7920616C69676E6585
:10AEA000642E00006D656D5F6D616C6C6F633A20A0
:10AEB00073616E69747920636865636B20616C6986
:10AEC000676E6D656E7400002DE9F0470746C91C7A
:10AED0004FF6FC7001EA00040C2C00D20C244FF455
:10AEE000A0594C4502D90020BDE8F087DFF8F88072
:10AEF000D8F80000874203D3D8F80400874206D36D
:10AF00003AA34FF4C37241A146A0F6F705FED8F864
:10AF10000000874203D3D8F804108F4205D306F00F
:10AF200043FD06F06BFD3846DEE7A7F10805281A59
:10AF300086B22888801B08381FFA80FA544506D943
:10AF40002AA34FF4CC7242A136A0F6F7E5FD544592
:10AF500002D94FF00000C7E701D13846C4E72248C4
:10AF60004FF0000100F10C0006F023FD2888D8F80E
:10AF70000020811800230879E8B104F1140050453D
:10AF800013D83019083080B21118D8F80840A142FF
:10AF900001D2C8F808100B712B880B804E802880D6
:10AFA0000988494501D0921C88520F480C3006F0A0
:10AFB0008DFD384698E7B1F800C03019083080B2EE
:10AFC000D8F808408C4202D11118C8F8081011189E
:10AFD0000B71A1F800C04E80288009884945E4D053
:10AFE000921C8852E1E70000080100202E2E5C6CC4
:10AFF0007769702D312E342E315C7372635C636F10
:10B0000072655C6D656D2E63000000006D656D5F9F
:10B010007472696D3A206C6567616C206D656D6F47
:10B0200072790000417373657274696F6E20222516
:10B030007322206661696C6564206174206C696E9E
:10B040006520256420696E2025730D0A000000002C
:10B050006D656D5F7472696D2063616E206F6E6CDB
:10B060007920736872696E6B206D656D6F727900FF
:10B0700070B505460C46002C14D0A00706D00AA3D4
:10B0800040F2BB1210A118A0F6F746FD06F08CFCAA
:10B09000204951F82520226041F82540BDE8704044
:10B0A00006F0ACBC70BD00002E2E5C6C7769702D74
:10B0B000312E342E315C7372635C636F72655C6D2C
:10B0C000656D702E630000006D656D705F66726562
:10B0D000653A206D656D2070726F7065726C7920B5
:10B0E000616C69676E656400417373657274696F42
:10B0F0006E2022257322206661696C65642061746C
:10B10000206C696E6520256420696E2025730D0A08
:10B110000000000008020120F0B50020401C80B2B1
:10B120000D28FBD3104820F0030100200E4B0F4DDB
:10B130000026373B05F11A0443F82060002209E09D
:10B1400053F820700F6043F8201035F81070394420
:10B15000521C92B234F810709742F1D8401C80B261
:10B160000D28E9D3F0BD00003F020120B6800108A0
:10B1700070B505460D2D08D310A34FF4C77217A163
:10B180001EA0F6F7C9FC002070BD06F00DFC0646B7
:10B19000254850F825405CB1216840F82510A007EB
:10B1A00006D006A340F29F1220A114A0F6F7B4FC2B
:10B1B000304606F023FC204670BD00002E2E5C6C4D
:10B1C0007769702D312E342E315C7372635C636F3E
:10B1D00072655C6D656D702E630000006D656D704D
:10B1E0005F6D616C6C6F633A2074797065203C20F0
:10B1F0004D454D505F4D415800000000417373654F
:10B200007274696F6E2022257322206661696C65F5
:10B2100064206174206C696E6520256420696E204D
:10B2200025730D0A00000000080201206D656D7095
:10B230005F6D616C6C6F633A206D656D702070722C
:10B240006F7065726C7920616C69676E656400006F
:10B250002DE9F0411D4E1E4D314628460BF04AFDAA
:10B260001C4C98B120883F2809D228460BF0EEFCF0
:10B270002288A11C50542088401C208002E02846CF
:10B280000BF0E4FC314628460BF02BFD208888B1FA
:10B29000114F284639460BF02DFD58B1012084F896
:10B2A000520028460BF0D2FC39462846BDE8F04152
:10B2B0000BF017BD28460BF0C9FC314628460BF0B1
:10B2C00010FD0CF05BFC6064BDE8F0810503050037
:10B2D00000380140843F01200403040030B50246D9
:10B2E0004FF6FF70064D07E012F8013B4340DBB21A
:10B2F000040A35F813006040491E89B2F4D230BD0B
:10B300004C84010810B5044600224FF480710548B2
:10B31000FDF726FA54210448F4F7D4FF0248C46428
:10B32000012010BD00080140843F01201346012286
:10B33000AFF300802DE9FC4104461D468DF8004026
:10B3400001208DF80100080A8DF802008DF8031025
:10B35000100A8DF804008DF8052006216846FFF7D5
:10B36000BDFF1D4F38808DF80600000A8DF80700DC
:10B3700064220821684600F0EBF8184EF06C00F0EB
:10B38000CBF828B1B078A04204D00020BDE8FC8101
:10B390000020FBE7F078012801D00020F6E73179A2
:10B3A0003446C91CB01CFFF799FF38800B4922793D
:10B3B000491DC3B2515C8B4205D1084B9B1DD35C28
:10B3C000B3EB102F01D00020E0E71DB1711D28461E
:10B3D000F4F75FFF0120D9E7B0010020843F01208E
:10B3E0007CB515461C4623462A4600F031F858B372
:10B3F000002015E0154991F85010012914D004EBF4
:10B4000040010A8801929DF805208DF800209DF8E2
:10B4100004208DF80120BDF800200A80401C80B275
:10B42000A842E7D301207CBD04EB40010A880192C9
:10B430009DF804208DF800209DF805208DF801204E
:10B44000BDF800200A80E9E700207CBD843F012090
:10B450002DE9FC4104461D468DF8004003208DF87F
:10B460000100080A8DF802008DF80310100A8DF80B
:10B4700004008DF8052006216846FFF72FFF244FB2
:10B48000F8808DF80600000A8DF807006422082174
:10B49000684600F05DF8642000F03EF830B11D4EC3
:10B4A000B078A04204D00020BDE8FC810020FBE77A
:10B4B000F078032801D00020F6E731793446C91C22
:10B4C000B01CFFF70BFFF88012492279491DC3B267
:10B4D000515C8B4206D10F4B31469B1DD25CB2EBC7
:10B4E000102F01D00020DFE785B1002006E00A1808
:10B4F0005479937953719471801CC0B20A79824255
:10B50000F5D80A79491D2846F4F7C3FE0120CBE798
:10B51000B0010020843F012070B505460CF02EFBE1
:10B52000044605EB8505094E0CF028FB001BB0EB2B
:10B53000450F01D9002070BD96F85200012803D0B4
:10B540000520F7F7EDFCEFE7308870BD843F012060
:10B550002DE9F05F06460F46DFF8988002E00120F3
:10B56000F7F7DEFC98F848000128F8D0012088F8A9
:10B570004800402108F10200F4F7A4FE4FF0000952
:10B58000A8F8009088F852900CF0F8FA0BF088FCBC
:10B59000DFF864B04FF4807A012251465846FDF737
:10B5A000DFF80120F7F7BCFC0024144D0BE0315DFF
:10B5B00028460BF04FFB072128460BF05DFB0028C7
:10B5C000F9D0641CA4B2BC42F1D3062128460BF08A
:10B5D00053FB0028F9D0002251465846FDF7C0F829
:10B5E0000BF06CFC88F8529088F848900120BDE878
:10B5F000F09F0000843F0120000801400038014016
:10B60000014981F850007047843F01201CB58DF836
:10B61000000005208DF80100080A8DF802008DF861
:10B6200003100020002A21D0FF218DF804108DF88E
:10B63000050006216846FFF751FE104908818DF884
:10B640000600000A8DF80700642208216846FFF70B
:10B650007FFF0B4CE06CFFF75FFF50B10822A11C8D
:10B660006846F4F76DFE30B100201CBD8DF8040073
:10B67000DDE700201CBD01201CBD0000B001002042
:10B68000843F01201CB58DF8000006208DF80100D4
:10B69000080A8DF802008DF80310100A8DF80400D6
:10B6A0008DF8052006216846FFF718FE0E494881EF
:10B6B0008DF80600000A8DF807006422082168460C
:10B6C000FFF746FF094CE06CFFF726FF38B1082270
:10B6D000A11C6846F4F734FE18B100201CBD002000
:10B6E0001CBD01201CBD0000B0010020843F0120D2
:10B6F0002DE9FC4781460F4615461E46012D15D003
:10B70000092000EB45084046FFF7A8F9044684F8F5
:10B71000009010216170390AA170E770290A217127
:10B7200065716900A1710020364F1FE0328802B0B8
:10B7300039464846BDE8F047FFF7A4BF97F85010D8
:10B74000012941D006EB4001098801919DF80410C0
:10B750008DF800109DF805108DF8011004EB4001E4
:10B76000BDF80020A1F80720401C80B2A842E5D314
:10B77000072000EB450081B22046FFF7AFFD224EC7
:10B78000B08104EB4501C871000A08721FFA88F104
:10B7900064222046FFF7DCFEF86CFFF7BDFE30B3F5
:10B7A00006212046FFF79AFDB081A071000AE071E2
:10B7B0000822B91C2046F4F7C3FDE8B12046FCF787
:10B7C00005FE0020BDE8FC8706EB400109880191D9
:10B7D0009DF805108DF800109DF804108DF80110EB
:10B7E00004EB4001BDF80020A1F80720BCE720468B
:10B7F000FCF7ECFD0020E5E72046FCF7E7FD012023
:10B80000E0E70000843F0120B00100202DE9F0476F
:10B810000646089F884691461D4605F1200004F023
:10B820000FF9044620001AD000F0DDFC04F10800F6
:10B83000824604F018FA5046F16A04F00CFAC4F893
:10B840000C80A4F81090258304F12000E06167616A
:10B850002A46316AF4F71DFD2046BDE8F087002036
:10B86000FBE710B50446002C07D0204600F0ADFCE5
:10B870002046BDE8104004F0EFB810BD806A4021BA
:10B88000B1EB102F01D80120704700207047000055
:10B89000FEB505460C4602A804F0E5F902A8E96ADF
:10B8A00004F0D9F904F10800E96A04F0D4F905F1CB
:10B8B0005000064604F0DAF8228BE169286AF4F7B2
:10B8C000E8FC218B02AA284601F0B8F9304604F0C2
:10B8D000D3F8208AE168CDE90010054B40F26312ED
:10B8E00004A10EA0F6F718F919A0F6F715F9FEBD98
:10B8F000A88101082E2E5C6D717474636C69656E8D
:10B90000745C6D717474636C69656E745C6D717474
:10B9100074636C69656E742E6300000025733A25AC
:10B920006420257328292E2E2E20726573656E647F
:10B93000202564207061636B6167652C20706163F2
:10B940006B65745F696420697320256420000000C2
:10B950000A0000002DE9F04104460D46164604F1A8
:10B960006000074600F042FC10B10020BDE8F08105
:10B97000236E1C6809E0188AB04204D1D868A84236
:10B9800001D10120F2E723461C68BB42F3D100201D
:10B99000ECE72DE9F8430646089C0F469046994689
:10B9A0000025424639463046FFF7D4FF18B16FF004
:10B9B0001600BDE8F8834B464246394630460094AF
:10B9C000FFF724FF04464CB1304600F070F806F152
:10B9D0006001204600F0F4FB2846EAE76FF0020021
:10B9E000E7E72DE9F04106460F4606F16000804684
:10B9F00000F0FCFB002832D1304600F04FFA01285D
:10BA00002DD1306E056828E0044604F1080004F0EA
:10BA10002DF908B9012F1ED0E268042A0AD0052AA0
:10BA200008D0062A06D0072A04D0092A07D00B2AF4
:10BA300005D00AE021463046FFF72AFF0BE0606997
:10BA400018B100F068FC002060612046FFF709FF94
:10BA5000304601F08FFB284605684045D4D1BDE84B
:10BA6000F0812DE9F04706460F4690461D4606F147
:10BA70006000814600F0BAFB10B10020BDE8F087FD
:10BA8000306E04680FE0018A41450AD1C168B942AD
:10BA900007D10DB141692960FFF7E3FE304601F09F
:10BAA00069FB204604684845EDD10020E6E770B503
:10BAB000044604F15400054603F0D8FFA06A00F5DF
:10BAC0008070A0622846BDE8704003F0D5BF2DE924
:10BAD000F041054605F16000804600F087FB002735
:10BAE000A0B92C6E26680CE0204600F06EFB606961
:10BAF00010B100F010FC6761204603F0ADFF344642
:10BB000026684445F0D1404600F063FB95F82800D4
:10BB1000A86205F15800804600F068FB80B9AC6D62
:10BB2000266808E0204600F050FBE760204603F05E
:10BB300093FF344626684445F4D1404600F049FB63
:10BB40002846BDE8F0414FF0FF3101F023B900F085
:10BB500001B800002DE9F0419AB004466FF00306E9
:10BB6000002018905822664902A8F4F792FBC4B14D
:10BB7000204600F093F9012816D0D4E903120023DF
:10BB8000A06E03F011F8A06E03F00AF80546280035
:10BB90000CD0A06E50B103F015F828461AB0BDE8DD
:10BBA000F0816FF00100F9E70020F7E7544B40F215
:10BBB000E1321C3B53A15DA0F5F7AEFF65A0F5F7A0
:10BBC000ABFFA08CADF8200094F82800C0F3400033
:10BBD0008DF8220094F82800C0F303108DF81000AF
:10BBE0002068059060681290A0681590A06AC1074F
:10BBF00011D000F001008DF82300A06C80680E9039
:10BC0000A06C00788DF84500A06C40788DF8440059
:10BC1000A06C40680B90A18C4FF47A70414304F102
:10BC2000740004F018F804F15000804603F01EFF81
:10BC300002AA616B206AF5F75DFD071E12DD19A8E7
:10BC4000E16A04F008F819AA3946204600F0F6FF28
:10BC5000051E07D119AA0221204601F0DFFB0228A8
:10BC60000DD03546C5B1A06E02F0ACFF00212046D4
:10BC700001F090F8404603F0FFFE28468EE718A931
:10BC8000481C236BE269F5F7CFFB012801D035464C
:10BC9000E8E79DF86050E5E7E06E40B101212046FD
:10BCA00001F078F8A06A20F00C00A062E2E73220F0
:10BCB0000321CDE900104FF400632246264927A056
:10BCC00003F09FFFE06650B10121204601F062F8C9
:10BCD000E06E03F0BCFFE06E03F0B6FFE2E7A06E9B
:10BCE00002F070FF3546064B40F217421C3B05A19F
:10BCF0001FA0F5F711FF17A0F5F70EFFD2E7000020
:10BD0000288201082E2E5C6D717474636C69656EF7
:10BD1000745C6D717474636C69656E745C6D717460
:10BD200074636C69656E742E6300000025733A2598
:10BD30006420257328292E2E2E206D7174742063A3
:10BD40006F6E6E65637420737563636573732E2EF7
:10BD50002E0000000A00000011D600086D717474F6
:10BD60005F7969656C645F74687265616400000086
:10BD700025733A256420257328292E2E2E206D71D7
:10BD80007474207969656C642074687265616420DC
:10BD90006372656174206661696C65642E2E2E0085
:10BDA0002DE9F84380460F469146012400250020E6
:10BDB00038606D1C042D13DC4B4601226946D8F80F
:10BDC000680002F0FDFE01280AD19DF80060386885
:10BDD00006F07F0101FB04003860E4013006E8D47E
:10BDE0002846BDE8F8832DE9F04192B080460E4622
:10BDF00017464FF0FF343146404600F052F80546F2
:10BE000055B13A46314601A800F0F2FA2A6901A973
:10BE10004046904700240DE0D8F87C0050B13A46E7
:10BE2000314601A800F0E4FAD8F87C2001A9404688
:10BE300090470024F868F4F76EFA0146F868F4F7C2
:10BE400041FAD6E90110F4F73DFA12B02046BDE8F8
:10BE5000F081F8B504464FF0FF35684603F003FF64
:10BE60006846E16A03F0F7FE04F15000064603F06D
:10BE7000FDFD616B206AF5F714FD0146002904DD24
:10BE80006A46204600F0DAFE0546304603F0F4FD2F
:10BE90000321204600F07EFF2846F8BD90F94C00B3
:10BEA00070472DE9F0410F46846D256800F1580672
:10BEB0000FE0E16859B13846F5F7BFFB20B93946C4
:10BEC000E06801F0B3F910B12046BDE8F0812C46DE
:10BED0002568B442EDD10020F7E770B5044604F1BF
:10BEE0005400054603F0C2FDE08CA0F57F41FE3909
:10BEF00006D0401CE084284603F0BEFDE08C70BDF7
:10BF00000120F7E72DE9F0470646DDE90989089F9A
:10BF100014461D46304600F001FF4146304600F011
:10BF2000FDFF3946304600F045FF2146304601F01E
:10BF300055F82946304600F0B5FF0121304600F0A3
:10BF4000AFFE4946304600F071FF3046FFF7FFFD77
:10BF500040B2BDE8F087000070B504460C2003F045
:10BF60006FFDA066E8B30146002008604860886065
:10BF70000121E18494F8281021F0020121F001014F
:10BF800044F62062E26284F84C0021F00C01C9B250
:10BF9000E063206460643222A28421F0F001403129
:10BFA000A1624FF47A71A163A064A061A067E06709
:10BFB0004FF480652946204600F06EFD2946204654
:10BFC00001F044FA04F1580000F00DF904F16000AA
:10BFD00000F009F904F1500003F040FD04F15400B1
:10BFE00000E00BE003F03AFD04F1700003F03BFECB
:10BFF00004F1740003F037FE002070BD064B40F2E0
:10C000005B4206A10FA0F5F787FD18A0F5F784FDA8
:10C010006FF0020070BD0000AB8201082E2E5C6D37
:10C02000717474636C69656E745C6D717474636C47
:10C0300069656E745C6D717474636C69656E742E81
:10C040006300000025733A256420257328292E2ECD
:10C050002E206D616C6C6F63206D656D6F72792041
:10C060006661696C65642E2E2E0000000A000000D7
:10C0700010B5FFF713FF032804D0012805D06FF097
:10C080000D0010BD6FF0170010BD002010BD70B581
:10C0900006460D462846F4F73EF904463046F4F7C6
:10C0A0003AF9A04201D0002070BD22462946304610
:10C0B000F4F75CF908B1002070BD012070BD0000EC
:10C0C00038B504462046FFF7D3FF05460DB1284694
:10C0D00038BD04F1700003F0C9FD28B904F1740003
:10C0E00003F0C4FD00282CD094F8280010F00C0FA9
:10C0F00013D0154B40F2AE4214A11EA0F5F70CFD73
:10C1000024A0F5F709FDA06E02F05CFD0221204697
:10C1100000F040FE6FF00D0513E0616B206AF5F74B
:10C12000C3FB0146002904DD6A46204600F086FD77
:10C130000546A06A4FF0804101EB30104FEA3070A5
:10C14000A062284638BD0000F28301082E2E5C6DE7
:10C15000717474636C69656E745C6D717474636C16
:10C1600069656E745C6D717474636C69656E742E50
:10C170006300000025733A256420257328292E2E9C
:10C180002E2070696E67206F75747374616E6469B8
:10C190006E6700000A00000010B5802003F050FC1C
:10C1A00004464CB180212046F4F78CF82046FFF776
:10C1B000D3FE18B1002010BD002010BD204610BDD8
:10C1C0004B680A461946F5F7C5BDD0E90010F5F7EA
:10C1D000C6BD10B504462046F5F7C4FD2046BDE8AF
:10C1E0001040AFF3008000604060704701688142FA
:10C1F00001D1012070470020704700002DE9FC416B
:10C2000004460025002C14D004F158000746FFF71F
:10C21000EDFF48B1134B40F2C15213A11CA0F5F73A
:10C220007BFC27A0F5F778FCA46D266840F2C75880
:10C2300013E06FF00100BDE8FC81E16859B16D1CAD
:10C24000CDE90051074B424607A11EA0F5F764FC5B
:10C250001BA0F5F761FC34462668BC42EDD10020F6
:10C26000E9E700001C8401082E2E5C6D7174746374
:10C270006C69656E745C6D717474636C69656E7401
:10C280005C6D717474636C69656E742E630000007C
:10C2900025733A256420257328292E2E2E207468B4
:10C2A00065726520617265206E6F207375627363BD
:10C2B000726962656420746F706963732E2E2E003C
:10C2C0000A00000025733A256420257328292E2EA4
:10C2D0002E5B25645D2073756273637269626520ED
:10C2E000746F7069633A2025730000002DE9F041F6
:10C2F00007460D461646142003F0A2FB044644B13F
:10C300002046FFF770FF25722661E7602046BDE8F2
:10C31000F0810020FBE710B50446002C07D0204632
:10C32000FFF753FF2046BDE8104003F095BB10BD5A
:10C330002DE9FC4104460E4604F158000746FFF77C
:10C3400055FF10B10020BDE8FC81A46D256817E001
:10C35000E06898B1F168FFF79AFE78B1F068E1689B
:10C36000CDE90010084B4FF4E77208A11148F5F72A
:10C37000D3FB11A0F5F7D0FB0120E4E72C4625689C
:10C38000BC42E5D10020DEE7C08101082E2E5C6DA5
:10C39000717474636C69656E745C6D717474636CD4
:10C3A00069656E745C6D717474636C69656E742E0E
:10C3B00063000000108B01080A00000070B50446FD
:10C3C0000D46002C0AD04DB129462046FFF7B0FF9C
:10C3D00038B12846FFF79FFF002070BD6FF00100C5
:10C3E00070BD04F158012846FFF7EAFE002070BD39
:10C3F00070B5054616464C683F2C00DB3F24896823
:10C4000022462846F3F745FF002028552E6470BDCC
:10C410002DE9F04105468846174600242E6BBE42A2
:10C4200000D93E46404603F02CFC03463246E969FB
:10C43000A86E02F0C5FB28B104442A6B3E1B96424D
:10C4400000D31646BC4201DA0028EBD1BDE8F081EA
:10C45000F8B504460E460020009032466946204654
:10C4600000F08AFB009B0E2B31D2DFE803F007308F
:10C47000301F102424103015301A3029083023D1F1
:10C480001548F5F749FB15A0F5F746FB1CE03146CA
:10C49000204600F025F817E03146204600F0DFFD89
:10C4A00012E03146204600F095FF0DE0314620466F
:10C4B00000F09CF908E03146204600F0C7FA03E09E
:10C4C000A06A20F00C00A0622046FFF7F9FD0028CA
:10C4D00000D10098F8BD0000AC8A01080A000000F5
:10C4E0001FB504462046FFF7C3FD00280FD1206B7F
:10C4F000009003AA02A901A8E369F4F76FFF0023E3
:10C50000BDF80C209DF804102046FFF7AAFA04B0ED
:10C5100010BD00002DE9F0438BB0064614464FF0E5
:10C52000FF354FF00008CDF82080CDF8248007912A
:10C530003046FFF7B3FC012806D0C4F808806FF03E
:10C540000D000BB0BDE8F083E06820B1A16811B91F
:10C55000F3F7E1FEA060A068716B884208D939A0AA
:10C56000F5F7DAFA47A0F5F7D7FA6FF00700E8E732
:10C5700006F15000814603F079FA207850B1304638
:10C58000FFF77CF910B16FF015053EE03046FFF77C
:10C59000A4FCA080D4E90210CDE9050107A802ABF4
:10C5A00007C807C3A0886178CDE90010237800226E
:10C5B000716B306AF5F77BF90746002F25DD0AAA73
:10C5C0003946304600F03AFB051E1ED12078E0B116
:10C5D0000121304600F0DEFC2078012802D002283C
:10C5E0000AD012E0CDF80080BBB2A2880421304608
:10C5F000FFF7CFF9054608E0CDF80080BBB2A2886E
:10C6000005213046FFF7C5F90546C4F808804846BD
:10C6100003F032FA15F1160F01D0E81C10D11A4BB5
:10C6200040F2AA5219A123A0F5F776FA15A0F5F762
:10C6300073FAB06E02F0C6FA0221304600F0AAFB8F
:10C6400028467EE77075626C697368207061796C4A
:10C650006F6164206C656E20697320697320677256
:10C660006561746572207468616E20636C69656EC3
:10C6700074207772697465206275666665722E2E05
:10C680002E0000000A0000000F8401082E2E5C6DB1
:10C69000717474636C69656E745C6D717474636CD1
:10C6A00069656E745C6D717474636C69656E742E0B
:10C6B0006300000025733A256420257328292E2E57
:10C6C0002E207468657265206973206E6F74206512
:10C6D0006E6F756768206D656D6F7279207370611C
:10C6E000636520746F207265636F72642E2E2E0056
:10C6F0002DE9FC4104460F46154601A803F0B3FAA4
:10C7000001A8E16A03F0A7FA04F15000804603F0A3
:10C71000ADF9052D04D0062D15D06FF0090525E0E3
:10C72000009700230622616B206AF4F7B7FF0646E4
:10C7300000200090B3B23A4607212046FFF729F9BE
:10C7400005469DB907E0009700230722616B206A28
:10C75000F4F7A4FF0646002E02DC6FF00A0505E0A0
:10C7600001AA3146204600F069FA0546404603F02A
:10C7700083F92846BDE8FC81F8B507460D46144606
:10C780001E460C2003F016FF0090601C03F012FF01
:10C7900000998860611CF3F795FD009822463946A0
:10C7A0008068F3F776FD3046F3F7B5FD401C03F0E3
:10C7B00001FF009948603046F3F7ADFD411C009839
:10C7C0004068F3F77FFD009831464068F3F7C5FDF8
:10C7D000009804808570044800231A466946406822
:10C7E0000BF064F8F8BD0000000000202DE9F043D4
:10C7F0008DB0044688460026002708972046FFF79C
:10C8000037FC0546280002D00DB0BDE8F08308AA29
:10C8100009ABE169206BCDE90132CDE903100AA82B
:10C82000009006A8031D421C05A9801CF4F72CFEED
:10C83000012802D06FF01000E6E70598C0B28DF82D
:10C84000180070B304F15000814603F00FF99DF811
:10C850001800012802D002280BD014E0BDF81C00FB
:10C86000009000230422616B206AF4F717FF06464C
:10C8700009E0BDF81C00009000230522616B206ACE
:10C88000F4F70CFF0646002E02DC6FF0110505E000
:10C8900042463146204600F0D1F90546484603F0AD
:10C8A000EBF8002D01DA2846AEE79DF818000228C3
:10C8B00005D006AA0AA92046FFF795FA0FE0B3B201
:10C8C0000097BDF81C2006212046FFF762F80546B8
:10C8D000173004D006AA0AA92046FFF784FA284692
:10C8E00092E700008AB00646FBF720FF0446394D68
:10C8F0004FF0FF3738464FF47A794FF0780812E05E
:10C9000048460AF07BFBE28A33A108A8F5F714F940
:10C9100032A0CDE9010833A1002300911A4635A1C8
:10C920003046FFF7EFFA0028EADB35A000905023ED
:10C93000364A37A10120F4F7D1FC012028603B4B97
:10C94000002204F14A01304600F0C2FB00220492AA
:10C950000592069207923046FFF750FC686800285F
:10C9600033D000230A2203A90AF0EFFE00282CD0BE
:10C97000039A1088069090788DF8100090680790C0
:10C98000516804AA3046FFF7C5FD18B13046FFF7DD
:10C9900060FAAFE70AF050FEA860254968230868EE
:10C9A000421C0A6023A1CDE90010184A18A10120F9
:10C9B000F4F794FC039840680AF08CFA03988068B6
:10C9C0000AF088FA03980AF085FA64200AF016FB48
:10C9D000C4E70000000000202568750031383833B6
:10C9E0000000000033362E3133342E32332E3131F5
:10C9F000000000006474755F73696D706C65000001
:10CA00004D5154542053746172740000A47E010887
:10CA10002E2E5C53797374656D5C736F75726365EC
:10CA20005C7379735F6D7174742E630059610108D2
:10CA3000240000204D5154542053656E64204D65F0
:10CA40007373616765204E6F3A2564001FB5044615
:10CA50002046FFF70DFB00280BD1206B009003AAA6
:10CA600002A901A8E369F4F7B9FC012803D06FF02B
:10CA7000080004B010BD9DF80420BDF80C1020463D
:10CA8000FFF736FE0023BDF80C209DF80410204669
:10CA9000FEF7E7FFEDE7000070B504460D46002CF9
:10CAA00014D0E06908B102F0D7FF2563022D03D945
:10CAB0006FF07040854202D34FF480602063206B9A
:10CAC00002F0BEFFE06168B1206B70BD0C4B40F21C
:10CAD0002B420CA115A0F5F71FF81CA0F5F71CF8C8
:10CAE000002070BD064B40F2394206A118A0F5F7B0
:10CAF00013F816A0F5F710F86FF0020070BD0000F3
:10CB0000808201082E2E5C6D717474636C69656E91
:10CB1000745C6D717474636C69656E745C6D717452
:10CB200074636C69656E742E6300000025733A258A
:10CB30006420257328292E2E2E20636865636B20C0
:10CB4000666F72206572726F722E00000A0000001C
:10CB500025733A256420257328292E2E2E206D61F9
:10CB60006C6C6F632072656164206275662066611B
:10CB7000696C65642E2E2E002DE9FC4104460E469C
:10CB800090460020019001250090002E16D04046CE
:10CB900003F069F84046E16A03F05DF8404603F0AF
:10CBA00070F803462A46E169A06E02F009F86FF0BA
:10CBB0000607012805D03846BDE8FC816FF001006A
:10CBC000FAE7404603F05DF8024669462046FFF763
:10CBD000E7F8E0690099401CF4F71AFD451C009A3B
:10CBE000216BA818884206D941462046FFF710FC61
:10CBF0006FF00700E0E7002A0EDD404603F041F841
:10CC00000346E069009A4119A06E01F0D9FF00992E
:10CC1000884201D03846CFE7E06900788DF80400FB
:10CC20000198C0F303103060A18C4FF47A70414337
:10CC300004F1740003F00FF80020BDE72DE9F04186
:10CC400005460E4617460024384603F00CF83846D1
:10CC5000E96A03F000F80CE0384603F012F80346E6
:10CC6000286A32460119A86E01F0B9FF002807DDD5
:10CC70000444B44204DA384602F0F8FF0028EBD04E
:10CC8000B4420AD1A98C4FF47A70414305F1700087
:10CC900002F0E1FF0020BDE8F0816FF01200FAE73A
:10CCA00010B5002806D0826A61F341028262C2F3A5
:10CCB000400010BD054B40F28E4205A10EA0F4F7D6
:10CCC0002BFF15A0F4F728FF002010BD5D8301089D
:10CCD0002E2E5C6D717474636C69656E745C6D711D
:10CCE0007474636C69656E745C6D717474636C6983
:10CCF000656E742E6300000025733A256420257349
:10CD000028292E2E2E20636865636B20666F7220A3
:10CD10006572726F722E00000A00000010B50246A4
:10CD20000846002A01D0106010BD064B40F2854233
:10CD300005A10FA0F4F7F0FE15A0F4F7EDFE00201A
:10CD400010BD0000B58201082E2E5C6D71747463F5
:10CD50006C69656E745C6D717474636C69656E7416
:10CD60005C6D717474636C69656E742E6300000091
:10CD700025733A256420257328292E2E2E206368DA
:10CD800065636B20666F72206572726F722E000091
:10CD90000A00000070B504460D4604F15400064632
:10CDA00002F064FE84F84C503046BDE8704002F05A
:10CDB00063BE000010B502460846002A01D0D060CC
:10CDC00010BD064B4FF4916205A10FA0F4F7A4FE2D
:10CDD00015A0F4F7A1FE002010BD0000ED820108AF
:10CDE0002E2E5C6D717474636C69656E745C6D710C
:10CDF0007474636C69656E745C6D717474636C6972
:10CE0000656E742E6300000025733A256420257337
:10CE100028292E2E2E20636865636B20666F722092
:10CE20006572726F722E00000A00000010B5024693
:10CE30000846002A01D0908410BD064B40F28C4277
:10CE400005A10FA0F4F768FE15A0F4F765FE002019
:10CE500010BD00002D8301082E2E5C6D717474636B
:10CE60006C69656E745C6D717474636C69656E7405
:10CE70005C6D717474636C69656E742E6300000080
:10CE800025733A256420257328292E2E2E206368C9
:10CE900065636B20666F72206572726F722E000080
:10CEA0000A00000010B502460846002A01D0906032
:10CEB00010BD064B40F2874205A10FA0F4F72CFEEF
:10CEC00015A0F4F729FE002010BD0000DB82010848
:10CED0002E2E5C6D717474636C69656E745C6D711B
:10CEE0007474636C69656E745C6D717474636C6981
:10CEF000656E742E6300000025733A256420257347
:10CF000028292E2E2E20636865636B20666F7220A1
:10CF10006572726F722E00000A00000010B50246A2
:10CF20000846002A01D0106110BD064B40F289422C
:10CF300005A10FA0F4F7F0FD15A0F4F7EDFD00201A
:10CF400010BD0000FB8201082E2E5C6D71747463AD
:10CF50006C69656E745C6D717474636C69656E7414
:10CF60005C6D717474636C69656E742E630000008F
:10CF700025733A256420257328292E2E2E206368D8
:10CF800065636B20666F72206572726F722E00008F
:10CF90000A0000003EB50C46006A02900190002194
:10CFA00000916FF0180500280BD002A803F004FED2
:10CFB0008DF800000098C0F30311032903D0284620
:10CFC0003EBD28463EBD64F3C30000909DF80010AE
:10CFD00001A80AF04BFA00203EBD000010B5024641
:10CFE0000846002A01D0506010BD064B40F2864230
:10CFF00005A10FA0F4F790FD15A0F4F78DFD00201A
:10D0000010BD0000C88201082E2E5C6D717474631F
:10D010006C69656E745C6D717474636C69656E7453
:10D020005C6D717474636C69656E742E63000000CE
:10D0300025733A256420257328292E2E2E20636817
:10D0400065636B20666F72206572726F722E0000CE
:10D050000A0000004FF47A71484302F01DBE30B55B
:10D0600087B0054600200690059003902846FEF7FD
:10D07000FFFF00280DD1296BE869CDE9000105AB60
:10D0800006AA012104A8F4F749FA012803D06FF099
:10D090000C0007B030BD059880280FD0002403ABEA
:10D0A000BDF8102009212846FEF7DBFC039838B1B3
:10D0B0004CB1FFF730F96FF00E00EAE70124EEE71C
:10D0C0006FF00200E5E701462846FFF777F9E0E751
:10D0D0002DE9F04F89B00646884693461F466FF00B
:10D0E0001304CDF820B0002005900690CDF81080F4
:10D0F0003046FEF7D3FE012803D0A01D09B0BDE8DD
:10D10000F08F06F15000824602F0B0FC3046FEF788
:10D11000E4FE814604A90122CDE9002108A802907D
:10D120004B460022716B306AF4F713FC0546002D64
:10D1300016DD07AA29463046FFF780FD041E0FD1F1
:10D1400007B90B4F59463A464046FFF7CFF860B152
:10D150000090ABB24A4609213046FEF71AFC04465D
:10D16000504602F089FC2046C8E76FF00204F7E75A
:10D170009D2E000870B50446002504F154000646B3
:10D1800002F074FCA06A010A02D0A0F58070A062CF
:10D19000304602F071FC284670BD00007FB5124D8C
:10D1A000124C02E0642009F029FF28782178084316
:10D1B000F8D0FEF7F1FF04460DA0F4F7ADFC002215
:10D1C00004210A200AF09DFA114948600020042138
:10D1D000CDE900100290CA01039023460DA1124828
:10D1E0000AF054FC7FBD0000180000200D00002054
:10D1F0000A77656C636F6D6520746F206D71747450
:10D20000636C69656E7420746573742E2E2E0A002B
:10D21000000000206D7174745F7075626C697368D2
:10D220005F7461736B000000E5C8000810B58A6880
:10D2300049688B181CE014782F2C01D12F291BD1A1
:10D240002B2903D0232901D0A14215D12B2902D0AB
:10D2500023290AD00AE0511C01E0521C511C9942BA
:10D2600004D209782F29F8D100E05A1E401C521C24
:10D27000017809B19A42DED39A4201D1007808B10F
:10D28000002010BD012010BD70B505466FF00304ED
:10D290002846FEF703FE012803D02846FEF757FC78
:10D2A00004463CB9284600F01BF8044600212846F5
:10D2B000FEF797FB204670BD10B50446A26F002A0A
:10D2C00002D02046A16990472046FFF7DDFF0028E5
:10D2D00004D0A06BFFF7BEFE6FF00F0010BD000082
:10D2E0002DE9F04105466FF01408184B40F23B223F
:10D2F00017A121A0F4F710FC29A0F4F70DFC05F10B
:10D3000058000646FEF772FF10B10020BDE8F0811C
:10D31000A86D046840F2472713E0D0E90313027AAE
:10D320002846FFF7D5FE8046163008D1074B3A460F
:10D3300007A11CA0F4F7F0FB19A0F4F7EDFB2046C1
:10D340000468B042E9D14046E0E70000DA81010814
:10D350002E2E5C6D717474636C69656E745C6D7196
:10D360007474636C69656E745C6D717474636C69FC
:10D37000656E742E6300000025733A2564202573C2
:10D3800028292E2E2E206D717474207472792072CB
:10D3900065737562736372696265202E2E2E0000BC
:10D3A0000A00000025733A256420257328292E2EB3
:10D3B0002E206D7174742061636B2068616E646CE3
:10D3C0006572206E756D20746F6F206D75636820B7
:10D3D0002E2E2E001CB50446002000902046FEF79D
:10D3E00047FE002808D16846226BE169F4F7D8F8B7
:10D3F000012802D06FF00B001CBD01ABBDF800206E
:10D400000B212046FEF72DFB0446019818B1FEF7CC
:10D4100082FF20461CBD6FF002001CBD2DE9F041CB
:10D4200007460D4616464FF0FF34304602F01EFC0C
:10D4300040B931463846FFF70BF80446AC4201D0FC
:10D44000002CF2DA2046BDE8F081000070B50446F9
:10D450000D46002C14D0206A08B102F0FDFA656375
:10D46000022D03D96FF07040854202D34FF48060E3
:10D470006063606B02F0E4FA206268B1606B70BDBB
:10D480000C4B40F241420CA115A0F4F745FB1CA047
:10D49000F4F742FB002070BD064B40F24F4206A15C
:10D4A00018A0F4F739FB16A0F4F736FB6FF0020072
:10D4B00070BD0000958201082E2E5C6D717474633E
:10D4C0006C69656E745C6D717474636C69656E749F
:10D4D0005C6D717474636C69656E742E630000001A
:10D4E00025733A256420257328292E2E2E20636863
:10D4F00065636B20666F72206572726F722E00001A
:10D500000A00000025733A256420257328292E2E51
:10D510002E206D616C6C6F63207772697465206278
:10D520007566206661696C65642E2E2E0000000011
:10D53000F8B505460E460024002D01D01EB103E0CB
:10D540004FF0FF30F8BDEE6A684602F08CFB3146C2
:10D55000684602F080FB2CE02846FEF79FFC03287B
:10D5600009D001280CD02846FFF7A6FE044614F186
:10D57000100F1ED102E06FF01700F8BD2046F8BD75
:10D5800069462846FEF764FF0446002C04DB0121AF
:10D590002846FEF726FA0CE014F10E0F0ED1084BC8
:10D5A00040F2993207A111A0F4F7B6FA17A0F4F7E8
:10D5B000B3FA684602F05AFB0028CDD02046F8BDE9
:10D5C000EF8101082E2E5C6D717474636C69656E59
:10D5D000745C6D717474636C69656E745C6D717488
:10D5E00074636C69656E742E6300000025733A25C0
:10D5F0006420257328292E2E2E206D717474206EC0
:10D600006F7420636F6E6E65637400000A00000023
:10D6100070B504462046FEF741FC01280CD01F4B94
:10D6200040F2AB321EA128A0F4F776FA34A0F4F74A
:10D6300073FAE06E02F00CFB40F2B73525E0174BB1
:10D6400040F2B23216A12FA0F4F766FA2CA0F4F73C
:10D6500063FAA06E01F0A6FA2046FEF738FAE46EEF
:10D66000002C1AD0204602F0C0FA2046BDE87040D7
:10D6700002F0F2B9103008D1084B2A4608A12BA0BD
:10D68000F4F74AFA1EA0F4F747FA2046E16AFFF7DA
:10D690004FFF10F1180FEDD1D1E770BDFA810108ED
:10D6A0002E2E5C6D717474636C69656E745C6D7143
:10D6B0007474636C69656E745C6D717474636C69A9
:10D6C000656E742E6300000025733A25642025736F
:10D6D00028292E2E2E2C206D717474206973206ED3
:10D6E0006F7420636F6E6E656374656420746F2061
:10D6F000746865207365727665722E2E2E000000A8
:10D700000A00000025733A256420257328292E2E4F
:10D710002E2C206D71747420636C65616E207365AE
:10D720007373696F6E2E2E2E2E00000025733A251E
:10D730006420257328292E2E2E2C206D71747420C0
:10D740007265636F6E6E6563742074696D656F7565
:10D75000742E2E2E2E00000003460120002201E030
:10D760005843521C8A42FBDB704710B50446002C1C
:10D770000CD0206820B101F0C5FE00206060206060
:10D780002146BDE810400520FDF772BC10BD000029
:10D7900010B50446002C07D0206808B101F0B2FE95
:10D7A00000206060206010BDBDE8104002A385220B
:10D7B00009A110A0F4F7B0B92E2E5C6C7769702D1A
:10D7C000312E342E315C7372635C6170695C6E65FE
:10D7D000746275662E6300006E65746275665F66BE
:10D7E0007265653A20696E76616C6964206275665F
:10D7F00000000000417373657274696F6E2022250A
:10D800007322206661696C6564206174206C696EA6
:10D810006520256420696E2025730D0A0000000034
:10D8200070B504460E461546002C13D0206808B18A
:10D8300001F068FE00210222084601F079FA20601A
:10D8400088B1466020680581206845812068606055
:10D85000002070BD06A398220DA113A0F4F75CF977
:10D860006FF00D0070BD00206060401E70BD0000B4
:10D870002E2E5C6C7769702D312E342E315C7372D4
:10D88000635C6170695C6E65746275662E6300002E
:10D890006E65746275665F7265663A20696E766160
:10D8A0006C69642062756600417373657274696F98
:10D8B0006E2022257322206661696C656420617484
:10D8C000206C696E6520256420696E2025730D0A21
:10D8D00000000000F8B504460D466FF00D06002D5F
:10D8E00022D000202860002C27D004F11400074625
:10D8F00004F0C2F8002829D094F90800761DB0423F
:10D9000011DB69463846E26904F014F8401C26D061
:10D91000E36A1BB1002201212046984700980028A5
:10D920002AD028600020F8BD1AA34FF48F7221A1DD
:10D9300028A0F4F7F1F83046F8BD16A34FF4907222
:10D940002FA124A0F4F7E8F83046F8BD11A340F267
:10D95000211233A11FA0F4F7DFF83046F8BD04F020
:10D9600023F894F908106FF00205B14200DB25722C
:10D9700004F044F82846F8BD04F016F894F90810AD
:10D980006FF00905B14200DB257204F037F8284634
:10D99000F8BD00002E2E5C6C7769702D312E342E70
:10D9A000315C7372635C6170695C6170695F6C6942
:10D9B000622E63006E6574636F6E6E5F6163636594
:10D9C00070743A20696E76616C696420706F696E5C
:10D9D00074657200417373657274696F6E202225DD
:10D9E0007322206661696C6564206174206C696EC5
:10D9F0006520256420696E2025730D0A0000000053
:10DA00006E6574636F6E6E5F6163636570743A20F8
:10DA1000696E76616C696420636F6E6E0000000051
:10DA20006E6574636F6E6E5F6163636570743A20D8
:10DA3000696E76616C6964206163636570746D62A0
:10DA40006F7800002DE9F04106460F460620FDF7ED
:10DA50008FFB044664B100252572267065600026A0
:10DA600004F10C000021804604F010F860B902E0D7
:10DA70000020BDE8F081314604F1100003F0D0FF32
:10DA800040B1404603F0FFFF21460620FDF7F0FAC3
:10DA90000020EEE704F1140003F0DDFF65704FF0A5
:10DAA000FF30A061E762A5626562E56184F82050FD
:10DAB0002046DEE730B587B00446002C16D010486B
:10DAC000019002940491ADF8142001A808F064F8C4
:10DAD000054603F069FF94F9081011F1090F00DB06
:10DAE000257203F08BFF284607B030BD05A3AB229B
:10DAF0000CA113A0F4F710F86FF00D00F4E700008C
:10DB0000A55700082E2E5C6C7769702D312E342EAF
:10DB1000315C7372635C6170695C6170695F6C69D0
:10DB2000622E63006E6574636F6E6E5F62696E6411
:10DB30003A20696E76616C696420636F6E6E0000D6
:10DB4000417373657274696F6E202225732220669B
:10DB500061696C6564206174206C696E6520256460
:10DB600020696E2025730D0A0000000030B587B0D3
:10DB70000446002C16D01048019002940491ADF890
:10DB8000142001A808F008F8054603F00DFF94F9E9
:10DB9000081011F1090F00DB257203F02FFF284652
:10DBA00007B030BD05A3C5220CA114A0F3F7B4FF44
:10DBB0006FF00D00F4E70000595A00082E2E5C6C3F
:10DBC0007769702D312E342E315C7372635C617015
:10DBD000695C6170695F6C69622E63006E65746375
:10DBE0006F6E6E5F636F6E6E6563743A20696E76FA
:10DBF000616C696420636F6E6E0000004173736531
:10DC00007274696F6E2022257322206661696C65CB
:10DC100064206174206C696E6520256420696E2023
:10DC200025730D0A0000000010B586B00446002CD4
:10DC30000BD0074800900194684607F0ADFF2046DE
:10DC400000F09CF8002006B010BD0020FBE70000AB
:10DC5000C55C0008F8B5044604F11000064603F060
:10DC60000BFF30B911E02078102816D00098FFF78C
:10DC70007CFD6946304603F087FE401CF3D13046F8
:10DC800003F0C4FE304603F0E6FE04F1140006463D
:10DC900003F0F2FE002825D1F8BD009D002DE8D04C
:10DCA000606810B1298906F029FC284601F02AFC99
:10DCB000DFE7009D606848B1007E012806D010A310
:10DCC00040F2D22216A122A0F3F726FF2846FFF742
:10DCD000C1FF686818B104F027F900206860284681
:10DCE00000F04CF86946304603F04EFE401CE0D18F
:10DCF000304603F08BFE304603F0ADFEF8BD000069
:10DD00002E2E5C6C7769702D312E342E315C73723F
:10DD1000635C6170695C6170695F6D73672E63003D
:10DD20007063622D3E7374617465203D3D204C49E3
:10DD30005354454E202863616C6C656420666F7295
:10DD40002077726F6E67207063623F2900000000C9
:10DD5000417373657274696F6E2022257322206689
:10DD600061696C6564206174206C696E652025644E
:10DD700020696E2025730D0A0000000070B504466E
:10DD80006068002806D017A340F293221DA129A0A5
:10DD9000F3F7C2FE04F1100003F06EFE002806D077
:10DDA00010A34FF425722EA122A0F3F7B5FE04F1C3
:10DDB000140003F061FE002806D00AA340F2972267
:10DDC00036A11CA0F3F7A8FE04F10C00054603F0F1
:10DDD0005AFE284603F077FE2146BDE87040062033
:10DDE000FDF746B92E2E5C6C7769702D312E342EDE
:10DDF000315C7372635C6170695C6170695F6D73E3
:10DE0000672E6300504342206D7573742062652055
:10DE10006465616C6C6F6361746564206F757473A5
:10DE200069646520746869732066756E6374696FD0
:10DE30006E000000417373657274696F6E20222555
:10DE40007322206661696C6564206174206C696E60
:10DE50006520256420696E2025730D0A00000000EE
:10DE6000726563766D626F78206D7573742062657C
:10DE7000206465616C6C6F636174656420626566C3
:10DE80006F72652063616C6C696E6720746869737A
:10DE90002066756E6374696F6E0000006163636570
:10DEA00070746D626F78206D757374206265206484
:10DEB00065616C6C6F6361746564206265666F7226
:10DEC000652063616C6C696E672074686973206695
:10DED000756E6374696F6E0030B587B004466FF07D
:10DEE0000D05002C1BD0002921D0002A27D018486E
:10DEF00001900294049105928DF8183001A807F062
:10DF00004BFE054603F050FD94F9081011F1090F7E
:10DF100000DB257203F072FD284607B030BD0DA36B
:10DF20008C2214A11BA0F3F7F7FD2846F5E709A3FF
:10DF30008D2223A117A0F3F7EFFD2846EDE705A3F7
:10DF40008E2227A113A0F3F7E7FD2846E5E700009E
:10DF5000FD5E00082E2E5C6C7769702D312E342EFC
:10DF6000315C7372635C6170695C6170695F6C697C
:10DF7000622E63006E6574636F6E6E5F67657461B9
:10DF80006464723A20696E76616C696420636F6EB6
:10DF90006E000000417373657274696F6E202225F4
:10DFA0007322206661696C6564206174206C696EFF
:10DFB0006520256420696E2025730D0A000000008D
:10DFC0006E6574636F6E6E5F676574616464723AE8
:10DFD00020696E76616C696420616464720000007F
:10DFE0006E6574636F6E6E5F676574616464723AC8
:10DFF00020696E76616C696420706F727400000035
:10E0000070B586B005460C466FF00D06002D1ED08B
:10E01000002C25D00021684603F038FD019000282F
:10E0200013D10295039401A80590CDF810D00122D8
:10E0300002A9104807F0D0FD0021684603F0B9FCA2
:10E04000684603F020FD9DF9040006B070BD0AA3E8
:10E0500040F2F72210A119A0F3F75EFD3046F4E775
:10E0600005A34FF43E7220A114A0F3F755FD3046EE
:10E07000EBE70000016000082E2E5C6C7769702DC4
:10E08000312E342E315C7372635C6170695C617037
:10E09000695F6C69622E63006E6574636F6E6E5F9C
:10E0A000676574686F737462796E616D653A206933
:10E0B0006E76616C6964206E616D65004173736595
:10E0C0007274696F6E2022257322206661696C6507
:10E0D00064206174206C696E6520256420696E205F
:10E0E00025730D0A000000006E6574636F6E6E5F2D
:10E0F000676574686F737462796E616D653A2069E3
:10E100006E76616C696420616464720030B587B0BA
:10E110000446002C13D00E480190029401A807F089
:10E120003BFD054603F040FC94F9081011F1090F7E
:10E1300000DB257203F062FC284607B030BD05A362
:10E14000FA220CA113A0F3F7E7FC6FF00D00F4E73F
:10E15000296000082E2E5C6C7769702D312E342ECC
:10E16000315C7372635C6170695C6170695F6C697A
:10E17000622E63006E6574636F6E6E5F6C6973749C
:10E18000656E3A20696E76616C696420636F6E6EAD
:10E1900000000000417373657274696F6E20222560
:10E1A0007322206661696C6564206174206C696EFD
:10E1B0006520256420696E2025730D0A000000008B
:10E1C00070B50D4686B01146FFF73CFC0446002CA6
:10E1D00041D0224800908DF80C500194684607F019
:10E1E000DBFC002837D0606828B11DA34F2224A192
:10E1F0002CA0F3F791FC04F10C00054603F06CFC35
:10E2000028B917A3502232A126A0F3F785FC04F108
:10E210001000064603F030FC28B911A3512233A1A7
:10E2200020A0F3F779FC04F1140003F025FC28B1D9
:10E230000BA3532233A11BA0F3F76EFC284603F077
:10E2400022FC304603F0E2FB21460620FCF710FFDB
:10E25000002006B070BD2046FBE70000DD6000082E
:10E260002E2E5C6C7769702D312E342E315C7372DA
:10E27000635C6170695C6170695F6C69622E6300E8
:10E2800066726565696E6720636F6E6E207769746C
:10E29000686F75742066726565696E672070636269
:10E2A00000000000417373657274696F6E2022254F
:10E2B0007322206661696C6564206174206C696EEC
:10E2C0006520256420696E2025730D0A000000007A
:10E2D000636F6E6E20686173206E6F206F705F6376
:10E2E0006F6D706C6574656400000000636F6E6E26
:10E2F00020686173206E6F20726563766D626F783F
:10E3000000000000636F6E6E2D3E61636365707484
:10E310006D626F782073686F756C646E277420650A
:10E320007869737400000000F8B505460E466FF07A
:10E330000D04002E12D000273760002D17D005F1F4
:10E34000100003F099FB00281AD02878102821D05B
:10E3500031462846BDE8F84000F0AAB826A340F2AE
:10E36000CD122DA134A0F3F7D7FB2046F8BD22A390
:10E3700040F2CF123BA130A0F3F7CEFB2046F8BD10
:10E380001DA34FF4E8723EA12BA0F3F7C5FB6FF07D
:10E390000C00F8BD00970520FCF7EAFE04465CB1CE
:10E3A0006946284600F084F805469DB121460520BF
:10E3B000FCF75EFE2846F8BD03F0F6FA95F9081062
:10E3C0004FF0FF3411F1090F00DB2C7203F016FB44
:10E3D0002046F8BD009830B907A340F2E51231A1FC
:10E3E00015A0F3F799FB0098206000986060A78162
:10E3F000A76034600020F8BD2E2E5C6C7769702D0C
:10E40000312E342E315C7372635C6170695C6170B3
:10E41000695F6C69622E63006E6574636F6E6E5F18
:10E42000726563763A20696E76616C696420706FFC
:10E43000696E746572000000417373657274696F70
:10E440006E2022257322206661696C6564206174E8
:10E45000206C696E6520256420696E2025730D0A85
:10E46000000000006E6574636F6E6E5F72656376A8
:10E470003A20696E76616C696420636F6E6E00008D
:10E480006E6574636F6E6E5F6163636570743A206E
:10E49000696E76616C696420726563766D626F780F
:10E4A000000000007020213D204E554C4C00000023
:10E4B000F0B587B004460D46002006906FF00D06BB
:10E4C000002D1CD02860002C23D004F1100007463A
:10E4D00003F0D2FA002825D094F90800761DB04246
:10E4E00015DB06A93846E26903F024FA401C23D064
:10E4F000207810282DD00698002854D05AE033A355
:10E5000040F25F1239A141A0F3F706FB304607B095
:10E51000F0BD2EA340F2611247A13CA0F3F7FCFA34
:10E520003046F4E729A34FF4B1724AA137A0F3F7BC
:10E53000F3FA6FF00C00EAE703F036FA94F90810EA
:10E540006FF00205B14200DB257203F057FA28464E
:10E55000DDE794F82000000701D5069860B9464829
:10E5600000900194069810B10089039001E0012009
:10E570000390684607F010FB069808B102891CE07A
:10E58000E36A1BB1002201212046984703F00CFAF0
:10E5900094F908106FF00B05B14200DB257203F00F
:10E5A0002DFA2846B3E709A340F2991233A117A028
:10E5B000F3F7B2FA069800680289E36A13B1012101
:10E5C00020469847069828600020A0E72E2E5C6C15
:10E5D0007769702D312E342E315C7372635C6170FB
:10E5E000695C6170695F6C69622E63006E6574635B
:10E5F0006F6E6E5F726563763A20696E76616C69E4
:10E600006420706F696E74657200000041737365F9
:10E610007274696F6E2022257322206661696C65B1
:10E6200064206174206C696E6520256420696E2009
:10E6300025730D0A000000006E6574636F6E6E5FD7
:10E64000726563763A20696E76616C696420636FE7
:10E650006E6E00006E6574636F6E6E5F61636365FE
:10E6600070743A20696E76616C69642072656376B5
:10E670006D626F7800000000FF6000086275662020
:10E68000213D204E554C4C0010B5002802D0027898
:10E69000102A09D006A340F2B7120DA113A0F3F778
:10E6A0003BFA6FF00D0010BDBDE81040FFF700BF52
:10E6B0002E2E5C6C7769702D312E342E315C737286
:10E6C000635C6170695C6170695F6C69622E630094
:10E6D0006E6574636F6E6E5F726563763A20696E05
:10E6E00076616C696420636F6E6E000041737365C0
:10E6F0007274696F6E2022257322206661696C65D1
:10E7000064206174206C696E6520256420696E2028
:10E7100025730D0A0000000000B587B000280DD059
:10E720000278102A0AD190F82020120706D5044A50
:10E7300001920290049101A807F02EFA07B000BDE3
:10E74000FF60000830B587B00446002C14D00F4895
:10E7500001900294049101A807F01EFA054603F007
:10E7600023F994F9081011F1090F00DB257203F069
:10E7700045F9284607B030BD05A34FF40F720CA130
:10E7800012A0F3F7C9F96FF00D00F3E74761000835
:10E790002E2E5C6C7769702D312E342E315C7372A5
:10E7A000635C6170695C6170695F6C69622E6300B3
:10E7B0006E6574636F6E6E5F73656E643A20696E2A
:10E7C00076616C696420636F6E6E000041737365DF
:10E7D0007274696F6E2022257322206661696C65F0
:10E7E00064206174206C696E6520256420696E2048
:10E7F00025730D0A000000002DE9F04186B00446A3
:10E800000C9D1646002C0FD020786FF005071028BD
:10E8100014D025A340F25E222BA134A0F3F77CF99B
:10E82000384606B0BDE8F0811FA340F25D223AA150
:10E830002EA0F3F771F96FF00D00F2E746B194F8EE
:10E840002000800701D4580704D54FF0010803E0E9
:10E850000020E6E74FF00008B8F1000F00D065B1E6
:10E8600034480090019403918DF814300496684662
:10E8700007F092F9074617B109E03846D1E735B1FC
:10E88000B8F1000F02D00498286000E02E6003F079
:10E890008BF894F9081011F1090F00DB277203F0CF
:10E8A000ADF83846BDE700002E2E5C6C7769702D00
:10E8B000312E342E315C7372635C6170695C6170FF
:10E8C000695F6C69622E63006E6574636F6E6E5F64
:10E8D00077726974653A20696E76616C6964206349
:10E8E0006F6E6E2D3E747970650000004173736524
:10E8F0007274696F6E2022257322206661696C65CF
:10E9000064206174206C696E6520256420696E2026
:10E9100025730D0A000000006E6574636F6E6E5FF4
:10E9200077726974653A20696E76616C69642063F8
:10E930006F6E6E00CD6100082DE9F047DDE908A596
:10E940000A9E04460F4690469946002D05D116A30F
:10E950008F221DA122A0F3F7DFF800206060A060E5
:10E96000E06084F831006062E061C4F820A0DFF864
:10E970009CA09AF8000084F83400401C8AF800003B
:10E9800026614B4642463946204600F042F8204672
:10E99000A84710B10020BDE8F087DAF80400206035
:10E9A000CAF804402046F6E72E2E5C6C7769702D7D
:10E9B000312E342E315C7372635C636F72655C6EF2
:10E9C000657469662E6300004E6F20696E6974205D
:10E9D00066756E6374696F6E20676976656E000098
:10E9E000417373657274696F6E20222573222066ED
:10E9F00061696C6564206174206C696E65202564B2
:10EA000020696E2025730D0A000000001801002007
:10EA1000704770B5064614461D46304600F024F88F
:10EA20002146304600F088F829463046BDE870405F
:10EA300000F013B8014988607047000018010020F9
:10EA400090F83110CA0707D021F0010180F8311089
:10EA5000890601D5F8F72ABC7047002902D0096859
:10EA6000C16070470021FBE770B505460C46002CDD
:10EA700021D02068696888421DD01448006809E0E8
:10EA800001686A68914204D1C66803F04DFA3046C5
:10EA900000E0C0680028F3D10D48006809E007D005
:10EAA000016829B16A68914202D144B121680160CC
:10EAB000C0680028F3D12CB12068686070BD4FF0A9
:10EAC0000001F4E74FF00000F7E7000040010020EC
:10EAD0003C010020002800D0C161704790F831103F
:10EAE000CA0607D521F0100180F83110C16900294C
:10EAF00000D00847704710B5044694F83100C106AD
:10EB000019D440F0100084F83100606A10B120463A
:10EB1000F4F74AFE94F83100C10705D0800603D50A
:10EB2000211D2046F9F70CF8E169002903D02046A1
:10EB3000BDE81040084710BD002902D00968816077
:10EB400070470021FBE790F83110CA070AD141F065
:10EB5000010180F83110CA0604D5890602D5011DCD
:10EB6000F8F7EEBF704710B504460022D4E9000163
:10EB700000F08AFFA060002800DB002010BD10B567
:10EB80000446002C02D0A06800F07CFF4FF0FF305C
:10EB9000A06010BD806800F0BEBF806800F0FBBFC1
:10EBA000FFF7E1BFFFF7EBBF002806D04FF0FF33C0
:10EBB000836001604260002070476FF00100704781
:10EBC000FFF7E8BF10B50446A068002806DB204622
:10EBD000FFF7E8FF002020606060A06010BDFFF735
:10EBE000DCBF00221146252000F00EB810B5002130
:10EBF0004FF0006000F060F800220221BDE81040F4
:10EC00003D2000F001B8000070B505460E46002317
:10EC1000002423480168C1F30221072932D001688A
:10EC2000C1F3022106292FD00168C1F30221052971
:10EC30002DD00168C1F3022104292BD00068C0F354
:10EC40000220032829D04FF4A06000F02BF8022303
:10EC50000224C3F104008640C4F104010F20C8401F
:10EC600010403043000105F1E02181F8000405F077
:10EC70001F01012088406909890001F1E021C1F8E4
:10EC8000000170BD0424E4E701230324E1E702232B
:10EC90000224DEE703230124DBE70423D9E7000095
:10ECA0000CED00E00249084302490860704700008B
:10ECB0000000FA050CED00E0034A1140014303484F
:10ECC0000160BFF34F8F704780FFFF1F08ED00E02A
:10ECD00038B504460D4629462046F1F70AFB28467A
:10ECE000F1F719FB29462046F1F703FB04462846B5
:10ECF000F1F711FB204400900A226946F1F778FCF5
:10ED000038BD000070B50D4616462946F1F7F1FAF8
:10ED100004462846F1F7FFFA20443246BDE8704029
:10ED200001A1F1F733BB0000255B5E225D2C0000E2
:10ED30002DE9F05F0D46904600280ED001280ED038
:10ED400002280ED003280ED076A3E8227DA184A04D
:10ED5000F2F7E2FE0020BDE8F09F362604E022260E
:10ED600002E00E2600E000264FF0010B4FF0000AF3
:10ED7000B8F1000F7CD0B8F1010F7AD0B8F1020FD2
:10ED8000FBD0B8F1030F08D066A34FF4AA727FA19D
:10ED900073A0F2F7C1FE0020DDE70C20FCF7E8F9D4
:10EDA000044620001AD084F80C80C4F800A0A019F2
:10EDB000133020F003006060800705D059A3FA22C9
:10EDC00079A167A0F2F7A8FE2581F61C26F00300C2
:10EDD000C0F5FA76AE4203DD284602E00020BAE72D
:10EDE000304680B26081616804F501790844484585
:10EDF00006D94CA34FF4807277A159A0F2F78CFE8C
:10EE0000002E06DC47A340F2031280A154A0F2F7C3
:10EE100083FEA4F80EB0274660892E1A3FE00C202E
:10EE2000FCF7A6F9054628003CD085F80C8085F84B
:10EE30000DA0C5F800A03D604FF6FF70864206DBCE
:10EE400038A34FF48F727EA145A0F2F765FEB0B2F1
:10EE500028814FF4FA71884200D30846688105F191
:10EE600010006860800709D02EA340F2231201E051
:10EE70001DE041E077A13AA0F2F74EFE618960689B
:10EE80000844484506D927A340F2251252A134A0D0
:10EE9000F2F742FEA5F80EB06889361A2F46002E0A
:10EEA000BDDC36E0204600F02DFB002053E706F1E4
:10EEB000130020F00301E81C20F00300084480B296
:10EEC000FBF7F6FE0446200014D0A019133020F002
:10EED0000300606025816581C4F800A084F80CA05F
:10EEE000800716D00FA34FF49F7266A11CA0F2F703
:10EEF00013FE0EE000202EE70B20FCF739F9044644
:10EF00006CB1C4F804A025816581C4F800A084F820
:10EF10000C80A4F80EB084F80DA020461BE700205A
:10EF200019E700002E2E5C6C7769702D312E342E7F
:10EF3000315C7372635C636F72655C706275662EC0
:10EF400063000000706275665F616C6C6F633A20ED
:10EF50006261642070627566206C61796572000080
:10EF6000417373657274696F6E2022257322206667
:10EF700061696C6564206174206C696E652025642C
:10EF800020696E2025730D0A00000000706275660E
:10EF90005F616C6C6F633A206572726F6E656F753E
:10EFA0007320747970650000706275665F616C6CC7
:10EFB0006F633A207062756620702D3E7061796CC7
:10EFC0006F61642070726F7065726C7920616C691A
:10EFD000676E656400000000636865636B20702DD8
:10EFE0003E7061796C6F6164202B20702D3E6C65E2
:10EFF0006E20646F6573206E6F74206F7665726625
:10F000006C6F7720706275660000000050425546B4
:10F010005F504F4F4C5F42554653495A45206D75DE
:10F020007374206265206269676765722074686125
:10F030006E204D454D5F414C49474E4D454E540065
:10F0400072656D5F6C656E203C206D61785F753117
:10F05000365F7400706275665F616C6C6F633A2036
:10F060007062756620712D3E7061796C6F616420ED
:10F0700070726F7065726C7920616C69676E65641F
:10F0800000000000706275665F616C6C6F633A200F
:10F09000706275662D3E7061796C6F61642070726C
:10F0A0006F7065726C7920616C69676E65640000D1
:10F0B00070B50D46002802D00DB104460DE0BDE844
:10F0C000704014A340F2ED221AA128A0F2F724BD4B
:10F0D00021892A8911442181044620680028F7D11A
:10F0E00020896189884206D00AA340F2F6222AA12B
:10F0F0001EA0F2F711FD206830B106A340F2F722FE
:10F1000031A11AA0F2F708FD20892989084420813D
:10F11000256070BD2E2E5C6C7769702D312E342EDB
:10F12000315C7372635C636F72655C706275662ECE
:10F1300063000000286820213D204E554C4C2920BA
:10F14000262620287420213D204E554C4C2920286D
:10F1500070726F6772616D6D65722076696F6C6138
:10F1600074657320415049290000000041737365A4
:10F170007274696F6E2022257322206661696C6546
:10F1800064206174206C696E6520256420696E209E
:10F1900025730D0A00000000702D3E746F745F6CC3
:10F1A000656E203D3D20702D3E6C656E20286F669B
:10F1B000206C617374207062756620696E206368CC
:10F1C00061696E2900000000702D3E6E6578742024
:10F1D0003D3D204E554C4C0010B50C462146FFF7E6
:10F1E00067FF2046BDE8104000F076BB002102E03A
:10F1F000491CC9B200680028FAD1084670470000CF
:10F200002DE9F04705460C46002600276FF00D0952
:10F21000002D04D01CB128892189884209D238A345
:10F220004FF457723EA14AA0F2F776FC4846BDE87B
:10F23000F0876FF0050A68896189801BC91B8842C5
:10F2400002DB1FFA81F801E01FFA80F8606842468D
:10F25000C11968683044F1F71CF806EB080086B263
:10F2600007EB080087B26889B04206D224A340F2B7
:10F270006D3242A136A0F2F74FFC6089B84206D247
:10F280001FA340F26E3243A131A0F2F745FC608922
:10F29000B84201D8002724686889B0420CD1002602
:10F2A0002D684DB944B116A34FF45E7240A128A059
:10F2B000F2F732FC4846BAE774B160892189884286
:10F2C0000AD1206840B10EA340F27D323CA120A0BB
:10F2D000F2F722FC5046AAE775B16889298988426D
:10F2E0000AD1286840B106A340F2823234A118A0A6
:10F2F000F2F712FC50469AE7002C9CD1002096E7CA
:10F300002E2E5C6C7769702D312E342E315C737229
:10F31000635C636F72655C706275662E63000000EB
:10F32000706275665F636F70793A207461726765A9
:10F3300074206E6F742062696720656E6F756768F0
:10F3400020746F20686F6C6420736F757263650042
:10F35000417373657274696F6E2022257322206673
:10F3600061696C6564206174206C696E6520256438
:10F3700020696E2025730D0A000000006F66667319
:10F3800065745F746F203C3D20705F746F2D3E6C20
:10F39000656E00006F66667365745F66726F6D20E0
:10F3A0003C3D20705F66726F6D2D3E6C656E000097
:10F3B000705F746F20213D204E554C4C00000000C2
:10F3C000706275665F636F7079282920646F65735A
:10F3D000206E6F7420616C6C6F77207061636B6559
:10F3E0007420717565756573210A00002DE9F04779
:10F3F000894616464FF00008002805D0B9F1000FE5
:10F400000CD00027044630E01AA340F29D3221A11F
:10F4100028A0F2F781FB0020BDE8F08715A340F299
:10F420009E322FA123A0F2F777FB0020F4E72BB147
:10F430006089984202D8181A83B215E06089C01A10
:10F4400085B2B54200D9354660682A46C11809EB35
:10F450000700F0F71EFF08EB05001FFA80F8781987
:10F4600087B2701B86B2002324680EB1002CDED157
:10F470004046D1E72E2E5C6C7769702D312E342EEC
:10F48000315C7372635C636F72655C706275662E6B
:10F4900063000000706275665F636F70795F706112
:10F4A000727469616C3A20696E76616C696420627D
:10F4B00075660000417373657274696F6E20222552
:10F4C0007322206661696C6564206174206C696ECA
:10F4D0006520256420696E2025730D0A0000000058
:10F4E000706275665F636F70795F70617274696175
:10F4F0006C3A20696E76616C696420646174617035
:10F50000747200002DE9F0410446002C10D0207BDD
:10F5100060B101280AD0022808D0032806D022A30F
:10F5200040F27B2228A12EA0F2F7F6FA00261EE078
:10F530001DA340F2712235A129A0F2F7EDFA0020B7
:10F54000BDE8F08102F030FA0746E08930B916A331
:10F5500040F28A2230A122A0F2F7DEFAE089401EB2
:10F5600085B2E581384602F049FA25B10024002C25
:10F57000E8D13046E4E72568207B03280AD001283B
:10F580000DD002280BD02046FBF79EFA761CF6B26F
:10F590002C46ECE721460C20FBF76AFDF6E72146F6
:10F5A0000B20FBF765FDF1E72E2E5C6C7769702D63
:10F5B000312E342E315C7372635C636F72655C70E4
:10F5C0006275662E63000000706275665F66726524
:10F5D000653A2073616E65207479706500000000E3
:10F5E000417373657274696F6E20222573222066E1
:10F5F00061696C6564206174206C696E65202564A6
:10F6000020696E2025730D0A000000007020213D46
:10F61000204E554C4C000000706275665F66726546
:10F62000653A20702D3E726566203E203000000055
:10F6300070B504460D46002C06D124A340F20522E5
:10F640002AA12DA0F2F768FA002D0FD074B10FDABD
:10F65000684281B2608988420BD21CA340F20D221D
:10F6600030A125A0F2F758FA012070BD002070BD2E
:10F67000A9B2207B626870B103280CD0022813D095
:10F68000012811D011A340F23B222EA11AA0F2F7BB
:10F6900043FA012070BD501B606004F110018842E4
:10F6A00009D26260012070BD002D0CDA60898842A9
:10F6B00009D3501B606060892844608120892844F8
:10F6C0002081002070BD012070BD00002E2E5C6CDA
:10F6D0007769702D312E342E315C7372635C636FE9
:10F6E00072655C706275662E630000007020213DBB
:10F6F000204E554C4C000000417373657274696F65
:10F700006E2022257322206661696C656420617415
:10F71000206C696E6520256420696E2025730D0AB2
:10F7200000000000696E6372656D656E745F6D61E7
:10F73000676E6974756465203C3D20702D3E6C6574
:10F740006E000000626164207062756620747970DA
:10F75000650000002DE9F04704460D46002C06D157
:10F760002BA34FF4DA7232A137A0F2F7D5F9207B40
:10F7700003280BD0012809D040B1022806D024A3C9
:10F7800040F2B5123BA130A0F2F7C6F92089A84299
:10F790003CD92E1A4FF6FF774FF4E6784FF4E8790C
:10F7A00014E0281A85B2BE4205DB19A3424638A1EF
:10F7B00025A0F2F7B1F920893044208124682CB9C2
:10F7C00013A34A4637A120A0F2F7A6F96089A84200
:10F7D000E7D3207B90B96089A8420FD0A088001B96
:10F7E000284481B22046FBF76FFB044634B908A3D6
:10F7F0004FF4ED7231A114A0F2F78EF965812581E5
:10F80000206808B1FFF77EFE00202060BDE8F08789
:10F810002E2E5C6C7769702D312E342E315C737214
:10F82000635C636F72655C706275662E63000000D6
:10F83000706275665F7265616C6C6F633A207020F0
:10F84000213D204E554C4C00417373657274696FB5
:10F850006E2022257322206661696C6564206174C4
:10F86000206C696E6520256420696E2025730D0A61
:10F8700000000000706275665F7265616C6C6F639A
:10F880003A2073616E6520702D3E747970650000BA
:10F8900067726F77203C206D61785F7531365F74D9
:10F8A00000000000706275665F7265616C6C6F636A
:10F8B0003A207120213D204E554C4C006D656D5F06
:10F8C0007472696D2072657475726E656420712042
:10F8D0003D3D204E554C4C0010B50446002C08D040
:10F8E00002F062F8E189491CE181BDE8104002F0B4
:10F8F00085B810BD70B5044620684068002806D061
:10F9000022A34FF4F67229A130A0F2F705F920687E
:10F910004FF0FF35007800F0F000102829D02028A3
:10F9200012D0402802D0FA20207170BD207A00F059
:10F93000F3FE21684860226820B1BDE870402E497E
:10F9400000F000BF257170BD06F06AFF21684860B5
:10F95000216818B10978222902D003E0257170BD11
:10F9600001210174226825495068BDE8704006F005
:10F9700089BF03F06FFB21684860216820B1BDE8B2
:10F980007040084601F0B4BF257170BD2E2E5C6C2E
:10F990007769702D312E342E315C7372635C617027
:10F9A000695C6170695F6D73672E63007063625F8D
:10F9B0006E65773A2070636220616C72656164796C
:10F9C00020616C6C6F6361746564000041737365E2
:10F9D0007274696F6E2022257322206661696C65DE
:10F9E00064206174206C696E6520256420696E2036
:10F9F00025730D0A00000000F1100108D112010862
:10FA000010B540B1017831B10A49F8F7D3FC094982
:10FA100009A0F8F7CFFCF2F7BDF80068F0F770FE28
:10FA20000449F8F7C7FCBDE81040024903A0F8F705
:10FA3000C1BC0000D80100203A2000000A000000EC
:10FA400070B50446204600F0B5FD0546214628461F
:10FA5000F0F738FC284670BD07F03CBA10B50446F4
:10FA6000012007F029FE2060002010BD002300685F
:10FA70005A1E194607F069BE002300681A46194647
:10FA800007F014BFFAF73EB9F0B589B006460F4645
:10FA900014466FF01905202101A8F0F713FC00208F
:10FAA0000290012C06D04FF00100039005D14FF0D9
:10FAB000110004E04FF00200F7E74FF00600049059
:10FAC0006B4601AA39463046FAF7EEF910B12846DE
:10FAD00009B0F0BD009C15E0201D07C8FAF7A8FE8C
:10FAE0000546002D02DA6FF01A050AE0D4E9042178
:10FAF0002846FAF75DF938B12846FFF7C3FF6FF0E3
:10FB00000305E469002CE7D10098FAF7C1F928460B
:10FB1000DEE7FAF7F3BAFEB507460D461646344659
:10FB20004FF47A7093FBF0F1019193FBF0F100FB3D
:10FB300011304FF47A71484302900198002803DB9A
:10FB400006D10298002803DC002001906420029076
:10FB5000082041F20602009001ABD11F384600F0A8
:10FB600014F80EE00023224629463846FFF7D1FF5D
:10FB7000002802DA4FF0FF30FEBD04D0A4EB0004F1
:10FB80000544002CEEDC301BFEBD38B5049C00940F
:10FB9000FAF7FEFC38BDFEB505460E4617464FF493
:10FBA0007A7493FBF4F0019093FBF4F004FB1030B3
:10FBB0002146484302900198002803DB06D10298B1
:10FBC000002803DC0020019064200290082041F20C
:10FBD0000502009001AB911F2846FAF7D9FC3A467E
:10FBE00031462846FAF7EBFEFEBD10B50446002C60
:10FBF00002D0206807F028FA2046BDE81040FFF741
:10FC00002BBF2DE9FF470746DDF830900D469046A3
:10FC10001E460420FFF714FF04460021CDE90141F0
:10FC20000391B2B24346CDF800903946284607F01A
:10FC30002DFF012806D02046FFF70EFF002004B05C
:10FC4000BDE8F0872046FAE7006807F0D9BA7047A8
:10FC5000006807F035BB70B504460D4600F01FF88C
:10FC60002844206070BD00210160704710B5044633
:10FC700000F015F82168884201D9012010BD00204C
:10FC800010BD10B5044600F00AF82168814201D881
:10FC9000002010BD081A10BD014607F0AFB907F0EB
:10FCA0006DBF000070B50446254D2868844205D21A
:10FCB00024A3F1222BA131A0F1F72EFF6868844222
:10FCC00005D320A3F22238A12CA0F1F725FF20793B
:10FCD00028B11CA3F3223BA128A0F1F71DFF208827
:10FCE000B0F5A05F05D917A3F6223DA123A0F1F737
:10FCF00013FF20882968084484420ED0027962B933
:10FD00006A68904209D0AA68824200D1AC60028839
:10FD100022800388621A881C1A5260880844A04214
:10FD20000CD00279002A09D1AA68A24200D1A860A9
:10FD3000228802802288401A891C505270BD00001F
:10FD4000080100202E2E5C6C7769702D312E342E28
:10FD5000315C7372635C636F72655C6D656D2E639D
:10FD600000000000706C75675F686F6C65733A2007
:10FD70006D656D203E3D2072616D000041737365BD
:10FD80007274696F6E2022257322206661696C652A
:10FD900064206174206C696E6520256420696E2082
:10FDA00025730D0A00000000706C75675F686F6C4A
:10FDB00065733A206D656D203C2072616D5F656EE4
:10FDC00064000000706C75675F686F6C65733A2043
:10FDD0006D656D2D3E75736564203D3D20300000DE
:10FDE000706C75675F686F6C65733A206D656D2D1B
:10FDF0003E6E657874203C3D204D454D5F53495A19
:10FE0000455F414C49474E454400000010B504464B
:10FE1000002C06D117A34FF48D721EA121A0F1F77B
:10FE20007BFE6078012802D0042804D006E020463A
:10FE3000F6F74AFA02E02046F5F7E2FC94F82010C3
:10FE4000C80615D5606898B1B0F8662040F66733EB
:10FE50009A420DD9B0F86800052809D221F01000A7
:10FE600084F82000E36A1BB1002202212046984753
:10FE7000002010BD2E2E5C6C7769702D312E342E33
:10FE8000315C7372635C6170695C6170695F6D7332
:10FE9000672E6300636F6E6E20213D204E554C4CE3
:10FEA00000000000417373657274696F6E20222533
:10FEB0007322206661696C6564206174206C696ED0
:10FEC0006520256420696E2025730D0A000000005E
:10FED0002DE9F04107460E461546214800680028E6
:10FEE0003CD007F04BFE1F4CA0600120F8F764FBEC
:10FEF000607890B1D4E90201A0F51C50103881421D
:10FF00000BDC2A463146384600F09CFE304601F0B4
:10FF100077FB07F033FEE0600EE02A4631463846B4
:10FF200000F090FE207838B100202070284601F0C3
:10FF300067FB07F023FEE060012060703046F0F7B9
:10FF4000EAF901463046F0F7BDF92846F0F7E3F943
:10FF500001462846BDE8F041F0F7B4B9BDE8F081AC
:10FF6000000000202000002070B504460B4D2868DA
:10FF70004460E868844206D22968686B091DBDE8C0
:10FF8000704006F069BF2968286B091D06F064FF00
:10FF9000A86A844200D2AC6270BD00007C000020E0
:10FFA00070B58600002908D00D467DB15C2000F0B8
:10FFB00001FB044634B1256309E0304600F0FAFA4B
:10FFC0000546F2E7284606F085FF00E0002424B14C
:10FFD000A5223146206BF0F76EF9204670BD000077
:10FFE00010B506F05DFF0E4C2068A0B90D4806F074
:10FFF00025FF0C48143006F021FF0A48A060143099
:020000040801F1
:10000000E06000220C210A2007F07BFB206010B189
:1000100005A106F0A5FFBDE8104006F04FBF0000A7
:10002000B400002034470020546D725100000000DD
:1000300070B5124E124D1CE007F08CF9306820B1FB
:10004000002407F069FEA4B901E00124F9E706F0F5
:1000500027FFF068C468201D06F091FEA868401EC6
:10006000A8606868401E686006F028FF204600F01F
:1000700055F868680028DFD170BD00000C470020EB
:100080007C00002030B40B46026C002A0CD0C16802
:100090001144C1604468A14201D30168C160C168D4
:1000A00030BC1846F0F7F5B830BC704770B5044660
:1000B00016460025226C002A10D0C6B1E068F0F781
:1000C000E8F8E168206C091AE1602268914202D2E6
:1000D0006168081AE060022E16D01AE02068C0B9E4
:1000E000606807F0ADFD05460020606011E0A06883
:1000F000F0F7CFF8216CA0680844A06061688842DE
:1001000007D32068A06004E0A06B10B1A06B401E74
:10011000A063A06B401CA063284670BD10B50446C8
:10012000206B06F0D7FE2046BDE8104006F0D2BE98
:1001300007498A681168002904D00021016019B1BB
:10014000002070470121F9E7D0680068704700007F
:10015000B40000204FF420410F48420706D0C01DD4
:1001600020F007000C49411AC1F520410B4A1060EC
:10017000002353600144083921F00701103A11604F
:100180004B600B600B1A43600160406890605060E8
:100190004FF00040D06070475C470020E000002036
:1001A000044CFFF745FF20680128FAD906F0CCFE81
:1001B000F7E700005846002070B5044615460020B9
:1001C00023180A5C83F834200A5C12B1401C102802
:1001D000F6D3002684F84360062D00D30525E5629A
:1001E000E5642665201D06F034FE04F1180006F0D3
:1001F00030FE2461C5F10600A0616462666584F882
:10020000586070BD70B50024124D04EB840005EBFE
:10021000800006F013FE641C062CF6D30D487830DF
:1002200006F00CFE0B488C3006F008FE0948A030A2
:1002300006F004FE0748B43006F000FE0548C8305A
:1002400006F0FCFD03490448783101631431416331
:1002500070BD0000584600207C00002030B51349D6
:1002600000E011460A688242FBD34B685C18844266
:1002700003D140681844486008460D684468231854
:10028000AB420DD1094B103B1B689A4206D0526815
:10029000224442600A681268026002E0036000E0E3
:1002A0000260814200D0086030BD0000E000002004
:1002B00070B50024416000610C4D91420AD8D11AFA
:1002C0008269914201D301240EE0011DE86806F025
:1002D000C3FD09E09A4203D2994201D3012403E00D
:1002E000011DA86806F0B8FD204670BDB4000020CE
:1002F00010B5044606F0D4FDA06B20B1002406F032
:10030000DDFD204610BD0124F9E710B5044606F0D6
:10031000C7FDA06BE16B884201D1012400E00024FD
:1003200006F0CCFD204610BDF8B505460E46104837
:100330008068C068C468201D06F021FDE0690128BE
:1003400010D1A0692B46411932462046FFF7B0FF75
:10035000012807D100200346014600902A46204686
:1003600007F04AFD616A01B02046BDE8F040084749
:10037000B400002030B585B0234D3BE00298002842
:1003800038DB049C606910B1201D06F0F8FC01A860
:1003900000F07CF8024602980A282BD2DFE800F031
:1003A0000505052A1F2705052A1F0398A16903468D
:1003B00001442046FFF77CFF01281BD1616A2046DB
:1003C0008847E069012815D1002000900398A169B1
:1003D000002342181946204607F00EFD0AE0039854
:1003E000A061811813462046FFF762FF02E0204615
:1003F00006F070FD00231A4602A9286807F0A5F947
:100400000028BBD105B030BDB4000020F8B50646C9
:100410000D4606F09FFF684600F038F80446009845
:1004200010B107F079FCF8BD45B9A64206D807F02F
:1004300073FC21463046FFF777FFF8BD09481DB130
:10044000C168096861B10025311B2A46006806F0C1
:10045000B5FD07F061FC0028EFD106F075FDF8BD91
:100460000125F1E7B40000200748016B0968002965
:1004700005D0016BC968C9684968816270474FF04F
:10048000FF318162704700007C00002070B5054696
:1004900007F074FB0446074E7068844204D200F0F3
:1004A0000BF80120286001E00020286074602046DD
:1004B00070BD0000B4000020F8B5154E1EE0C06805
:1004C0000568C468201D06F05AFC616A204688470A
:1004D000E069012812D1A0692844A84206D96060C9
:1004E0002461211DB06806F0B7FC07E00020034638
:1004F000014600902A46204607F07EFCB06801685D
:100500000029DCD1B068F168B160F060F8BD00008E
:10051000B4000020EFF76CFEFEE700000021064B60
:1005200042699A4206D1806AA3F12802904201D022
:1005300000B90121084670472047002008B56846E9
:10054000FFF7F6FD0099FFF761FFFFF713FFF6E7EE
:1005500070B5044606F0A4FC04F124050AE0606AC4
:1005600058B1284607F0A4FB08B106F0AFFDA06C17
:10057000401EA064A06C0028F1DC4FF0FF35A5649C
:1005800006F09CFC06F08CFC04F110060AE02069E1
:1005900058B1304607F08CFB08B106F097FD606C4F
:1005A000401E6064606C0028F1DC6564BDE870404A
:1005B00006F084BC2DE9F0410546002606F0CAFE8F
:1005C000234F386808B9FFF7C5FDF868054236D1F2
:1005D0003DB10835680704D005F00700C0F10800F8
:1005E000054465B37868854229D819491031084611
:1005F000046801E0214604466068A84202D22068EF
:100600000028F7D13868844219D00E68083620686F
:1006100008606068411B102904D960194160656059
:10062000FFF71CFE61687868401A7860BA689042EB
:1006300000D2B860F868014361600020206007F0D4
:100640006BFB0EB906F0B6FB3046BDE8F08100004A
:10065000D000002004490868002803D00868026D13
:10066000521C0265086870477C00002020384FF05B
:100670008073C36181610249416140F8202970475C
:1006800015050108002903D00968016000207047A2
:100690000021FAE7002903D0096841600020704773
:1006A0000021FAE72DE9F04780460027D8F804003A
:1006B00090F809900025DFF854A0DAF800401EE019
:1006C000207C484519D12CB1206818B1104909681F
:1006D000884212D1666986B10E4B42462146A06916
:1006E000B04750B14FF00008012735B1E068E8602D
:1006F000DAF80000E060CAF800402546E4680FB967
:10070000002CDDD13846BDE8F08700002401002030
:10071000800100207C01002070B505460020FAF71A
:1007200027FD044654B11C212046EFF7CBFD25746C
:10073000FF20A07202480168E1600460204670BD9D
:1007400024010020416182617047000009490A6864
:10075000824209D1D2680A6008E0D16819B18142A9
:1007600001D1C168D160D268002AF6D101460020CB
:10077000FAF77EBC24010020021D00F001B8000041
:100780002DE9FE4304460E46174614213046FEF777
:100790004FFF4FF0FF3888B1002211460120FEF7CD
:1007A000C7FA05463DB13089002816D031462846A3
:1007B000FEF712FD11E04046BDE8FE8335466FF0BE
:1007C00013012846FEF734FF38B116A3E7221DA116
:1007D00026A0F1F7A1F94046EEE73846F8F7D0FE3B
:1007E000A8B1E4B12168D1B12146227C637ACDE978
:1007F00000320290A37A3A462846F8F71DFE0446D6
:10080000B54202D02846FEF77DFE2046D4E7B54229
:1008100002D02846FEF776FE6FF00300CCE7011DFC
:10082000E3E700002E2E5C6C7769702D312E342E9C
:10083000315C7372635C636F72655C7261772E63A7
:100840000000000043616E277420726573746F723C
:100850006520686561646572207765206A757374C8
:100860002072656D6F7665642100000041737365C9
:100870007274696F6E2022257322206661696C652F
:1008800064206174206C696E6520256420696E2087
:1008900025730D0A00000000034A516821F07061C1
:1008A00001435160704700000010024070B588B0ED
:1008B0000446002046A104AE91E82C00C9682CC66D
:1008C000079144A106C9CDE9021242A106C9CDE9AA
:1008D0000012434D6968C1F38101424B002924D0C5
:1008E000414A012902D0022921D01A466968C1F380
:1008F000031104AB595C22FA01F16B68C3F30223C4
:1009000002AEF35C21FA03F36D68C5F3C2251DF84E
:10091000055021FA05F584B3012C54D0022C54D093
:10092000032C00D1284608B070BD1A46DEE769687E
:1009300001F480314FF4803399421FD1E96A01F00C
:10094000804101B1294AE96A01F4803199420DD10F
:10095000E96AC1F303135B1CE96AC1F30321891C33
:10096000112900D11421B2FBF3F24A43E96A01F0E4
:100970000F01491CB2FBF1F301E022E01C4B696856
:10098000C1F383416A68920001D541F010016A68A1
:10099000520001D541F020010F2901D2891C06E047
:1009A000A1F10F022F2A01D8491C00E03F2103FBCF
:1009B00001F20F299AD103EB4301490001EB5302E5
:1009C00094E71046AFE70846ADE71846ABE70000EE
:1009D00000000000000000000102030406070809EF
:1009E0000010024000127A0040787D01006CDC02A9
:1009F00000093D00064A02EB9011096800F01F0251
:100A000001209040014201D0012070470020704732
:100A100000100240054901EB90110A6800F01F0325
:100A20000120984002430A60704700000010024015
:100A300070B50146002300240020494D4FF40066A4
:100A40001C2970D007DC81B3102912D0182961D07D
:100A50001A2917D16CE0B14215D0B1F5106F45D00D
:100A6000A1F54051103978D130E01120FFF7C2FFD5
:100A70005B1C08B9B342F8D11120FFF7BBFF002877
:100A80006BD0012469E040F601066FF07C4503E07D
:100A90003046FFF7AFFF5B1C08B9AB42F8D13046D8
:100AA000FFF7A8FF08B3012457E0FFE74FF4A06564
:100AB00003E00120FFF79EFF5B1C08B9AB42F8D1B1
:100AC0000120FFF797FF80B1012446E043F21106B1
:100AD00003E03046FFF78EFF5B1C08B9AB42F8D14C
:100AE0003046FFF787FF00B1012436E040F60116DB
:100AF00003E03046FFF77EFF5B1C08B9AB42F8D13C
:100B00003046FFF777FF40B3012426E01920FFF7B6
:100B100071FF5B1C08B9AB42F8D11920FFF76AFFDF
:100B2000D8B1012419E010E01B20FFF763FF5B1C24
:100B300008B9AB42F8D11B20FFF75CFF68B1012474
:100B40000BE01D20FFF756FF5B1C08B9AB42F8D144
:100B50001D20FFF74FFF00B10124204670BD0000AB
:100B6000FFFF0F00054901EB90110A6800F01F0319
:100B70000120984002430A607047000000100240C4
:100B8000054901EB90110A6800F01F03012098400D
:100B900082430A607047000000100240054901EBE3
:100BA00090110A6800F01F030120984002430A6078
:100BB0007047000000100240016811F8012B01602D
:100BC0001046704701684A7811F8023B02EB032295
:100BD000016010467047F0B505460C4616460027E2
:100BE0002068301A01280CDD2046FFF7EBFF686013
:100BF00021680A18B24204D8A9602168084420601C
:100C00000127002028603846F0BD000070B5054679
:100C10000A480468642006F0F1F9601C02D0002143
:100C2000074A07E04FF0FF3070BD8818D0F804087D
:100C30006850091DA142F8D3002070BD0088030848
:100C4000008003082DE9F04F8BB006460F46914611
:100C5000B06904688568DFF8C4A3CEE1707D03281D
:100C600004D0012801D00228F7D1FDE0208C4008F3
:100C70004000F9F7F3FE8346B07DFAF7C1FC6078D7
:100C8000012823D1208C0AAA41082078FAF74EFBCC
:100C900058B19DF8280058B13846EFF73CFB38446E
:100CA000A31C721CDEA1F0F747FF646A54B10DE08B
:100CB0003846EFF730FB3844A31C721CE0A1F0F774
:100CC0003BFFF2E7F669B06904681EB1607803285B
:100CD0000FD057E03846EFF71EFB3844401ED7A12F
:100CE000F0F72AFF5846F7F771FB01200BB0BDE87B
:100CF000F08F208CE18A420820785B46FAF770FB7F
:100D0000B0B3208C042802D0022807D008E0BBF83A
:100D10000080BBF8020048EA000801E0BBF8008050
:100D2000E069404510D09AF80000401C8AF80000A5
:100D30004846EFF7F0FA4844A31C721CC8A1CDF84E
:100D40000080F0F7F9FE0AE03846EFF7E4FA38449D
:100D5000A31C721CC2A1CDF80080F0F7EDFE94F840
:100D6000221041B10A20FCF7F7FCB8FBF0F0E0617B
:100D7000646A1CB106E0C4F81C80F9E7F669B06942
:100D800004681EB16078052815D034E03846EFF7C6
:100D9000C2FA3844401EA9A1F0F7CEFE4846EFF74C
:100DA000BAFA4844401EA5A1F0F7C6FE5846F7F728
:100DB0000DFB01209AE7208C2A4641082078FAF79B
:100DC00025FC48B13846EFF7A6FA3844A31C721C3C
:100DD000AAA1F0F7B1FE08E03846EFF79CFA3844D4
:100DE000A31C721CAEA1F0F7A7FE646A1CB9F669D9
:100DF000B06904681EB1607806280DD023E038463B
:100E0000EFF789FA3844401E8CA1F0F795FE58465A
:100E1000F7F7DCFA012069E7208CE18A42082078A4
:100E20005B46FAF765FC40B13846EFF774FA384490
:100E3000A31C721CA2A1F0F77FFE646A1CB9F669BC
:100E4000B06904681EB15846F7F7C0FAD5E03846D5
:100E5000EFF761FA3844401E78A1F0F76DFE58466E
:100E6000F7F7B4FA012041E7002085F8290008903F
:100E700009900A9005F120000A218346EFF722FA33
:100E800029469948F4F7DFF8707D012802D002283E
:100E900009D010E0012308AA9348E969F4F788F81B
:100EA0004FFA80F807E0022308AA8F48E969F4F7AF
:100EB0007FF84FFA80F8B8F1FF3F47D00A22594631
:100EC00008A8F1F7C1FEE8B3B8F1040F05DC0898F3
:100ED0002862042085F829000CE0B8F1050F36D00F
:100EE00008DD4FF0090208A95846EFF7D2F90920AA
:100EF00085F8290095F8230095F8201040EA01684C
:100F000095F8210095F82210000440EA012048EAF3
:100F100000084846EFF7FFF96A792B79E969CDE9CE
:100F20000518CDE90332AA78E9786B78CDE900326B
:100F3000029148442B78AA1D6C49F0F7FDFD9AF800
:100F4000000000E00DE0401C8AF8000044E0089832
:100F500028629DF8240085F82400052085F82900E2
:100F6000C8E7B8F1040F05DC08982862042085F86A
:100F700029000CE0B8F1050F31D008DD4FF009026F
:100F800008A95846EFF785F9092085F8290095F852
:100F9000230095F8201040EA016895F8210095F8A3
:100FA0002210000440EA012048EA00083846EFF722
:100FB000B2F969792B79EA69CDE90528CDE90331E0
:100FC000A978EA786B78CDE90031029238442B7821
:100FD000AA1D4649F0F7B0FDED6A75B909E0089819
:100FE00028629DF8240085F82400052085F8290052
:100FF000CDE7F669B06985682EB1B06900287FF445
:101000002DAE012072E63846EFF785F93844401ED0
:101010000AA1F0F791FD012068E600002000002001
:101020007B226465766963654964223A22257322CE
:101030002C222573223A6F70656E7D2C0000000013
:101040007B226465766963654964223A22257322AE
:101050002C222573223A636C6F73657D2C0000008F
:101060007B226465766963654964223A222573228E
:101070002C222573223A25647D2C00007B22646596
:10108000766963654964223A222573222C222573EE
:10109000223A20737563636573737D2C0000000032
:1010A0007B226465766963654964223A222573224E
:1010B0002C222573223A206661696C7D2C00000089
:1010C0007B226465766963654964223A222573222E
:1010D0002C222573223A77726974652073756363D5
:1010E0006573737D2C000000C0010020B0880108EA
:1010F0002DE9F04106460F461546002E39D006F17F
:101100001000804600F0B8FC98B329890022032023
:10111000FDF70EFE044644B129462046FEF770F85E
:1011200018B12046FEF7EEF9002414B30520FAF7B3
:101130001FF8054695B12C606C600F480068A860E8
:10114000387CA88124892946404600F087FC50B1AC
:101150002846FCF70AFB0020BDE8F0812046FEF798
:10116000D1F90020F8E7F36A1BB12246002130468E
:1011700098470020F0E700007C0100202DE9F041B5
:1011800004460E4615461F46002E05D124A3DE2236
:101190002BA134A0F0F7C0FC2CB921A3DF223CA185
:1011A00030A0F0F7B9FC6068B04205D01CA3E12282
:1011B0003FA12CA0F0F7B0FC94B104F110008046E0
:1011C00000F05AFC80B100F0EFFB94F9081011F127
:1011D000090F00DB277200F011FC7DB12E890EE0B3
:1011E0006FF00500BDE8F08135B12989304603F084
:1011F00085F92846FEF786F90020F3E70026294600
:10120000404600F02BFC10B14FF0FF30EAE7E36AF4
:101210001BB132460021204698470020E2E700003B
:101220002E2E5C6C7769702D312E342E315C7372EA
:10123000635C6170695C6170695F6D73672E6300E8
:10124000726563765F746370206D75737420686176
:10125000766520612070636220617267756D656ECE
:1012600074000000417373657274696F6E202225EB
:101270007322206661696C6564206174206C696EFC
:101280006520256420696E2025730D0A000000008A
:10129000726563765F746370206D75737420686126
:1012A000766520616E20617267756D656E740000F1
:1012B000726563765F7463703A2072656376206648
:1012C0006F722077726F6E6720706362210000007A
:1012D0002DE9F047DDF8208005460C4616461F46EE
:1012E000002C05D125A39B222CA135A0F0F714FCDE
:1012F0002DB922A39C223DA131A0F0F70DFC686816
:10130000A04205D01DA39E2240A12DA0F0F704FC11
:10131000E5B105F11000814600F0AEFBB0B105204B
:10132000F9F726FF0446B4B126606660C7B1386895
:10133000A060A4F80C8036892146484600F08EFB58
:1013400080B12046BDE8F047FCF70FBA3046BDE853
:10135000F047FEF7D7B83046BDE8F047FEF7D2B801
:101360000020E5E7EB6A002B05D032462846BDE8B1
:10137000F04700211847BDE8F08700002E2E5C6C76
:101380007769702D312E342E315C7372635C61701D
:10139000695C6170695F6D73672E63007265637667
:1013A0005F756470206D7573742068617665206167
:1013B0002070636220617267756D656E7400000055
:1013C000417373657274696F6E20222573222066E3
:1013D00061696C6564206174206C696E65202564A8
:1013E00020696E2025730D0A000000007265637687
:1013F0005F756470206D7573742068617665206117
:101400006E20617267756D656E740000726563763B
:101410005F7564703A207265637620666F7220771C
:10142000726F6E67207063622100000070B5054620
:10143000084600F02DF82020FFF7BCF804462046AF
:10144000EEF769FF01462046EEF73CFF08A4204670
:10145000EEF761FF0246002321462846F8F7A0FF79
:10146000204605F037FD09490120487070BD000095
:101470007B2277726974655F636F6E666967223A73
:101480002273756363657373227D00000C00002076
:101490002DE9FC4780464046EEF73DFF0190274C82
:1014A00020680090642005F0A9FD01984FF0010725
:1014B000810703D007EB900080000190DDE9001068
:1014C000DFF878A081420AF1040A12D007EBD0209D
:1014D00081B27120EFF7D4FE042201A92046EFF774
:1014E000E5FE41465046019AEFF7E0FE0120BDE8D7
:1014F000FC870124DFF848901AE009EB8400D0F85B
:101500000068601E58F82050642005F077FDAE4258
:101510000DD0019807EBD02081B27120EFF7B0FE1B
:1015200041465046019AEFF7C1FE0120DFE7641CF7
:101530000198B4EB900FE0D3D9E7000000880308CE
:1015400000800308F0B589B00546F7F7EFF80446C8
:101550004FF440673846FFF72DF8064639463046C7
:10156000EEF7B0FED4F8E80070B394F8F200E18A28
:10157000D4F8C43004F11802CDE90610CDE90432E4
:1015800094F8F020601C04F1A40104F14A03CDE9B1
:101590000210CDE90032EC341249637930462268FA
:1015A000F0F7CAFA3046F7F713F83046EEF7B3FE15
:1015B0000246002331462846F8F7F2FE09B03046CD
:1015C000BDE8F04005F086BC07A13046F0F7B4FA5C
:1015D0003046EEF7A0FE0246002331462846F8F7D3
:1015E000DFFEEBE7D48601087B22726561645F63EE
:1015F0006F6E666967223A226572726F72227D0091
:10160000F8B50546F7F792F804464FF42F70FEF749
:10161000D1FF06460B48009504F1A40342680AA1D5
:101620003046F0F789FA3046EEF775FE82B204F1E3
:10163000180300213046FBF79FF83046BDE8F8401C
:1016400005F048BC2000002049443A202564207B56
:10165000224445564943454944223A222573222CC7
:101660002264617461223A5B25735D7D0000000095
:1016700070B504461546002C06D117A34FF49F728F
:101680001DA121A0F0F748FA6078012802D00428B3
:1016900004D006E02046F4F717FE02E02046F4F7F7
:1016A000AFF8BCB16068A8B1B0F8661040F6673218
:1016B00091420FD9B0F8680005280BD294F82000A9
:1016C00020F0100084F82000E36A1BB12A460221B2
:1016D00020469847002070BD2E2E5C6C7769702DD7
:1016E000312E342E315C7372635C6170695C6170A1
:1016F000695F6D73672E6300636F6E6E20213D20FE
:101700004E554C4C00000000417373657274696F54
:101710006E2022257322206661696C6564206174E5
:10172000206C696E6520256420696E2025730D0A82
:10173000000000002DE9F14F86B05FA10698FDF78B
:10174000C7FA02905CA10698EEF7D3FD401C5DA19C
:10175000FDF7BEFA044658A10698EEF7CAFD401CF4
:1017600058A1EEF7C6FD401C56A1FDF7B1FA05469B
:1017700051A10698EEF7BDFD401C52A1EEF7B9FD50
:10178000401C50A1EEF7B5FD401C4EA1FDF7A0FA9C
:1017900006464DA10698FDF79BFA01904AA10698CE
:1017A000EEF7A7FD401C47A1FDF792FA074646A1B8
:1017B0000698EEF79EFD401C42A1EEF79AFD401CF4
:1017C00040A1FDF785FA80463FA10698EEF791FD0E
:1017D000401C3CA1EEF78DFD401C3AA1EEF789FDBF
:1017E000401C38A1FDF774FA81463BA10698FDF72D
:1017F0006FFA009038A10698EEF77BFD401C31A1EE
:10180000FDF766FA824634A10698EEF772FD401C99
:101810002CA1EEF76EFD401C2AA1FDF759FA834674
:101820002DA10698EEF765FD401C26A1EEF761FD9F
:10183000401C24A1EEF75DFD401C22A1FDF748FAF3
:1018400001463006EAB240EA0240E2B240EA022231
:101850000298C0B2024305924FEA096008F0FF0205
:1018600040EA0240FAB240EA02220198C0B20243C2
:10187000049208060BF0FF0140EA01400AF0FF0164
:1018800040EA01210098C0B20143039103AB04AACE
:1018900005A91648FDF7BDF81448F2F7B1FE134844
:1018A000FDF751F91148FDF7CBF81048FDF74BF95A
:1018B00007B0BDE8F08F00002269707634223A222A
:1018C000000000002E000000227375626E65744DEA
:1018D00061736B223A2200002264656661756C7444
:1018E00047617465776179223A2200007C09002003
:1018F00010B544680146204600F070FB09492046B7
:1019000002F09EFD0849204602F0CCFF0422074960
:10191000204601F01DFF2046BDE81040044900F0BC
:1019200029BF00007D110108711601080DFE000895
:10193000C16F00082DE9F84304460E46174606F02D
:101940001DF9054606B96E464FF0FF3887B10023F2
:101950003A463146206805F0F8FE012804D0002000
:1019600030604046BDE8F88306F008F9401BF9E70F
:10197000002342463146206805F0E7FE0128F7D1F2
:1019800006F0FCF8401BEDE708B5002900D16946D8
:10199000002300681A4605F0D8FE012802D04FF057
:1019A000FF3008BD002008BD10B505F079FA012010
:1019B00010BD2DE9F04104460E4606F0DFF805465D
:1019C0004FF0FF3776B1002332461946206805F004
:1019D000BCFE012802D03846BDE8F08106F0CEF802
:1019E000401BF9E700233A461946206805F0ADFE92
:1019F0000128F7D106F0C2F8401BEDE705F05EBA0A
:101A00000149002008807047A801002010B5044655
:101A1000206805F0C6F92068BDE8104005F0B2BAAC
:101A200010B5044600220421062005F06AFE20605D
:101A300008B1002010BD4FF0FF3010BD73B5044653
:101A40004FF0FF3500232A4601A9206805F02EFF3C
:101A50000128F7D17CBD00210160704713B5002338
:101A600000681A4601A905F021FF012802D04FF0B5
:101A7000FF301CBD00201CBD0068002801D00120E3
:101A8000704700207047006805F07CBA70B50446C6
:101A90000D4603220021012005F033FE206020B115
:101AA00000231A46194605F001FF206808B11DB150
:101AB00007E04FF0FF3070BD00230122194605F00A
:101AC00044FE002070BD00210160704700230068C3
:101AD0001A46194605F0EABE0068002801D0012028
:101AE000704700207047000070B586B00D46114663
:101AF0000A9A06460C480088062812D2002005AC37
:101B0000CDE9014000929AB203900B463146284637
:101B100005F0BCFF012802D0002006B070BD05987A
:101B2000FBE70020F9E70000A801002070B504469B
:101B30000D4616460920F9F71BFB80B10022026012
:101B40008560C6604460164B1968002910D04A6849
:101B5000A2421DD9121B4A600160186070BDBDE829
:101B6000704010A340F2111218A128A0EFF7D4BFC3
:101B7000186070BD54689C4209D90B681BB153684A
:101B800044681B1B53600A680260086070BD114600
:101B900042684B68D31A43600A68002AEDD0E9E72F
:101BA000000100202E2E5C6C7769702D312E342EB2
:101BB000315C7372635C636F72655C6C7769705FD4
:101BC00074696D6572732E63000000007379735F32
:101BD00074696D656F75743A2074696D656F75749D
:101BE00020213D204E554C4C2C20706F6F6C204DA9
:101BF000454D505F5359535F54494D454F555420FF
